:02000004417049
:10000000070000000300000000000000280070410D
:1000100020F9000020F9000048F9704100000000BC
:1000200048F970410000000010119FE50C219FE588
:1000300008319FE504419FE500519FE5FC609FE585
:10004000F8709FE5F4809FE5F0909FE5ECB09FE5A8
:10005000E8C09FE5E4E09FE500000FE1801080E349
:1000600001F021E1D7F021E3D4D09FE5DBF021E3DB
:10007000D0D09FE5D2F021E3CCD09FE5D3F021E3AF
:10008000C8D09FE5C8009FE5010010E3C4E09F15BC
:10009000C4E09F0510FF2FE178470000BC009FE5FA
:1000A000BC109FE5BC309FE50140A0E30020A0E329
:1000B000010050E104208034004083E5FBFFFF3A5B
:1000C000100F11EEA0109FE5010080E1100F01EE6E
:1000D000100F11EE010A80E3100F01EE8C009FE576
:1000E00010FF2FE1DEEEDEEE78470000101F10EE6D
:1000F0000F1A01E20B0A51E3060000AA0220A0E356
:10010000101E10EE021001E0000051E3FBFFFF1A89
:10011000100E01EE1EFF2FE10222A0E3111E10EED1
:10012000021001E0000051E3FBFFFF1A150E00EE84
:100130001EFF2FE1784700000070A0E117FF2FE1BC
:10014000EFBEADDE48127141481371414811714153
:1001500048397141DF037041990070419C00704142
:1001600048F970411CF6724138A000027820450021
:10017000B3037041794B4FF6FF7210B50AE010F8E7
:10018000014B083984EA122489B233F8144084EA16
:10019000022292B20829F2D2A9B1007841F22103D9
:1001A0004FEA00200AE082EA00044FEA42422404B7
:1001B0004FEA124200D55A404004000C0C00A1F155
:1001C000010189B2EFD1D04380B210BD10B5644CAB
:1001D0004FF6FF7209E010F8013B5340DBB20839DB
:1001E00089B234F8133083EA12220829F3D289B194
:1001F000007848F20843000207E082EA00044FEA70
:100200005202E40700D05A4040080C00A1F101015D
:1002100089B2F2D1D04380B210BD524B6FF0404250
:1002200010B50AE010F8014B083984EA9254E4B2A0
:1002300089B253F8244084EA02220829F2D289B113
:100240000078494B4FEA805007E082EA00044FEA09
:100250004202A40000D55A4040000C00A1F1010167
:1002600089B2F2D1D04320F0404010BD6FF040433E
:1002700083433C4810B50AE011F8014B083A84EA80
:100280009354E4B292B250F8244084EA0323082A3B
:10029000F2D28AB1087834494FEA805007E083EA05
:1002A00000044FEA4303A40000D54B404000140073
:1002B000A2F1010292B2F2D1D84320F0404010BD29
:1002C000C043264B80B210B50AE011F8014B521E14
:1002D00084EA102492B233F8144084EA002080B2F9
:1002E000002AF2D1C04380B210BDC0431C4B80B283
:1002F00010B508E011F8014B4440E4B2521E33F847
:10030000144084EA1020002AF4D1C04380B210BD0A
:1003100003461046154A10B509E013F8014B083999
:1003200084EA106489B252F8244084EA0020082943
:10033000F3D2002910D01A780D4B4FEA026206E082
:1003400090EA02044FEA400000D5584052000C00E9
:10035000A1F1010189B2F3D110BD000010DD70419F
:1003600010DF704110D97041C7B9306010E17041A1
:10037000B71DC10410B504460843800707D0002309
:1003800002E0C85CE0545B1C9342FAD302E02046D2
:100390000CF010ED204610BD10B50D4C20688047C4
:1003A000012805D1606880470028FBD00948046017
:1003B00010BD10B501F004FA074901208863FFF76A
:1003C000EBFF00F055F8BDE8104001F0A3B90000C4
:1003D000E4EC7041A4EB704100A00002FEE71B4971
:1003E00040F2804088634FF0D2510F200863012013
:1003F0001749086470471748016841F0100101600F
:100400001548016821F0030101F101010160134861
:10041000016841F0100101601148016841F01001CC
:1004200001601048016841F0100101600E48016848
:1004300041F01001016042F21070401EFDD20B48E5
:10044000016821F00301491C0160704700000102AE
:1004500000A000026C2190004C269000C026900065
:10046000E026900050269000642690000000301B8B
:1004700030B5FB4C002301202360A38000EB40013A
:1004800001EBC012401C04EBC201A1F5836544F8E6
:10049000325002288B80F1DBF348F249C0E90D139A
:1004A000036401210370C363417030BDEE4A002331
:1004B00010B540F20E44106C8188C91EA14201D3D0
:1004C000838010BDD16B21B10860106CC2E90F03AD
:1004D00010BDD0631364906310BD2DE9F041E34F6C
:1004E0003868C0688047386801697E2088470125E0
:1004F000DFF87483002411E0E043C00602D13868BD
:10050000C0688047DA48065D7E2E1FD07D2E1DD044
:1005100038680169F0B288476D1C641CB8F80A009D
:100520008442E9DB3868C0688047386801697E200A
:1005300088476D1CA80615D1386801697E20884758
:10054000386801697E20BDE8F041084738680169D4
:100550007D208847396886F02000C0B20969884745
:10056000AD1CDAE7BDE8F081002100E0491C10F87D
:10057000012B002AFAD10846704770B504460E4692
:100580000846FFF7F1FF0546304600F03CF8B84852
:100590000D210170210A44708170210CC170210E5F
:1005A000017140F2F9318D4200DD0D463146401DAA
:1005B0002A46FFF7DFFEAC486D1D458100F00CF8C0
:1005C000BDE8704089E70720AAA1FFF7D6FFB3482E
:1005D0004FF001018163FDE710B5A34C40F2FE31FD
:1005E000608988420DD8C004010CA148FFF7EEFDD8
:1005F0009F4A618950540A44000A891C50706181E5
:1006000010BDFFF7E0FF70B50346FFF7ADFF984D53
:1006100004460E20287040F2FC30844200DD04467F
:100620001946681C2246FFF7A5FE641C8E49A0B23D
:100630000A222A54401C4881FFF7CEFFBDE87040D3
:100640004BE770B5884C6169491C6161216C0025DC
:1006500031B9616BC9B121640A6862638D800D6034
:100660007D281AD07E2814D0216C8A88B2F5826F3A
:1006700006D2237813B180F020002570891D5054D4
:10068000206C8188491C818070BDBDE8704084A0C9
:10069000B9E7FFF70BFF257070BD0120207070BD1A
:1006A0002DE9F84F0F46704905464FF0000948699B
:1006B00038444861086C40B9486B98B108640268D6
:1006C0004A63A0F80490C0F8009088460E6C4FF082
:1006D000010A297840F2104B3046B488B61D302903
:1006E00005D03CE06EA0FFF78EFFBDE8F88F3A46DC
:1006F000294687803046FFF73DFEFFF7D7FEF4E737
:100700002A687D200092B0EB126F3DD0C2F3074CF7
:10071000BCF17D0F38D0C2F307207D2834D0D1B290
:100720007D2931D07E23B3EB126F2DD0BCF17E0F2B
:100730002AD07E2828D07E2926D030196946042266
:10074000FFF718FE98F8001029B1315D81F0200103
:10075000315588F80090241DA4B22D1D3F1F042F91
:10076000CEDCC4467F1EC0D328787D283DD07E28AD
:1007700031D05C453DD29CF80010A9B380F0200038
:1007800030558CF8009034E04FF0040C1FE02878CE
:100790007D2815D07E280AD05C4515D298F8002017
:1007A0008AB180F02000305588F800900CE024B128
:1007B000D8F840008480FFF779FE88F8009005E0C3
:1007C00088F800A002E03055641CA4B26D1CBCF196
:1007D000010CDCD2C2E724B1DCF840008480FFF7D2
:1007E00065FE8CF8009006E002E08CF800A002E0C4
:1007F0003055641CA4B26D1CB4E72DE9F0411A4FCA
:100800001C25B869FFF7B0FEB969044602462C48BA
:10081000FFF7B0FD2A4E04F108032A484FF0000804
:100820007A6915E0402C0BDBF869FFF79DFEF9694A
:10083000054602462248FFF79DFD06F8058009E0BF
:1008400022FA05F101F00F012D1F415C3155641CA6
:100850009C42E7DB06F80480BDE8F0411848D2E688
:10086000C0137141D8177141A8EB7041A4EB7041DE
:10087000F41F7141496E7465726E616C206572720D
:100880006F72202D207265706C795F627566666587
:1008900072206F76657272756E00000000A0000213
:1008A0004552523A2057696E646F77206F766572B1
:1008B00072756E2064657465637465642E2E2E00F7
:1008C000F423714110E570410520F1A110B5FFF747
:1008D00054FE002010BD2DE9F0470446F0480025E5
:1008E000007800286BD1EF492022E01D0CF09AF926
:1008F00020B1EDA107E0FFF740FE74E094F8280076
:10090000022802D2EEA10520F5E7A088242802D211
:100910000320F2A1EFE7DFF8ECA30027FA4E202234
:10092000E0494FF00209701C8AF80170213186F805
:100930000090FFF71FFD94F827100420042904D32A
:10094000F249F34A0968914203D0032106F8211FB6
:1009500001E006F8210FB770F0703771777106F873
:10096000019F7771B771F7713772A6F1220600F017
:1009700033FF030023D0FFF7F7FDC2B286F82B2028
:100980002D30B0F5806F31DADF4819462C300CF08D
:1009900012EA96F82B8008F12C0806F8089008F166
:1009A000010806F8087008F10108A8F2FD31494273
:1009B00006EB080000F013FF20B1804403E008209C
:1009C000D4A198E7012594F82900012D00F0090031
:1009D00006F8080008F10108AAF80A8006D0FFF717
:1009E000FBFDFFF77AFD0020BDE8F087FFF7EBFD88
:1009F00070B5841D8088072801D0CDA10FE025792E
:100A0000601C0CF0FDFA65F31F6063790146A07964
:100A100043EA0022551DB5F5806F04D9CAA1032011
:100A2000FFF7ABFD16E0B84804230370637843700A
:100A3000A3788370E378C37023790371401D00F0BD
:100A4000FDFF08B1C5A1EBE7AE484581FFF7C4FD46
:100A5000FFF743FD002070BD00EB4001C4482DE9C5
:100A6000F04300EBC101002587B0087DE0B11822FA
:100A700068460CF00AEABF4C0127A7630E21DDE9A6
:100A8000012000F020FFBE024FF0FF39002830D0D7
:100A90009C48407A042805D0012809D0022809D0B2
:100AA000032809D0B4A108E0012007B0BDE8F08315
:100AB000BAA102E0C5A100E0D1A10720FFF75DFDCA
:100AC0004846F2E7C8F8387034460398A04200D888
:100AD00004460498A2B2294600F099FF08B1D4A1B7
:100AE000EBE704982544204404900398001B0390EE
:100AF00001E00398A0460028E4D100F06EFF00203A
:100B0000D3E7804810B5C1780279114304D00F2093
:100B1000CFA1FFF732FD13E07B4A0C2101241170B5
:100B20004481FFF759FDFFF7D8FC0320FFF794FF3E
:100B3000904884637548006880688047FFF74EFCE2
:100B4000002010BD0520C9A110B5FFF716FD00203B
:100B500010BD2DE9F0410646801DB1880779401C83
:100B6000491F8DB20CF04CFA67F31F60044606F182
:100B70000B007F4E6036317D012910D044EA000120
:100B80002943C90718D006F648032A4601461846E5
:100B9000FFF7F0FB06F648002A4621460EE0F16812
:100BA0002A462944F1603369014618460CF002E9EF
:100BB00030692844306108E02A46214600F027FFCA
:100BC00018B1B1A1FFF7D9FC10E04F48082101701E
:100BD000210A44708170210CC170210E0171052021
:100BE00048494881FFF7F8FCFFF777FC0020B9E49B
:100BF00010B5811D80880A22401E84B242480270CE
:100C000040F2FD32944201D9FFF7DDFC491C224637
:100C1000401CFFF7AFFB3B48641C4481FFF7DCFC42
:100C2000FFF75BFC002010BD3749122010B508709B
:100C3000012034494881152098A1FFF79EFC00202F
:100C400010BD10B52F4CE0782179084306D000F094
:100C5000D0FE30B197A1FFF790FC0BE00F2099A1D7
:100C6000F9E729491E20087001206081FFF7B4FCD4
:100C7000FFF733FC002010BD70B5224DC4792879F0
:100C800020B1A04203D00F2098A14BE144E13FE105
:100C9000496E76616C696420436F6D6D616E6400AE
:100CA000BCEC704121E57041496E76616C6964204D
:100CB0006D61676963206E756D626572000000008A
:100CC000496E76616C69642070726F746F636F6CCB
:100CD0002076657273696F6E00000000506172616A
:100CE0006D6574657220526571756573742050610D
:100CF000636B6574204C656E677468204572726F13
:100D000072000000A8EB7041F41F7141A4EB704128
:100D1000E4EC7041556E7265636F676E697A656465
:100D200020666C6173682064657669636500000005
:100D3000496E76616C6964207061636B6574206CC8
:100D4000656E6774680000005061636B65742074A1
:100D50006F6F206C6172676500000000526561640E
:100D600020756E7375636365737366756C00000040
:100D70004813714100A000024F70656E206D756CC4
:100D80007469206661696C65642C20756E6B6E6F8A
:100D9000776E206572726F72000000004F70656E92
:100DA000206D756C7469206661696C65642C204FD8
:100DB00050454E5F4D554C54495F4C454E47544845
:100DC0005F45584345454445440000004F70656EFB
:100DD000206D756C7469206661696C65642C204FA8
:100DE00050454E5F4D554C54495F5041594C4F4111
:100DF000445F4E4F545F414C4C4F574544000000F8
:100E00004F70656E206D756C7469206661696C65E4
:100E1000642C204F50454E5F4D554C54495F504116
:100E2000594C4F41445F5245515549524544000089
:100E30007A74655F496D6167655F7265636F65723E
:100E40002C207772697465206661696C65640000A6
:100E500043616E6E6F74207265736574206265669F
:100E60006F726520636C6F736500000053696D706D
:100E70006C65207772697465206E6F7420616C6C8C
:100E80006F77656400000000577269746520756EA5
:100E90007375636365737366756C0000506F776577
:100EA00072206F6666206E6F7420737570706F723B
:100EB000746564004572617365206661696C656480
:100EC0000000000043616E6E6F742065726173658F
:100ED000207768656E206E6F742070726576696F1A
:100EE00075736C79206F70656E656400416C726516
:100EF000616479206F70656E656420696E20646935
:100F000066666572656E74206D6F64650000000032
:100F1000F8A0FFF778FB12E0204600F0C4FC20B1F7
:100F20000720FFA1FFF729FB09E014202C71FF49DE
:100F3000087001206881FFF74FFBFFF7CEFA002011
:100F400070BDFB4A012101E0401E91630028FBD1E6
:100F50007047014600E0491C0A78002AFBD1081AB4
:100F6000704770B5F44D0024F2482863E96A8AB2EC
:100F7000214600F06CFCA0B1287A002129610528E7
:100F80000AD0EA491A220A70487002206881FFF7E5
:100F900023FBFFF7A2FA39E00720E8A1FFF7EDFAFB
:100FA00034E0E5484830FFF7D4FF0246E2480E211E
:100FB000483000F088FC002819D0687A042805D051
:100FC000012806D0022807D0032808D0AFF2582104
:100FD00007E0AFF2382104E0AFF2102101E0AFF2F8
:100FE000E0110720FFF7C9FA4FF0FF3070BD00F0A5
:100FF000F4FC2046FFF730FD641C032CF9DB0023D2
:101000006420FFF79EFF5B1C642BF9DB002070BDA2
:1010100070B5D44D0026C84C287840B100F085FB4F
:101020002878042801D1FFF79CFF2E700EE0E078AD
:101030002179084307D000F0D0FC38B1CAA1FFF7EE
:101040009CFA002070BD0F20CBA1F8E7B74916200D
:10105000E6702671087001206081FFF7BDFAFFF786
:101060003CFAEEE710B5C07900F0E6FB18B1CCA170
:10107000FFF783FA0AE0B0490120AC4B1822C860A0
:101080001A704881FFF7A8FAFFF727FA002010BD71
:1010900010B5A94C00F108018088801E82B2E0687A
:1010A000012804D00F20C5A1FFF767FA11E0A1487D
:1010B000C4E90B200BF07EEE012020619B481A2131
:1010C00001700021417002206081FFF785FAFFF76F
:1010D00004FA002010BD2DE9F047DFF85CC20021C2
:1010E000A04F81460B464FF001089CF80720CAB973
:1010F000BF4DA7F16004BF4E01EB4102491C04291A
:1011000004F8323004EBC202C2E903351375C2E9B8
:101110000136F1DB3B70C7E903353B75C7E90136A2
:101120008CF80780B9F1000F1CD03B700722FB60E0
:10113000B1A13B757B600BF075FDB0B1072248464D
:10114000AFA10BF06FFD90B107224846AEA10BF0A6
:1011500069FD78B106224846ADA10BF063FD58B198
:10116000002041E44FF0FF303EE4042000E0032083
:10117000387003E00220FBE787F80080012033E4A9
:101180002DE9F05FC67900F1080B6B4D8088801E59
:101190001FFA80F8E868012801D09FA103E02869C0
:1011A000012804D0A7A10F20FFF7E7F938E058463F
:1011B000FFF791FF5D4F01284FF0020A4FF01C0925
:1011C00012D042463146584600F07DFBD0B1687AD5
:1011D000042805D001281AD0022818D0032816D0D8
:1011E000AFF26C410720DFE75E4C012042465946D2
:1011F000C4F804802075A0680BF0DCEDD4E9011080
:101200000844A060EE70002087F8009001E087F8A5
:1012100000907870A5F80AA0FFF7DEF9FFF75DF9F6
:101220000020BDE8F09F2DE9F041841D477B064674
:10123000201D0BF0E5FE67F31F60E77A054604F119
:1012400008000BF0DDFE014606F1120067F31F6196
:101250008AB2294600F0DBFB18B186A1FFF78DF9B1
:1012600010E0324831210170290A45708170290C43
:10127000C170290E017105202F494881FFF7ACF993
:10128000FFF72BF90020B2E403460020024610B518
:1012900002E010C9521C2044B2EB930FF9D39A0715
:1012A00008D003F003020968C2F10402D2009140A1
:1012B000D140084410BD2DE9F84F817B0024437BC9
:1012C000A046027B43EA012149BA62F31F41C27A78
:1012D000C07B0090234841EA0266007D012801D1CD
:1012E0002048C6604FF0010B134880F806B0009903
:1012F0000229D1E0416C7265616479206F70656E7E
:1013000065642C2069676E6F72696E67206F706507
:101310006E20696E2073616D65206D6F64650000DD
:101320004F70656E206661696C656400F41F7141E1
:1013300000A0000200B07441A8EB7041556E6B6EC6
:101340006F776E206572726F72206163636570746F
:10135000696E6720706172746974696F6E20746160
:10136000626C6500A8137141436C6F736520666100
:10137000696C65640000000043616E6E6F742063E9
:101380006C6F7365207768656E206E6F7420707265
:101390006576696F75736C79206F70656E65640032
:1013A000536574207365637572697479206D6F6419
:1013B00065206661696C65642E0000004E6F2073C5
:1013C00065637572697479206D6F646520726563F9
:1013D0006569766564206265666F7265207061720A
:1013E000746974696F6E207461626C65000000003E
:1013F00000C4744100B47441303A44535031000089
:10140000303A53424C320000303A53424C310000E3
:10141000303A52504D0000004E6F20736563757274
:10142000697479206D6F646520726563656976659E
:1014300064206265666F7265206F70656E206D75E1
:101440006C7469004E6F20706172746974696F6E9C
:10145000207461626C6520726563656976656420DD
:101460006265666F7265206F70656E206D756C7455
:1014700069000000556E6672616D65642073747258
:1014800065616D20777269746520756E737563632D
:1014900065737366756C000002D90020BDE8F88F93
:1014A000DFF8F0A200214162CDE04FF40035AE42FA
:1014B00000D835460098012800D12D1DB64F0020D8
:1014C000D9462921B8624FF08440786403208AF815
:1014D00000108AF801B08AF802B07881FFF77CF832
:1014E000FEF7FBFFCB4687F8059006E0AB480068A7
:1014F000C0688047AA49C1F838B0B86AA842F5D395
:1015000000227A71B86AB946A84221D029238AF804
:1015100000308AF801204D468AF80220AA228AF873
:101520000320020E8AF80420020C8AF80520020A21
:101530008AF806208AF807000820A9F80A00FFF7B1
:101540004BF8FEF7CAFFD5E90901401A68627AE054
:101550000098012810D029218AF800108AF801206B
:1015600003208AF802B0A9F80A00FFF735F8FEF761
:10157000B4FF4FF0844762E0D9F824102923091FF3
:10158000C9F824108AF8003003218AF801208AF86B
:1015900002B0A9F80A10E8E780480068C0688047F0
:1015A0007D4804F58061406A814202D240F20045E4
:1015B00000E0051B7B48017D01290DD0AAB2414600
:1015C000384600F024FA20B3002001280FD0AFF2F3
:1015D0004871FEF7D2FF32E0814600692A4639465B
:1015E0000BF0E8EBD9F810004119C9F810106B485E
:1015F000761B2C442F44A8440068C0688047684983
:10160000C1F838B0644A506A844204D0E00316D16D
:1016100001E00120D9E708218AF800108AF801408A
:10162000210A8AF80210210C8AF80310210E8AF888
:10163000041005205081FEF7CFFFFEF74EFF564DF8
:10164000686A8442A8D3002E7FF42FAF524900204D
:10165000887122E72DE9F047DFF84091D9F80000C2
:10166000C06880474C4F4FF0000A3BE00120B87043
:101670002068B86308B9C7F83CA0C4F800A0386A6D
:10168000F8B14FF00008454610E0D9F80000C068F6
:101690008047A088461B802E00DD802640466119C9
:1016A0003246891DFEF721FE35448046A088A842B7
:1016B000EBDCA8F57061473903D03BA0FEF7A3FF30
:1016C0000DE0A088801EA080A079411E302903D89B
:1016D000797869B101280BD02046FFF7F5F8786BCF
:1016E00020607C63BC6B002CC0D187F802A038E579
:1016F0003249097829B1AFF6E4110820FEF73DFF21
:10170000EDE72549503101EB800050F8041C2046DC
:101710008847E4E7214E0124214D3068C0688047A6
:10172000AC63FFF797FFAC63F7E730B51D4D0024BE
:10173000601E87B02978012906D0022923D0032909
:1017400023D0042923D00446611C1AD0154918223D
:1017500068460BF09AEBDDE903101822401A04905A
:10176000DDE90110401A0F49029004EB4400603992
:1017700001EBC00069460BF088EB0020E86028759B
:10178000686007B030BD0124DEE70224DCE70324F3
:10179000DAE70000F41F7141A8EB7041A4EB70413F
:1017A00000A00002A81371414552523A204352430F
:1017B00020696E76616C696400000000BCEC7041C9
:1017C00010B5A44C02202070A3480168201D884752
:1017D000002800D1207010BD9E48406870479D4A87
:1017E0000346F0B554680020D4E90827A46A01E054
:1017F00052107F00C82AFBDC022505EB82058D42D2
:1018000019D81A546743401CC2F30721FCB219547B
:10181000401C0021C7F30726C7F307453F0E08E029
:101820001C54401C1E54401C1D54401C1F54401C82
:10183000491C9142F4DBF0BD884A012110B5916347
:10184000854949688847002800D0072010BDF8B5B1
:101850000B46114600228DF8002001247F4A946334
:1018600022467D4EB568A847002812D0B2690021F3
:10187000684690477A49052248B99DF80000092832
:101880000AD0232806D0282808D0492808D00A7072
:101890000720F8BD0C70FBE7032002E0022000E007
:1018A00004200870F4E76D4A012110B59163042803
:1018B00007D169490F200022CB68114698470028BC
:1018C00000D0072010BD2DE9F84386460D460020C4
:1018D0008DF80000012161488163AB1E614C032635
:1018E00002204FF00408162B40F2002C65D2DFE8EE
:1018F00003F00B10143135646437333B493F431D0B
:1019000029254D59212D55510AB1207060E0012043
:101910004BE0002AF9D1022047E01AB1624503D911
:10192000217055E0267053E003203EE0002AECD100
:1019300010203AE0002AE8D11B2036E0002AE4D14A
:10194000112032E0002AE0D112202EE0002ADCD162
:101950001C202AE0042028E0052026E0062024E0C0
:10196000002AD2D1082020E0002ACED109201CE094
:10197000002ACAD10B2018E0002AD3D06245CFD864
:101980000D2012E0002AC0D10A200EE0002ABCD1AE
:101990000C200AE0002AB8D11E2006E0002AB4D1AB
:1019A0001D2002E0002AB0D10E202B4E7146F368B4
:1019B000984700280DD00E2D02D084F8008007E053
:1019C000B2690021684690479DF80000402802D087
:1019D0000720BDE8F883052097E770B51F4D012467
:1019E000AC631D4840698047AC63002800D00720E5
:1019F00070BD70B5194D0124AC631748C0698047AC
:101A0000AC63002800D0072070BD0020704770B57F
:101A10000646154814460D460068C26890470E4BAE
:101A200030462A4621461B69984708B1002000E04D
:101A3000012008B1002070BD072070BD30B5002422
:101A4000234603E0CD5C0555641C5B1C9342F9DB27
:101A5000002030BDBCEC7041FCEC704100A00002E5
:101A6000B0EB7041B1EB7041A4EB704135480068B8
:101A700000F08BBC00F02CBA10B5324C02E02068AC
:101A800000F083FC00F066FA0028F8D110BD0120B8
:101A9000704770B506464068022828D12A48007869
:101AA000012802D0F569746918E0F269002A19DD8D
:101AB000264C716920680BF07EE9F06921680144C9
:101AC000216023490A6802440A6022490A681044D6
:101AD000086007E014F8010BFEF7B3FD281EA5F11E
:101AE0000105F7DC3046BDE8704000F06DBA70BD0E
:101AF00038B5002000F032F912490120002300908F
:101B00001548091D1A4600F037F90E4C2060B0B197
:101B1000C068002101F0A2F81049451807E02068CC
:101B200000F033FC2068C06908B1012038BD20688E
:101B30000021C06801F092F8281A0028EFDC00208C
:101B400038BD0000C4EC7041ADEB7041ECEB70416E
:101B5000D0EB7041CCEB7041931A704120A107008B
:101B600070B5514D2C78012C04D0012A04D040F2DC
:101B7000001070BD002070BD4C4C2022C4E907202D
:101B8000C4E9051302F000FEE0690004000CF2D184
:101B90000121297070BD2DE9F0411F2804460E4631
:101BA000904640F200172ED2404D0120A86101F06E
:101BB00016FD40BB0F2C06D00023414601223046C3
:101BC000FFF7CEFFF8B91F2C1DD2DFE804F01C137D
:101BD0001310101010131313131313101C131313DB
:101BE000131C1C1C131313131C1313131300C5F81D
:101BF00014802E622220C5E9064002F0C5FDE86986
:101C000080B2BDE8F0813846FBE710B5274C0123D0
:101C1000E36100232062C4E90332C4E9051302F042
:101C2000B3FDE06980B210BD10B5204C2320E06107
:101C30000020A06102F0A8FDE06980B210BD10B5DF
:101C40001A4C4320E0610020A06102F09DFDE06994
:101C500080B210BD10B5154C0120A0612120E061BB
:101C600002F092FDE06980B210BD70B50F4C0546E0
:101C700049200026C4E9066002F086FDE069B0F55F
:101C8000807F04D0A0692860E06980B270BD2E60BA
:101C9000FAE7064B9A69D2B2027011B10AB1D8695B
:101CA0000860002070470000F8EC7041203372415A
:101CB00070B50546DF48416801290ED0816B0129C6
:101CC0000BD0002101EB810202EBC10200EB820488
:101CD000E26952B1491C0229F4DB70BDD64800F01C
:101CE00054FB95F829000028F7D0204600F049FA67
:101CF0000028F3D170BD012910B50DD0032921D1E1
:101D0000CE4C2178012901D1FFF7D2FFE0680028ED
:101D100018D0BDE810400047C06900210C2803D04E
:101D2000B0F5F07F04D101E0402101E040F2002154
:101D3000C14A503A0B0A50680171437190690171B0
:101D4000090A417110BD00218161BC49496800291F
:101D500000D008477047B94989680847B649C86044
:101D6000704710B504468068FFF7A2FFB3492046CC
:101D70008968BDE8104008472DE9FC47DFF8BC92B0
:101D800082460C4617460A9D984689F8005000F096
:101D90001FF9A94E0CB1B068C461A849343101F1F2
:101DA00090046160C91DA1F11000A161B1314860CA
:101DB000093800F1E2025060123830600120D16031
:101DC00000F0E8FF9C4800F0BAFA4846C9F808A0BD
:101DD00007B14760B8F1000F01D0C9F80C8001A924
:101DE000F0686A4600F019FC9549012700983B46C7
:101DF000884200D000238F48214668388660626898
:101E0000904C92780274A0F5804242610022826177
:101E100080F820704462F5B3DFF818828E468A4954
:101E2000002008F1680941F2000A00EB800404EB8D
:101E3000C00C08EB8C04A660DEF818C09CF802C049
:101E400084F810C009EB003CC4E905CA401C84F8C2
:101E50002020C0B2E26102286162E6D303B3764873
:101E600000F0CCF986F828700022F068012100F01B
:101E700075FE0122F068114600F070FEF068002245
:101E8000022100F06BFEF0680122022100F066FEE4
:101E90006948012100E004E000F005F9012D0ED0B1
:101EA00010E0644C343CA6608869807820746261DC
:101EB000A26184F820206548E2616062CEE7A068F4
:101EC000FFF7F6FE5C48BDE8FC875B4800F063BAAC
:101ED00070B5584C0546683C02E0574800F055FA8A
:101EE00060680128F9D0D4E90520411CA1617E2D4C
:101EF000155402D1A069012803D8A069B0F5804F1C
:101F000004D32046BDE8704000F03BB970BD70B509
:101F1000484C05460E46683C02E0474800F035FA5A
:101F200060680128F9D035B92EB16069324629467A
:101F30000AF040EF00E065612046A66100F021F95B
:101F400002E03D4800F021FA60680128F9D04048DD
:101F5000606170BD374868384068012805D0364850
:101F6000806B012801D000207047012070472DE9C7
:101F7000F041304C06460F46343C254602E02E48E0
:101F800000F003FA68680128F9D0C4E90567204623
:101F900000F0F7F80020BDE8F0810021C161704732
:101FA000264A103200B11081002900D051817047BB
:101FB000002A08D1214A103208B113890380002970
:101FC00001D05089088070470021C16180686FE6A8
:101FD0002DE9F0410225002402F050FC064602F0F3
:101FE00037FC164F103708B1F08978817620F081E0
:101FF000788141F6D2103881304602F034FC00215D
:10200000B0B10E4A032010363874423204E0505505
:102010006D1C51556D1C641C305D08B17F2CF6DBC6
:10202000022000EB44001070034880688262B2E72F
:102030003974B0E79C64714130EE70411CED704121
:10204000EFCDAB00471D7041631D7041571D7041BE
:10205000342471412DE9FC410646C06843689C78F0
:102060008C421DD1D97891421AD1C468002512E062
:1020700061684B790F79887847EA0323CDE9003509
:10208000C978C20901F0030300F00F01B068C0680D
:1020900000F0E8FB2468002CEAD10020BDE8FC81B8
:1020A0004FF0FF30FAE72DE9F047044690F8290099
:1020B00000260F464FF0FF3A10B10FB1B8421AD1C7
:1020C000B84240F200294AD04FF0000817B36568C3
:1020D000084604E069684979814202D02D68002DE4
:1020E000F8D145B1E8680022406881782846FFF7BA
:1020F000B1FF002802DA5046BDE8F08784F8297065
:10210000C4F82480E5626868007A4100204600F047
:102110006EF920E084F8298000212046C4F82C8044
:1021200000F065F90125E0680022294600F0CFFCA7
:10213000E0680022294600F0E6FBE068012229461B
:1021400000F0C5FCE0680122294600F0DCFB6D1CB4
:10215000EDB2032DE7D30321204600F043F9E068F8
:1021600000F097FD28B1012805D0022804D14E4681
:1021700002E0402600E00826304600F092FD0020F4
:10218000BAE7F849016000214160C161816839B155
:10219000CA68C26091F8291031B9017C090703D0DF
:1021A00003214160081F704700F056BC70B5064619
:1021B0001D4634304FF0FF3409B906F1680041681C
:1021C000012904D0C0E90525FFF7DBFF0446201EE6
:1021D00000DB284670BD10B50B46496814008A78AC
:1021E0001C61C06802F00F014FEAD21202D000F069
:1021F00004FB01E000F019FB002010BD70B504469F
:10220000C06802F043FB0546A0690026A8421CD026
:10221000E661B5B364212046666200F0E8F8E06844
:1022200002F042FB28B140F2DC51204600F0DFF81A
:1022300006E00021204600F0DAF8E06802F03AFB00
:1022400000212046A56100F0CDF8E06800F021FDF6
:10225000D0B1012802D0022818D00020E1698142C3
:1022600005D066620121E061204600F0BBF8E0681D
:1022700000F01BFD616A0546A9421AD04DB100214C
:102280000DE0FFE70021D0E70C20E7E740F2E01087
:10229000E4E7E06A0028F2D04068007A4100204676
:1022A00000F0A5F820466562BDE87040052100F009
:1022B00099B870BD10B50446FFF7A0FF0021204675
:1022C000FFF7F1FE002184F82810E06800F089FA99
:1022D0000320E066A06310BD10B50446087810F036
:1022E0001F0004D0012806D0022820D107E0204694
:1022F00000F085F806E0204600F0C6F802E020462F
:1023000000F001F9002809DD04F130022046BDE8A3
:1023100010404FF004034FF0000147E706D120467C
:102320004FF00001BDE8104000F064B806DAE06844
:102330000022BDE81040114600F05FBA10BD70B534
:1023400000258561C561044680F828502946C5628C
:1023500080F8295000F04BF8E463802084F84400B2
:102360000320A56521462467A06384F87850C4F84B
:102370008C50E0667C4AE06800F05FF9E06801227A
:10238000BDE87040002100F02ABC002802D0C068DF
:1023900000F0FAB9704770B5734E00240546361F39
:1023A00003E02846FFF7F1FF641CA86B012802D167
:1023B00030688442F5D300212846FFF774FEE868B0
:1023C00000F0EBFB0020A861E86185F8280070BDF3
:1023D00010B50446FFF7D9FF94F82900002800D073
:1023E000012010BD0269002A00D010477047016229
:1023F0000421F7E700F130020B460121D6E610B5C3
:102400004A780A2A38D2DFE802F0053C373C370F19
:102410001E3C222FCA798B7943EA0221022930D34C
:102420000021018602211CE0CA788B7843EA022150
:1024300090F829202ABBC9B280F82810C06800F0A3
:10244000D0F9002010BDBDE8104000F0A2B8CA7954
:102450008B7953EA022114D090F8291080F83010BB
:102460000121BDE81040C5E7CA788B78BDE810406F
:1024700043EA0221C9B216E6426912B1BDE8104032
:1024800010474FF0FF3010BD034630B44879DC6A86
:102490000A7942EA00254A78E068032A2FD003DC53
:1024A0005AB1012A04D12AE00A2A11D00B2A1CD0E1
:1024B00028B302691AB330BC104700B3C8798979D0
:1024C00041EA002002281AD300201886022109E0E0
:1024D000A8B1CA798C7954EA022110D0007D01217B
:1024E00083F83000184630BC84E744B1C878897856
:1024F00041EA0020C2B22046E9B230BCAAE54FF062
:10250000FF3030BC704730B4034648790C7944EA58
:102510000022D86AC068C06804E04468A478944285
:1025200002D000680028F8D14FF0FF3450B34A7849
:102530004AB1012A1AD0032A1FD00C2A22D0C2681D
:1025400002B330BC1047CA798D7945EA02210229CD
:1025500018D300690221C0F30000188630BC184669
:1025600048E700005155524200EF7041CA788D781B
:1025700055EA022106D1002207E0CA788D7855EA93
:10258000022101D02046BCE70122014630BC18469A
:1025900021E6F0B4CB7800228E1C0546501E012B9C
:1025A0000AD0022B0AD0032B32D14B790C79367822
:1025B00044EA0327AC6818E02A681AE034786B68AC
:1025C00002E01B68641EA4B20BB1002CF9D18BB1E0
:1025D0005A68D078937843EA00200BE02389BB4205
:1025E00002D1A37AB34202D02468002CF6D10CB1F8
:1025F00062681078002A0BD0CB798C7944EA0321E9
:10260000814200DA084603462846F0BC0121CDE5A8
:10261000F0BC7047FF484078704710B5FD4C002370
:10262000A4780CB1FC4805E0FC4B53F8200050F8AE
:10263000803F80680B60106010BD2DE9F041F54EC1
:102640000446002700EB4400B260F54A02EB80002C
:10265000816002F09BF918B1204600F007FC10B928
:10266000204602F043F9ED4D55F82400D0F8A811AA
:1026700021F00301891CC0F8A811204600F0A7FB37
:1026800055F82410E748C1F85801002255F82400F5
:10269000C0F8482155F82400D0F8A81141F00801ED
:1026A000C0F8A81155F82400C0F8AC21082055F84E
:1026B0002410C1F898007078012807D155F824003B
:1026C000D0F8401141F00101C0F840113846BDE892
:1026D000F0812DE9F05FD14951F82000D0F8BCB16C
:1026E000C0F8BCB100274FF0010A002507EB051127
:1026F0000AFA01F01BEA000F31D0CA48402100EB72
:10270000C71000EB851002F039F9C74807EB8711B5
:10271000002600EB8110B04605EB851100EB41145B
:10272000A1462046202102F029F9616808EB1148F2
:102730000EB96068C6B22068012802D02468002C57
:10274000EFD1D9F81C40A169A1EB0801E1616069F2
:1027500002F014F96EB1802E13D0032060606D1C5E
:10276000EDB2012DC2D97F1CFFB2032FBDD3BDE84E
:10277000F09F02206060616A0029F0D020468847FF
:10278000EDE7C4F804A0EAE770B50546A34850F8A1
:10279000250000F5A2700468866E0460600609D505
:1027A0009F4905EB450001EB80009A4980688968E4
:1027B00009688847E00502D5284600F0A6FB6007B7
:1027C00002D5284600F0A1FBE00702D02846FFF71B
:1027D00080FFF00704D02846BDE8704000F055BBEC
:1027E00070BD8E4B4FF0807242EA416253F8200078
:1027F000C0F854218748017070470346002010B587
:1028000019B12AB14FF4803203E04FF0011200E019
:102810000122824C54F8233040F2C01404EB8101B1
:102820005C58944314435C5010BD30B504460020FE
:10283000034629B13AB14FF482024FF4800304E019
:102840004FF0011201E041224023744D55F824401D
:1028500040F2C01505EB81016558134095431D43B7
:10286000655030BD2DE9F0470C00054616461F4661
:10287000DDE9089A4FF0000808D0032C03D2022E9D
:1028800001D2022D04D30320BDE8F0870020FBE72E
:10289000012E284604D000F0E9FA70B100200DE0C6
:1028A00000F0E4FA08B1002001E04FF480005F4935
:1028B00000EB874000F5000005E040204FF6FF7177
:1028C00000EB87008030574A4FEA094302EBC412FD
:1028D00002EB86121360BAF1010F136810D043F0B7
:1028E000005313604D4A40F2C01303EB840352F8C7
:1028F0002520D45808408C430443D4504046C3E7B5
:1029000023F00053EDE70346002030B5032903D23E
:10291000022A01D2022B01D3032030BD414D0024F5
:1029200005EBC11505EB82152C600029F5D0012AB5
:102930000BD08022394C54F8233040F2C01404EB01
:1029400081015C5894435C5030BD4FF40002F1E7C4
:102950002DE9FF4F81B0344900EB801090461E46B0
:102960009B4601EB801002994FF0FF354FF0800A33
:10297000009001EB811100EB411944F200076D1C3E
:10298000BE4200D2374609EB4514202120460AF00A
:10299000C0FA0AEB07406060002D02DDA4F12000C0
:1029A0000460C4F80880A0686FF30B00E060E06882
:1029B00000F58050E060E06800F5805020612069FB
:1029C00000F580506061606900F58050A061F61BE1
:1029D000B84401D03F2DD0DB0E9848B302980128AF
:1029E00031D10C48C16858460AF042EC01BBBBF13A
:1029F000000F28D0681C26D000986D1C202100F5FF
:102A0000026000EB451420460AF083FAC4F804A0E3
:102A1000002D0EE00CEF7041EFCDAB004CEF70419C
:102A20004433724100887141808971410000FFFF89
:102A300009E002DDA4F120000460FF48A060E0602E
:102A400020616061A06101202060606840F4004066
:102A5000606005B0BDE8F08F2DE9FC410446C06818
:102A6000217CD4E9053794F820C001F00F05CE0988
:102A7000032D02D30320BDE8FC81F04940F2C012CF
:102A800002EB850251F820108A58012E4FF4000104
:102A900000D080210A4209D0CDE9007C3246294687
:102AA00000F03DFA20B103216160E4E70720E2E78E
:102AB000012161600021E24AE16105EB851102EB31
:102AC000811106EB861201EB4211CC61D3E72DE9AF
:102AD000F047DFF868A301240646884601EB0210A0
:102AE000914684405AF82600D0F8B871274033D078
:102AF000D44901EBC81101EB8910402101F03EFFE0
:102B0000CF4908EB8810002501EB801109EB8910F3
:102B100001EB4018202108EB451001F02FFF6D1C40
:102B2000412DF7D3D8F81C2053460CE053F826006B
:102B3000C0F8B44153F82610D1F8B4012042FBD1BB
:102B4000D1F8B8712740002FF0D12AB1032050608E
:102B5000516A09B110468847002095E610B5B74C78
:102B600001EB02120121914054F8202009E054F8B1
:102B70002020C2F8B41154F82020D2F8B4310B420E
:102B8000FBD1D2F8B8210A42F1D154F82000D0F894
:102B9000BC11C0F8BC11002010BD70B50025064660
:102BA0000024294622463046FFF791FF641CE4B218
:102BB000022CF6D36D1CEDB2032DF1D300250024B9
:102BC000294622463046FFF79EFE641CE4B2022CE2
:102BD000F6D36D1CEDB2032DF1D3002070BDF0B51E
:102BE0000024022901D2022801D30320F0BD924D16
:102BF0000D3D6B5C0BB10620F0BD4FF040430AB1B8
:102C00004FF041438D4A6FF07F4652F8207049B132
:102C1000C7F8886052F82000C0F88C300120685452
:102C20002046F0BDC7F8806052F82000C0F884301C
:102C3000F4E7022901D2022801D3032070477F4B19
:102C4000002253F8200031B1C0F88C2010467A4B96
:102C50000D3B5A547047C0F88420F7E70022022940
:102C600001D2022801D303207047744B11B101290E
:102C700005D00AE053F82000D0F8840003E053F8B0
:102C80002000D0F88C0020F07F426FF07F40801A47
:102C900070476A4951F82000D0F88401C0F3816080
:102CA000704765491039C8607047644951F8200081
:102CB000D0F8840110F0800000D00120C0B270472D
:102CC0005E4951F82000D0F88401C0F3812070479C
:102CD0005A4951F82000D0F8401141F00101C0F8E4
:102CE000401170472DE9F0474FF08042074602EB54
:102CF0000140524900252C4651F82730C3F8700195
:102D00008846914640F2F41A0AE058F82700D0F8B5
:102D10007051012005F0804601F05CFE4E4503D164
:102D20002046641C5045F0D3C5F30720ACE52DE9DF
:102D3000F04700241D46FF2B06464FF08048894689
:102D4000174606D0FFF7CEFFC0B2A84305EA070238
:102D500002433A4F02EB094000F1C04057F82610F9
:102D6000C1F8700140F2F4190AE057F82600D0F8D3
:102D7000700100F08045012001F02CFE454503D193
:102D80002046641C4845F0D37EE510B501F0F8FDFF
:102D9000C0B210BD284910394870704770B50D4653
:102DA000164600210446FFF744FF01212046FFF7A5
:102DB00040FF224850F82410C1F8805050F82400F9
:102DC000C0F8886070BD1C491039887070472DE9C3
:102DD000F04740F280181B4841460AF09AF843F247
:102DE000C009174849460AF094F8DFF858C0002295
:102DF000DFF84CE0012302EB821000210CEBC2153E
:102E00000EEB801601EB811006EB401405EB8110F0
:102E10008460002004EB40173B60401C4028F9DB35
:102E2000491C0229EEDB521C032AE4DB4FF480002C
:102E3000CCF8000008E000001CEF70414CEF70413E
:102E40008089714100887141CCF84000DCF80000B5
:102E500040F40040CCF800005D48414601F08FFD91
:102E600049465C48BDE8F04701F089BD0CB500213A
:102E700001AA009101916946FFF7CFFB564A012054
:102E80000199914200D000200CBD2DE9F041534D35
:102E90000446012055F82410C1F8AC01504F55F8F4
:102EA0002410D1F8AC0110F0010FFAD1484E06F110
:102EB000280855F82400D0F8401141F40051C0F81A
:102EC00040110821404601F059FDD6E90A01C7E941
:102ED000050155F82400D0F8400110F4005FE8D057
:102EE00055F82400D0F8401121F40051C0F84011E9
:102EF0003C4904EB440001EB8000B96880684A68F3
:102F0000BDE8F041364914311047364900EB400026
:102F100001EB8000324980688968896808472DE99B
:102F2000F84F0C0005462A48174699461A4600EB0A
:102F3000C41000EB87164FF0010004EB0713DDE926
:102F40000AA100FA03F8254B09D153F82500D0F85F
:102F5000AC0110F0010F02D00520BDE8F88FBAF5E2
:102F6000801F01D90320F8E753F825009B46D0F8CD
:102F7000B80110EA080F01D00720EEE753462046BB
:102F800000913946FFF7E4FC124804EB841100EB92
:102F9000811007EB871100EB4117B7600020F0604C
:102FA0005146484601F0EBFC0024202107EB441079
:102FB00001F0E5FC641C412CF7D34021304601F0C0
:102FC000DEFC5BF82510C1F8B0810020C5E70000E9
:102FD0000088714180897141EFCDAB004CEF7041A9
:102FE0000CEF7041443372412DE9F043DFF80C845B
:102FF000012787B04546C8F8387002F089FE0146BF
:10300000FF4E306802F0A1F9AF630446FD4D401C4D
:1030100040F2001910D0F26CA6F58440FA490090F5
:1030200062434B78311D306802F01DFB30B1401D0A
:103030002CD00B20A86128E03220FBE7F348C8F829
:103040003870F34A0168914201D03320F2E74068BA
:10305000F049884201D03420ECE7306804AA2146C8
:1030600001F082FB08B11E20E4E7049802280CD08E
:1030700005A80194012201A9CDE90270306801F090
:1030800070FB002802D00920D4E7484607B0BDE80D
:10309000F0832DE9F04F0446C06F85B00D4616460B
:1030A0004FF0000998B942F2FC502718386828B14F
:1030B000204601F05CFB002808D108E001203860C0
:1030C000204602F06BFB10B1C7F8009080E004F5D9
:1030D0008057DFF83483211DD7F824010095CDE90E
:1030E000016098F80030D4F88020206802F0F8FAE7
:1030F000DFF810B308B10A2126E0D8F818004146DD
:1031000000286DD0CDE903560025C04A28464B461D
:1031100002E0401C02F8013BD4F88CC08445F8D88A
:10312000BD4BBA48D7F824818DE809014B78211DA1
:10313000D4F88020206802F0F1FA40B161680329D8
:1031400001D1401D03D00B21CBF8181040E060687E
:10315000D4F88C3003282ED16EB3B04842F2F4512B
:10316000002600EB010A091D00EB010842F2F051B4
:1031700000EB01090BE0A848FF22DAF80010284410
:103180000844D8F8001009F0BCFE1035761CD9F8B8
:103190000000B042EFD8A04A00210498D7F824617B
:1031A00006E010F8013B12F8015BAB420DD1491C5F
:1031B0008E42F6D8236D0021944A03980EE010F851
:1031C000015B12F8016BB54207D00C20CBF8180058
:1031D00040F2001005B0BDE8F08F491C9942EED3D3
:1031E00004F17C04606800F1010060602068A0F1D7
:1031F000010020604FF00000ECE770B506468848FB
:103200000C461546FF2141F2000201F0F9FB84480B
:10321000002304E054F8231040F823105B1CAB4259
:10322000F8DB76490120002288633046BDE8704013
:103230007B492EE710B50022044600F19001FFF70C
:1032400028FF10B140F2001010BD04F5805400209A
:10325000C4F8AC0210BD2DE9F04F0446C06F002742
:103260000E46C3B090464FF0010A40F2001998B9DB
:1032700042F2FC502518286830B1204601F077FA58
:1032800050B1484643B0A6E72046C5F800A002F07A
:1032900085FA08B12F60F4E7FF22CB4603A8494620
:1032A00009F02FFE0822414603A802F055FAD4F88F
:1032B0008C10002004E056F82020521C03D1401C42
:1032C000B0EB910FF7D3B0EB910F04F580551BD104
:1032D000D5F82411002004E058F82020521C03D116
:1032E000401CB0EB910FF7D3B0EB910F0CD104F170
:1032F0007C04606800F1010060602068401E20606E
:1033000067D1C5F8147164E0D5F8240103AA0096CA
:103310000223211DCDE90120D4F88020206802F08D
:10332000DFF9DFF8E08008B10A2120E0374900200A
:1033300002E0401C01F8017BD4F88C208242F8D8CE
:1033400038490020B946401C402801F8019BFAD3B7
:10335000344902232D48D5F824218DE80700D4F8FC
:103360008020211D206802F0D9F918B10B21C8F87E
:1033700018101DE025490020D4F88C704FF00C0C7B
:1033800006E016F8012B11F8013B9A420ED1401CC1
:103390008742F6D8234A0020D5F8247103A90AE011
:1033A00011F8013B12F8016BB34203D0C8F818C002
:1033B000584667E7401C8742F2D804F17C046068F5
:1033C00000F1010060602068401E206001D1C5F856
:1033D00014910020C5F82CA254E72DE9F0430446CF
:1033E000C06F01260F4693B0914640F2001850BBC3
:1033F00042F2FC5025182868E8B115E000A0000250
:10340000200D72412033724128EF704120CB714171
:1034100033DE01AAAF99FEDB20EB7141E0B17241CE
:1034200020BB714120EC7141204601F0A0F950B160
:10343000404613B02BE620462E6002F0AFF910B1E3
:1034400000202860F4E7FF22402103A809F059FD7D
:1034500004F58055494603A8D5F8242102F07CF9EB
:10346000D5F8240103A900970223CDE90110D4F86F
:103470008020211D206802F033F918B1FF490A208D
:103480008861D5E704F17C04606800F101006060A8
:103490002068A0F1010020604FF00000C5F82C6208
:1034A000C7E72DE9F043F64F012685B00546002415
:1034B00040F200190DF11008BE6318E0286803AA55
:1034C000214601F051F910B1484605B0DFE50398F7
:1034D00002280BD08DE8500128680122694601F0CE
:1034E00040F918B1E54909208861EDE7641CA86C32
:1034F000BE63A042E2D80020E7E72DE9F043E04FA9
:10350000012685B00446E148DEA1BE6301F090FDCE
:10351000DE4D0DF1100840F20019BE631EE0BE63DF
:1035200003AA2868214601F01FF9A0B903980228D0
:1035300013D08DE8500128680122694601F011F985
:1035400058B154B1E00506D1E01704EBD0506FF349
:103550000800201A01904846B7E7641CA86CA042F6
:10356000DDD80020B1E70020C7E738B5C7490446D9
:10357000C74BCA6C58694243A1F54850009001C935
:103580005B78521C02F06FF828B1BC490B208861AF
:103590004FF0FF3038BDBF4D102204F1100105F18E
:1035A000100009F088EBB0B9286A216A884212D16C
:1035B000686A616A88420ED11022B7A104F12C001A
:1035C00009F078EB38B9E96BE06B814203D12A6CE2
:1035D000216C8A4201D0002038BD084438BDA74B79
:1035E0000120A74A30B499699063000219B10129FA
:1035F00001D02A2106E0A64CA268551C07D08A42B9
:1036000003D02B21996130BC70470020FBE7A160FB
:10361000084630BC02F0D7BA2DE9F84FDFF860B2A7
:103620004FF0010A9A4F8046944DCBF838A0B86805
:10363000401C16D0954EFF21A6F58050326D01F04A
:10364000DFF92C6AA6F580500090974920688842DF
:103650000CD1964A6168914208D1A168032905D12D
:1036600001E02C200CE0E16816290BD99049884232
:1036700005D190496068884201D1382000E03520AA
:10368000A8616BE081487FA101F0D2FC08B1022063
:10369000F6E7316D414501D24920F1E7F26E30463F
:1036A0007A61B046326FB9463A615646CBF838A0D7
:1036B0005F4600682146009A01F089FE08B1362075
:1036C000DEE7BE63B246D9F810004E46401C02D178
:1036D0007069401C05D00099204602F049FCA0BB4F
:1036E00002E002F026FCFAE75046B863D146724881
:1036F000D8F85020FF21BA46474601F081F96E48BC
:1037000040F27822009902F027F86C48FF213A6DC8
:10371000A8466D6901F074F968482A46214602F00E
:103720001BF802F09CFB80B9CAF83890C6F80C90E0
:10373000386820F00100416849698847386801F01D
:1037400025FB18B10220C8F8180007E000203860F7
:103750004E484CA101F06CFC002801D040F2001052
:10376000BDE8F88F10B5494C206878B120F0010011
:10377000416849698847206801F008FB20B13F494A
:1037800002208861C00110BD00202060002010BD13
:103790002DE9F84F3A4B0122384907469A630C6AE3
:1037A000C8684D6926180C6920440C68001B411933
:1037B0000091D7F8841009B9C7E921209246114633
:1037C0002F4A07F1900907F580544FF0000B9163E1
:1037D000D7F8881081423AD002D94FF0190122E07F
:1037E000A0EB010830E0D7F88C00D4F8AC12A0EBC5
:1037F000010C4046C44500D38446FF2208E0411C2A
:10380000C4F8AC12A8F10108ACF1010C00F80920D1
:10381000D4F8AC02BCF1000FF1D1D7F88C1088427B
:1038200004D94FF01A01154881617DE00CD114498B
:103830001748C1F838A08078012875D03846FFF7BE
:10384000F9FCE8BBC4F8ACB2B8F1000FCBD1DFF89B
:1038500030A00120CAF838005CE0D7F88C20D4F8FA
:10386000AC02A2EB0008A8452ED948442A463146AE
:1038700001F072FFD4F8AC02284422E020337241F8
:1038800000A00002303A414C4C000000200D724173
:1038900028EF704120DB7141303A53494D5F534569
:1038A00043555245000000009A1B7DAABC487D1F6D
:1038B000AA73EE55DBBD5EE320ED714120FD714141
:1038C00032E0C4F8AC0227E003D110B148442A46E4
:1038D00004E0A8450CD258B148444246314601F0B4
:1038E0003BFF46444946A5EB0805C4F8ACB202E0EC
:1038F00031465618AD1A4FF00108FF48CAF8388013
:103900008078012810D000223846FFF7C2FB58B952
:10391000CAF83880002DA0D1009847F8880FD4F855
:10392000AC027968884202D940F2001018E7002002
:1039300016E72DE9F04FF14B0122F14985B007461A
:103940009A630C6AC8684D6926180C6920440C6893
:10395000001B41190491D7F8841009B9C7E9212047
:1039600092461146E54A07F1900907F580544FF059
:10397000000B9163D7F8881081423AD002D94FF0FA
:10398000190122E0A0EB010830E0D7F88C00D4F850
:10399000AC12A0EB010C4046C44500D38446FF2284
:1039A00008E0411CC4F8AC12A8F10108ACF1010C0C
:1039B00000F80920D4F8AC02BCF1000FF1D1D7F81F
:1039C0008C10884204D94FF01A01CD48816166E01D
:1039D0000CD1CA49C848C1F838A0807801285ED007
:1039E0003846FFF727FCF0BBC4F8ACB2B8F1000FC3
:1039F000CBD1C2490120886347E0D7F88C10D4F8B6
:103A0000AC020A1AAA4290460AD948442A463146CC
:103A100001F0A2FED4F8AC022844C4F8AC0236E0AF
:103A200003D110B148442A4603E0A8450BD250B157
:103A30004844314601F090FE4644CA46A5EB0805CD
:103A4000C4F8ACB203E0B2466D1A01EB0A06DFF827
:103A5000AC820120C8F83800A748807801281ED021
:103A60001020FF2200E01AE0C4F82CB20146C4F88E
:103A70002401684609F045FA6A4651463846FFF780
:103A8000ACFC60B90120C8F83800002DB5D104980D
:103A900047F8880FD4F8AC027968884204D940F21C
:103AA000001005B0BDE8F08F0020FAE72DE9FF5FB8
:103AB000924B0122924907464FF0000A9A630C6A22
:103AC000C8684D6926180C6920440C684021019192
:103AD000001B41190291D7F8841009B9C7E92120C8
:103AE00001219963D7F8881007F1900907F58054F0
:103AF0009B46814238D002D94FF0190122E0A0EB59
:103B000001082EE0D7F88C00D4F8AC12A0EB010C21
:103B10004046C44500D38446FF2208E0411CC4F857
:103B2000AC12A8F10108ACF1010C00F80920D4F89E
:103B3000AC02BCF1000FF1D1D7F88C10884204D947
:103B40004FF01A016E48816196E00AD14FF00100F2
:103B5000CBF838003846FFF76DFB00287ED1C4F85B
:103B6000AC02B8F1000FCDD164490120886341F265
:103B700028103844009075E0019AD7F88C10A2EB19
:103B80000A0B5D4AD4F8AC02A1EB0008D278012AF6
:103B90000DD0A84542462ED948442A46314601F068
:103BA000DBFDD4F8AC022844C4F8AC025CE05D450F
:103BB00018D351484FF000085A4680F80380D4F8D3
:103BC000281200980844314601F0C6FD00980121F2
:103BD00003905E444848A5EB0B05C4F82C82C2460E
:103BE000017126E0D4F828122A460098084431468C
:103BF00001F0B2FD38E003D110B148442A4603E099
:103C0000A84512D288B14844314601F0A5FD3A4892
:103C1000002146444FF0000AA5EB0805C0F81C90AF
:103C2000C4F8AC120121C17003E033486D1AC661BB
:103C30000E44DFF8C8804FF0010B2F48C8F838B0A9
:103C4000017901290ED1002101711021C4F824113C
:103C5000039AC1693846FFF7C0FB00E00CE058B991
:103C6000C8F838B0002D87D1029847F8880FD4F8EB
:103C7000AC027968884204D940F2001004B0BDE873
:103C8000F09F0020FAE70146002007E0303A092AB9
:103C900008D800EB8000491C02EB40000A78002A9B
:103CA000F4D170470020704741F2B94110B5441873
:103CB00000F5805000F52C70002288B00260E17899
:103CC00042EA01610160A37841EA0341016063783F
:103CD00041EA03210160237841EA0301C0E90012AF
:103CE000E17942EA01614160A27941EA0241416021
:103CF000627941EA022105E028EF704100A000024C
:103D0000203372414160227904F1080441EA020142
:103D100041604FF00000694614F8012B0A54401C22
:103D20001828F9DBF8A1684609F01AE9FC4B0100F4
:103D300040F2001001D047210DE0A278002141EAB5
:103D40000241627841EA022221781143A1F5007212
:103D5000013A03D04421996108B010BD0020FBE76F
:103D60002DE9F05F074641F2B9403D1842F23C5060
:103D70004FF00008DFF8AC934FF0450BC2463C58BB
:103D800070E000260EE020B1202802D009F80600DD
:103D9000761CE4486D1C641EE3A109F806A009F036
:103DA000E0E8B0B128783D2801D0002CEBD16D1CA3
:103DB000641E0020B8F1010F58D0DA4A6432297825
:103DC00051B14CB1202901D01154401C6D1C641E0E
:103DD000F5E74FF00108EAE702F800A0D1486D1CB2
:103DE000641ED5A109F0BCE850B9CE486430FFF795
:103DF0004AFF396D814203D0C949C1F818B00EE0BD
:103E0000C848D1A109F0ACE860B9C6486430FFF7F2
:103E10003AFFF96C814205D0C148C0F818B040F2B1
:103E200000102CE7BF48CBA109F09AE830B9BD4893
:103E30006430FFF728FFB96C8142DDD3B948C9A1CE
:103E400009F08EE870B9B7486430FFF71CFFF968D5
:103E5000082902D0102905D102E0082802D0CBE7BA
:103E60001028C9D114B1B8F1000F8AD0002006E79C
:103E700041F2B9412DE9F047421842F23C51DFF8D6
:103E8000A0924FF0000E73464FF0460850F801C064
:103E900040F2001A0021BCF1100F5DD9D4780CF16A
:103EA000040C41EA0461947841EA0441547841EAFF
:103EB000042112F8044B0C43611C44D0202B4BD23C
:103EC00019465B1C00EB011505F5805101F52E71BB
:103ED000ACF1080C0C604FF000044C60D67844EA5A
:103EE00006664E60977846EA07464E60577846EA7F
:103EF00007264E60177846EA0706C1E90164D679BD
:103F000044EA06648C60967944EA06448C605679EB
:103F100044EA06248C60167902F1080244EA060499
:103F20008C604FF0000114786E1806F58056491C1D
:103F3000042986F8C442F6D3121DBEF1000FACF17D
:103F4000040CA7D005E000EB031000F58050C0F88A
:103F5000B8420020BDE8F0875046C9F81880F9E75C
:103F60002DE9F04F87B00546002081494FF0000A47
:103F7000019005F1900005F58059CDE902A00120DE
:103F800088636748026AC168571802691144026869
:103F900040698E1A42F23C5284B23019059041F2C7
:103FA000B840D5F8841005EB000B05F517500690C6
:103FB000A8180490002902D10120C5E921066CE16E
:103FC0009BF8000003286FD04FF0000820B10128B3
:103FD00004D0022822D10CE0242008E0D9F8B00255
:103FE00041F280012438884201D9884616E0804693
:103FF00014E0D9E9AC0141F28002091A914201D9D9
:10400000904600E08846B04208D9811BA14201D900
:10401000002403E0621A064694B20F440498016833
:10402000A8EB0100A04201D9009400E0009041F209
:10403000B9402844009A0844394601F08DFB0498A1
:104040000168009808440499086000990F44611AB7
:104050008CB2009940450E4426D19BF8000088B1EF
:10406000012807D0022814D12846FFF701FF0321B9
:10407000019004E02846FFF773FE022101908BF8BF
:10408000001006E02846FFF70FFE019001208BF894
:104090000000019800286ED10499002C08606BD0B4
:1040A0009BF8000003288BD1D9F8B412B14212D981
:1040B000881BA04260D8221A0E46074494B2069A82
:1040C0000120029005EB0A1000F58050C2F800A014
:1040D000D0F8B802686706986A6FD0F800A005EBC0
:1040E0000A1000F58050D0F8B832D0F8C002D21AC9
:1040F00005EB8A0303F515531B68D21A521C904234
:104100006ED8E86FB0B36BE0496D61676520666992
:104110006C65207769746820686561646572000069
:104120002033724140BA7141656E645F6F665F68AB
:104130006561646572000000706167655F62797433
:1041400065735F7573657200626C6F636B5F70613E
:10415000676573006465766963655F626C6F636B46
:1041600073000000646174615F77696474680000C3
:1041700000A0000231E09DE080E005EB0A1000F5B0
:104180008050D0F8C802421C0AD0D5F88C20504389
:10419000EA6C00FB0210821BA24205D900241FE03A
:1041A0000598C5F8880088E017440646A21A0AF167
:1041B000010A94B2069A05EB0A1000F58050C2F885
:1041C00000A0D0F8B8226A67D0F8C0220AB1012254
:1041D0000292D0F8B802401CE2D002980028CCD05D
:1041E000029801280AD142F2FC516850284601F099
:1041F000D5FAB0F5807F5DD000200290F4B3D5F8F9
:104200008C20D9F8AC02A2EB0008A0450DD9D9F852
:10421000AC12224603980844394601F09DFAD9F8B9
:10422000AC020119C9F8AC123AE004D118B10399F3
:104230002246084405E0A04510D278B103994246D1
:104240000844394601F088FAA4EB0800039984B2C7
:104250000020C9F8AC024744464404E039465718E8
:10426000A01A84B216444FF00108FF4AC2F8388001
:104270006868032807D00022284600E010E0FEF717
:1042800008FFA8B906E0D5E91402131AC9F82431C9
:104290004218F1E7F449C1F83880002C7FF490AE61
:1042A000059845F8880FD9F8AC026968884204D9A6
:1042B00040F2001007B0BDE8F08F0020FAE72DE9CA
:1042C000F04FE94B00F190090746E848012285B01C
:1042D0009A63046AC16865180469214404684069E6
:1042E000091B86B288190290D7F8840007F580541C
:1042F00080B9C7E9212128780621442812D084F802
:1043000011110C20C4F89C020820C4F8A4020F3537
:104310000F3EB6B2D4490120886341F2281007EB62
:10432000000ADBE1072084F81101C4F8A412082078
:10433000C4F89C02EBE7D4F81401002872D1D4F839
:104340009C02B0422BD90120042EC4E9A50619D342
:1043500004F58C74206860604FF000002060E978FC
:1043600040EA01602060A97840EA01402060697855
:1043700040EA01202060297840EA01002060A4F58D
:104380008C74AEE1002007E03A1802F5805215F86F
:10439000011B401C82F8A812B042F5DBA1E1D4F861
:1043A000941201291BD004F58C74216861604FF0D0
:1043B00000012160EA7841EA02612160AA7841EABD
:1043C000024121606A7841EA022121602A7841EAAB
:1043D00002012160A168A4F58C74B1B37EE0D4F829
:1043E0009812421A042944DAD4F81801C4F81C01BE
:1043F00000200129C4F8180128D0022913D003296C
:1044000037D194F8AA1240EA014094F8A91240EA80
:10441000012094F8A8120843C4F81801297840EA4A
:10442000016024E0C6E094F8A91240EA012094F863
:10443000A8120843C4F81801697840EA0160C4F87A
:104440001801297840EA014011E01BE094F8A80225
:10445000C4F81801A97840EA0160C4F81801697825
:1044600040EA0140C4F81801297840EA0120C4F864
:104470001801B01A86B20020C4F894021544C4F89A
:1044800098022EE0EA7941EA0261C4F82011AA7983
:1044900041EA0241C4F820116A7941EA0222C4F8D3
:1044A000202129790A43C4F82021D7F88C10B1F5CE
:1044B000006F04D0B1F5805F01D03F2108E0D4F84F
:1044C000A43219448901C4F8A0128A4203D03E21C3
:1044D000664881610DE10821C4F824110544301AB1
:1044E00086B20120C4F81401C4F82C02D4E9462095
:1044F000D4F82011101A88425AD0EAB308F0B8EE66
:10450000D4F89012401E4FF0000807EB810101F52E
:104510008051D1F83012049194F81121062A03D168
:10452000814201D93C21D3E70190786F401C009073
:10453000002016E04C49012003AA8863796F38688F
:10454000491C00F011F908B11E21C1E703980228A7
:1045500048D0454901208863384600F008F90BF13E
:104560000100834601998B45E4DB0098014401EB8F
:104570000800F96C484300E01AE0B8F1000FC7F8F2
:1045800080000DD0D4F89002049907EB800000F56C
:1045900080504144D0F830228A4201D0C0F8301215
:1045A000D4F89002401CC4F89002384600F0DFF8BE
:1045B000002E2FD0D4F82802D0B1D4F8A412A1EB49
:1045C00000084645504460D34246294601F0C4F8ED
:1045D0004544A6EB080086B20020C4F82C02C4F8BB
:1045E000280260E0786F08F10108401C7867B9E79D
:1045F000D7F88C20D4F8AC02A2EB0008B0450AD959
:1046000048443246294601F0A7F8D4F8AC023044B9
:10461000C4F8AC0265E003D110B14844324604E06E
:10462000B0450DD260B148444246294601F094F8A5
:10463000A6EB080086B20020C4F8AC02454408E0AE
:104640004844294601F088F8D7F88C000544301A10
:1046500086B2054901208863D4F82C0201281FD1B5
:10466000D4F8A422B24203E000A000022033724139
:10467000D4F8281201EB0A0007D8294601F06CF89B
:10468000D4F8A4020544301AA5E73246294601F0C1
:1046900063F8D4F8280235443044C4F828020026D0
:1046A000D4F82C02B8B994F8110107280BD104F5FD
:1046B00096742078A0706078E0704FF0FF00207052
:1046C0006070A4F59674524649463846FEF7C3FD1D
:1046D000B0F5807F0FD0284901208863002E7FF439
:1046E0002AAE029847F8880FD4F8AC02796888425D
:1046F00003D940F2001005B0DDE50020FBE770B5FE
:104700001D4E0124AFF684611C48B46300F090FC98
:104710001B4D18B10220A861C00170BDB4632022F6
:10472000184C16492046143101F016F8134904F1CB
:1047300020020020E077886C10600832086D10605D
:10474000C86C111F08600020AC6170BD0A4A0121CD
:1047500001E0401E91630028FBD17047642148436B
:10476000F4E743685B6B184743689B6C1847416FDD
:10477000491C416701F012B800A00002200D7241EF
:1047800020337241E4327241002010B500F0F3F999
:10479000284CE069222818D006DC012818D02028EF
:1047A0000FD0212806D109E0232839D043283DD055
:1047B000492838D040F20010E06110BDFEF70FFF2D
:1047C000FAE76069FEF728FFF6E701F08BF8F3E7F8
:1047D000194800780D2813D0122815D01E2817D09C
:1047E000202815D0222813D0242811D01F2813D018
:1047F000212811D023280FD01048FEF7C9FFDBE78E
:104800000E48FFF75CFDD7E70C48FFF7A9FBD3E79D
:104810000A48FFF74BF9CFE70848FFF78AF8CBE7DC
:1048200001F00AFCC8E7FFF76AFFC5E7FEF79BFE49
:10483000C2E700002033724170EF7041E0B1724175
:1048400000207047002802D04FF6FF71C1817047E9
:10485000002805D0D0F894000949884201D10120F0
:10486000704700207047002805D0D0F8980005490F
:10487000884201D1012070470020704702487047EC
:104880000929437174539461C800002B3D4951F8C4
:104890002000D0F8840110F0010000D00120394937
:1048A000C0B2091F48707047002070473548001F8C
:1048B00000787047334A0121121F1170111D51F801
:1048C0002000D0F8401141F00101C0F840117047BC
:1048D0002C4A0021121F1170111D51F82000D0F830
:1048E000401121F00101C0F8401170472DE9F0415D
:1048F000044625480221234F4FF000460171042150
:10490000017404EB440100EB8105287902281BD1D6
:10491000002000F03DF8012000F03AF8022000F0FD
:1049200037F8012000F036F8012000F053F801209C
:1049300000F040F8012000F04DF857F82400C0F8CE
:104940008461012000F025F82879042814D157F853
:104950002400C0F884610B2000F01BF8FF232046E0
:1049600033211A46FEF7E3F92046BDE8F041FF2364
:10497000E9223021FEF7DBB9BDE8F08170477047CE
:10498000082070474CEF704144337241012070475A
:104990007047704701280BD0022808D115480168DC
:1049A00041F080010160016841F001010160704740
:1049B0001148F8E701280BD0022808D10D480168FA
:1049C00021F080010160016821F001010160704760
:1049D0000948F8E770B50024054640F2E83603E0E0
:1049E000304601F09FFB641CAC42F9D370BD01F06E
:1049F00099BB0000400250121029900008F0D8B96D
:104A00000B4611461A4608F07CBA70B504460D46AE
:104A1000204608F058EC06462946204608F058EC97
:104A20000028F5D1304670BD70B50546284608F01F
:104A30004AEC441C2846214608F04AEC0028F5D1EF
:104A4000204670BD70B50546284608F03CEC441E73
:104A50002846214608F03CEC0028F5D1204670BDE0
:104A60002DE9F04107460D461646384608F02AEC77
:104A700000EA050438463443214608F02AEC0028B1
:104A8000F3D12046BDE8F0812DE9F04107460D46FF
:104A90001646384608F016ECA842044605D00146F2
:104AA000384608F016EC2046ECE73146384608F068
:104AB00010EC0028EDD13046E4E770B5002405463F
:104AC0000E46A00607D1286828B931462846FFF7C8
:104AD0009CFF002801D0641CF3E770BD70B5002472
:104AE00005460E46A00607D1286828B93146284653
:104AF000FFF78BFF002804D0641C402CF2D94FF044
:104B0000FF3070BD00210160704770B504460D464E
:104B100029462046FFF779FF0028F9D170BD002112
:104B200073E710B5FFF771FF002801D04FF0FF3099
:104B300010BD70B504460D4629462046FFF765FFB7
:104B40000028F9D170BD00215FE710B5FFF75DFFC8
:104B5000002801D04FF0FF3010BD00000020106091
:104B6000401E7047F9487047F9490968016070476D
:104B7000F74840687047F748016800290BD1F649AB
:104B800021F01F010160F54921F01F014160F14949
:104B9000F3480831086070477047002070474FF0B5
:104BA000FF3070474FF0FF3070474FF0FF307047D5
:104BB0004FF0FF3070474FF0FF333AB131B180060C
:104BC00004D52120106000200A6070471846704705
:104BD00070B50C4611461A464FF0FF35049B30F075
:104BE00001000AD0B4F5807F06D10468A40604D57C
:104BF000C46814B10069A0470025284670BD4FF075
:104C0000FF3070474FF0FF30704730F0010006D0A2
:104C100003689B0603D5C0E90312002070474FF0DC
:104C2000FF30704712B10A6000207047CB481E3831
:104C30000860F9E77047704700207047012901D1EB
:104C400007F0E8FF7047C34B1F3010B520F01F027C
:104C500018685C680244A24203D90020086007F08B
:104C6000D9FF086000201A6010BD2DE9FF4383B012
:104C70001E460023804640021D46DDE90E474FF0E8
:104C8000FF39236019D4049A01200146521C00D038
:104C90000021059A521C00D00020009541EA4000F6
:104CA000032808D169463046FFF7CDFF00B10095D3
:104CB000009804900590009B73B1DDE90401424621
:104CC000CDE900013146384600F02FF920B12060CF
:104CD000002007B0BDE8F0834846FAE7002070479F
:104CE00030F001000DD042690A6082694A60C268F2
:104CF0008A60C268CA6000689A4A10400861002051
:104D000070474FF0FF307047012806D0022804D0CA
:104D1000032802D04FF0FF3070470020704701F0A9
:104D200001BA4FF0FF3070474FF0FF3070474FF03F
:104D3000FF30704701F0F8BB01F017BD70472DE957
:104D4000F041074683488E4608300023016813600F
:104D5000D1F800C014E04C68002054F82340666885
:104D60000BE0A56855F82050BD4205D123683946AF
:104D70007046BDE8F0411847401C8642F1D85B1CE4
:104D80009C45E8D84FF0FF30BDE8F08110B5C10771
:104D900020F0010408D18068C0680068012803D1B0
:104DA00061682046C9688847616820464968BDE84F
:104DB0001040084770B503460846002614461946B9
:104DC0001660FFF7BCFF08B1674870BD2068C107D7
:104DD0000ED18168C9680968012909D100F09BF8E2
:104DE000050005D02068FFF7D1FF2846266070BD7A
:104DF000002070BDF0B58BB016461C461A46FFF772
:104E0000D9FF002510B125600BB0F0BD2068282225
:104E1000694600F085F84FF0FF3708B13846F3E7F0
:104E20000199300CB0EB114F04D02068FFF7AEFFB2
:104E30002560F3E70020E7E770B50D460A4600213C
:104E4000FFF77DFF040010D12868C1070DD18168EC
:104E5000C9680968012908D100F05DF8040004D090
:104E60002868FFF793FF00202860204670BDF8B542
:104E700000260D461660144669462846009601F045
:104E800074FB38B9009800212246C06803682846A0
:104E9000984708B13448F8BD2068C1070ED1816831
:104EA000C9680968012909D100F035F8050005D065
:104EB0002068FFF76BFF28462660F8BD0020F8BD8C
:104EC0000A4601460020D2E7F0B58BB016461C46D4
:104ED0001A46FFF7CCFF002508B1256094E720684B
:104EE0002822694600F01CF84FF0FF3708B1384619
:104EF0008AE70199300CB0EB114F04D02068FFF71E
:104F000045FF2560F3E700207EE74FF0FF30704754
:104F10004FF0FF30704720F0010041688968084772
:104F200020F0010043689B6918472DE9FF410D46B9
:104F3000164600211F460A9C0098D0B924206946D5
:104F4000FFF781FE90B1002004B01DE70D0000B016
:104F5000C8EF704158EF70417B3372419A817241C2
:104F6000E0EF7041F0FF0F000600008000984FF066
:104F7000004101600098016841F00301314321F0D4
:104F800080410160C0E90354446104498461C0E97F
:104F900001100CB1C761D7E707F03CFE0D0000B06F
:104FA0002DE9F84FDFF8E4A34FF00109F84F06466A
:104FB000DFF8E0830023391DCAF83890FA6CCDF889
:104FC00000803868724300F04EFBF34D0B2440F232
:104FD000001B28B1401DAC6128D05846BDE8F88FB1
:104FE000FA6C0023CDF80080391D38687243521CDA
:104FF00000F039FB0028EDD1FA6C0023CDF80080D9
:10500000391D38687243921C00F02DFB0028E1D155
:10501000FA6C0023CDF80080391D38687243D21C29
:1050200000F021FB0028D5D1CAF838900020D5E740
:105030002DE9F047DFF854830127D74E04460225B7
:10504000894640F2001AC8F83870006830B9D34871
:105050002146FFF7F1FE60B9206850B14268494629
:10506000926A904728B92068221D002100F097FA23
:1050700018B15046B561BDE8F08704F58051C8F815
:1050800038700020C4F88400C1F8AC02236DC4F865
:105090008C3081F8100142F2FC516067C4F8800046
:1050A000E06760506068032816D1082542F2F0508E
:1050B00042F2F45142F2F852B3F5006F2044214419
:1050C000224404D90560062008600A2003E0042376
:1050D000036005200D6010600020CCE770B5AB4D7B
:1050E0000124AB48AEA1AC63FFF7A2FF20B1AA49EF
:1050F00002208861C00170BDA548AB49AC63C06E99
:105100000860411C01D0FFF74BFF0020AC6370BD6D
:10511000F8B59E4D01249E48A1A1AC63FFF788FF1E
:105120009D4E270210B10220B06113E09849002380
:105130009D4AAC63C86E1060CA6C424395480090AB
:10514000921C01C900F08FFA30B1401D4FF00B01E5
:10515000B1610BD03846F8BD8E4900204FF6FF777D
:10516000CE6801E0401CAC63B042FBD30020F8BD28
:105170002DE9F843854F0126854889A1BE63FFF7D5
:1051800057FF854C350210B10220A06118E0BE63C4
:10519000B9467F4FB0468448FB6E0360581C10D060
:1051A000FA6C391D7B4800905A4338680023521C22
:1051B00000F059FA38B1401D4FF00B01A1611BD02E
:1051C0002846BDE8F883734D0024EE6810E0C4EB78
:1051D000C400FA6C002305EB8000016A734800905C
:1051E0004A433868391D00F03EFA641CC9F838801B
:1051F000B442ECD3FFF78CFF0020E2E72DE9FF413A
:10520000634E0125D0E9084740F200181DE05F48D1
:105210002146654A121D8563306800F0C3F978B9EC
:105220006148406802280FD003A800942A466946C6
:10523000CDE90150306843685B6B984720B11CB1E1
:10524000404604B0BDE8F081641CBC42DFDB0020B6
:10525000F7E72DE9F041884601680546D8F80000D7
:1052600081422CD16968D8F80400814227D1A9680D
:10527000D8F80800814222D1E968D8F80C008142B0
:105280001DD100241FE0C4EBC401102205EB8106F0
:1052900008EB810706F1100007F1100107F00AED95
:1052A00068B9306A396A884209D1706A796A884275
:1052B00005D196F82B0097F82B10884201D00020DA
:1052C000C0E7641CA4B2E868A042DCD80120B9E7BA
:1052D0002DE9F041884601680546D8F80000814272
:1052E0002AD16968D8F80400814225D1A968D8F884
:1052F0000800814220D1E968D8F80C0081421BD116
:1053000000241DE0C4EBC401102205EB810608EB6C
:10531000810706F1100007F1100107F0CCEC58B935
:10532000306A396A884207D1B08CB98C884203D17F
:10533000F08CF98C884201D0002083E7641CA4B271
:10534000E868A042DED801207CE72DE9F043002484
:105350004FF0FF389DB00E468146454627466A46C7
:10536000214600F01CF960BB1198B04229D320E01F
:105370001CAA2146484600F015F910BB1C980228CB
:1053800016D06D1CB54213D1012712E000A0000217
:10539000200D7241A0817241203372415000000201
:1053A000303A414C4C00000064EF7041A0917241D2
:1053B000641C1198A04202D90FB9B542D8DBA042B3
:1053C00003D840461DB0BDE8F0832046FAE72DE93A
:1053D000F04FA1B0884600249346661E15461D96E0
:1053E000B2461E960968714A91427ED1704AD8F839
:1053F00004109142F9D1D8F808100329F5D1D8F852
:105400000C10162971D800216A4600F0C8F800284F
:10541000EBD1DDE91201119A002966D0002864D091
:10542000002A62D0B1F5007F09D0B1F5006F08D035
:10543000B1F5805F09D0B1F5005F56D107E04008B3
:1054400000E040001C90002007E08000FAE7C00068
:10545000F8E74FF0FF32401C04C5B0EB910FF8D3D2
:105460005449CBF800105449CBF804100321CBF871
:1054700008100026D8F80C10CBF80C1088E0C6EB0A
:10548000C607102208EB870505F110008146AFF230
:10549000F00107F010EC002864D00BEB87074946B9
:1054A000102207F11000209000F056F907F12807AC
:1054B00035F8260FF870A8783870E8787870287971
:1054C000A5F12605B870A7F128071C981F901AF1BE
:1054D000010007D12098102238A107F0ECEB08B9A1
:1054E0001EB9B2461D98401C00E03BE00BD120984D
:1054F000102234A107F0DEEB28B91AF101001D9645
:1055000001D086422ED1B5F82490286AB9F1000F57
:1055100028D038B3814525D895F82B1031F0FE01FD
:1055200006D000211E9195F82810032905D007E028
:105530001E99491C16D1484426E0E10700D0641C9E
:10554000411C14D1A9F57F42FF3A10D1C6EBC60128
:105550000BEB81000462501E7862D8F80C00401EEC
:10556000B0421AD040F2001021B0BDE8F08F1F9970
:1055700007F07EEE054601B1451C1F99484607F02D
:1055800078EE284401B1401C761CC7E90840044469
:10559000D8F80C00B0423FF672AF0020E4E7436851
:1055A000DB6A184743689B6C184700009A1B7DAA6A
:1055B000BC487D1FAA73EE55DBBD5EE3303A4D4912
:1055C00042494200303A53494D5F53454355524595
:1055D0000000000070B50025DDE9044639B101295D
:1055E0000DD0022907D003290BD1006D00E0C06C5B
:1055F000C4E9020505E0C06CC4E9020601E0C4E9A3
:105600000256C4E9002370BD2DE9F047614C054600
:1056100001261746DDF820909846206828B9022216
:105620004946002000F0B4FD26600021484600F005
:10563000A5FD01210446484600F0A0FD0222C9F85C
:10564000182027606760D5E901215143C4E902169B
:10565000C0F80080C0F80480EA6869685143C0E976
:105660000216BDE8F087F0B587B00F460021054669
:1056700002A81C460C9E0123CDE9000121463846B4
:10568000FFF7A8FF4448002332462146009002A8B5
:10569000FFF7BAFF404A02AB2846E1B200F074F8C7
:1056A00007B0F0BDF0B587B00F460021054602A84F
:1056B0001C460C9E0123CDE9000121463846FFF728
:1056C00089FF3548002332462146009002A8FFF7A3
:1056D0009BFF314A02AB2846E1B200F04FF8DFE70A
:1056E000F0B587B01C460546084602A9DDE90D73F2
:1056F0000C9ECDE9001301232146FFF76BFF2648DE
:105700003B4632462146009002A8FFF77DFF224A21
:1057100002AB2846E1B200F031F8C1E7F0B587B03E
:105720001C460546084602A9DDE90D730C9ECDE92D
:10573000001301232146FFF74DFF17483B46324631
:105740002146009002A8FFF75FFF134A02AB2846EC
:10575000E1B200F019F8A3E710B50446084380074A
:1057600007D0002302E0C85CE0545B1C9342FAD3EC
:1057700002E0204607F01EEB204610BD30B444681E
:10578000E46CA44630BC604730B44468A46DA446C1
:1057900030BC60476CEF7041A0A172412DE9F0412F
:1057A000416F8CB009AA0446006800F08BFC002809
:1057B00040F2001870D127E0401C60673078122852
:1057C0001BD142F2C050005904EB800202F5155281
:1057D00004EB001000F58050116800F52E70491C94
:1057E0001160D0E900328068A2EB030202F10102ED
:1057F0000844824201D2AF614EE0616F09AA20687D
:1058000000F060FC18B147E0F84D0827F84E099801
:105810000228606FD0D0A16C8842ECD206900120A3
:1058200007900AA808900122206806A900F047FC0A
:1058300010B10920A8612FE0616F0022E06C032302
:10584000DFF8B8C3DFF8B8E34143C4E91F01E94812
:10585000E94902700A7032780A26252A1CD2DFE84C
:1058600002F03F1B1B1B3F131F3F3F3F3F3F3F3F8C
:105870003F3F3F33361B1B1B253F3F1B1B3F3F3F1B
:105880003F3F3F3F3F3F3F00DE48022200906946D6
:10589000DD48019012E0AE6140460CB0BDE8F081F9
:1058A00002226946CDE900CE204608E0D74801AB88
:1058B00000900422D6486946A3E801502046FDF72F
:1058C0009CFC0028E7D10BE003700B7005E06268D8
:1058D000032AF9D1022202700A70606DC4F88C00AC
:1058E0000020DAE72DE9F04FC04D0126C94F4A21CB
:1058F00085B04FF0240AA869BE63C0B20F2809D052
:10590000C54A12681AB11F2804D3A96153E1C5F82A
:1059100018A050E1B64C001F1B284FF01B084FF099
:105920000E0B4FF00409F0D2DFE800F0373E45617E
:105930004C535AE7F4766F680F171E0E0E0EF2F1F5
:10594000F0DF0E252830FB00DFE706226846B3A112
:10595000FFF702FF84F80090FFE007226846B1A13C
:10596000FFF7FAFE0520F7E007226846AFA1FFF730
:10597000F3FE0620F0E00622A8A101E00722ADA177
:105980006846FFF7E9FE84F80080E6E006226846F4
:10599000AAA1FFF7E1FE1C20DEE007226846A9A1CC
:1059A000FFF7DAFE0720D7E009226846A7A1FFF734
:1059B000D3FE0820D0E007226846A7A1FFF7CCFE5F
:1059C0000920C9E007226846A5A1FFF7C5FE0A2005
:1059D000C2E00B226846A4A1FFF7BEFE0C20BBE08C
:1059E0000B226846A0A1FFF7B7FE0D20B4E0072206
:1059F0006846A0A1FFF7B0FE0B20ADE00622684686
:105A000086A1FFF7A9FE1220A6E00B22684696A108
:105A1000FFF7A2FE11209FE06869296A022804911D
:105A200072D90498072295A107F0FCF800284FF0DE
:105A3000060239D0049891A107F0F4F800283AD072
:105A4000049910226846FFF787FE049809228DA169
:105A500007F0E8F8002838D004980D228CA107F050
:105A6000E1F880B3049807227BA107F0DBF858B374
:105A700004980B228AA107F0D5F868B304980B228A
:105A80008AA107F0CFF848B30498072274A107F061
:105A9000C9F828B304980A2287A107F0C3F808B30D
:105AA00084F800B0BE6358E05CA16846FFF754FE7E
:105AB00084F80080F6E70622684658A1FFF74CFEFE
:105AC00084F80090EEE702E004E01E200BE084F88A
:105AD00000A0E7E71F2006E0232004E0202002E0EA
:105AE000212000E022202070DCE70A22684675A110
:105AF000FFF732FE84F800B02FE00722684674A159
:105B0000FFF72AFE0F2027E055E00AE01EE016E02E
:105B10000EE0FFE7072268466FA1FFF71DFE102089
:105B20001AE0072268466EA1FFF716FE1D2013E05B
:105B3000092268466CA1FFF70FFE16200CE009222F
:105B400068466CA1FFF708FE172005E008226846AA
:105B50006BA1FFF701FE182020706B486946FFF724
:105B600067FA08B1282025E0BE632078001F2128AD
:105B700021D2DFE800F02525252525251111111159
:105B80001625251111202020111111202025252551
:105B900016161616161616005B48FDF782FC50B94D
:105BA0000EE05948006EC0F30740FF2801D00028DE
:105BB000F2D04020A86140F2001005B0BDE8F08F9F
:105BC0000020BE63F9E738B1012805D007492A2033
:105BD000886140F2001070474C48002101600121AB
:105BE0004160022181600020704700002033724133
:105BF00070EF704128EF704129EF7041FD1CBA6CC5
:105C0000E9CBD268DF23C16FC7EFFD601E2DCB7DCE
:105C1000FADCE37900A0000234EF7041303A414CE5
:105C20004C000000303A4653424C0000303A4F538B
:105C3000424C0000303A53424C320000303A52504D
:105C40004D000000303A414D53530000303A41506E
:105C50005053424C00000000303A41505053000075
:105C6000303A454653320000303A454653324150AF
:105C700050530000303A464F54410000303A5342EE
:105C80004C310000303A53595354454D0000000048
:105C9000303A5245434F5645525946530000000092
:105CA000303A5245434F564552590000303A555309
:105CB0004552444154410000303A5A5445444154FD
:105CC00041000000303A514453505F51350000000C
:105CD000303A445350310000303A445350320000BF
:105CE000303A445350330000303A4F53424C5F42F5
:105CF00000000000303A414D53535F420000000065
:105D0000303A4453505F4200E0B17241E0D77241F3
:105D1000EE48406870472DE9FF5FED4C0746FF20D5
:105D20004FF00008039002AA3946206800F0CAF933
:105D3000002878D10298022875D0E66C211DDFF882
:105D400098A3206DDFF88C937E43CDF80090C500BA
:105D50009AF8003032462068FFF785FC002879D198
:105D60004846DE4A0168914274D1DD4A4168914259
:105D700070D1806804286DD1A9B242460D464846CC
:105D8000FAF7C6FAD7494FF0010B0190761CA046EE
:105D90003246C1F838B0211DCDF800909AF8003095
:105DA0002068FFF760FCF0BB4846CF4A016891428B
:105DB00050D1CE4A416891424CD18068032849D1E4
:105DC000019A29464846FAF7A3FA5C46DFF814B36D
:105DD000019008F10401CBF83840D8F84C20CDF8F8
:105DE00000909AF800307A43D8F80000921CFFF730
:105DF0003AFCC0B94846BE4902688A422AD1BD4A27
:105E00004168914226D18068032823D1019A29460E
:105E10004846FAF77DFACBF838408246D8F8502049
:105E20005F46454600E015E003994846FEF7E8FD69
:105E30004946B148B21C01C1B048A1E81104B049BB
:105E4000BC63CDF8009028680B78291DFFF72AFC69
:105E5000002801D040F2001004B0BDE8F09F2DE909
:105E6000F04FAA4885B0A74FDFF89C92994C006884
:105E7000401C5CD1964DFF2120462A6DFEF7C0FDE7
:105E800096484FF0010ADFF8888201A92060524647
:105E9000934860600420C4E9020AD8F80000CDE904
:105EA000010A04A80390286800F009F9994D08B187
:105EB000092038E086499648DFF844B2CE6C006885
:105EC00000949BF80030464301C93246FFF7EAFBD5
:105ED0000A2408B1AC6127E0D0465046DFF804A29E
:105EE000761C3246CAF838000097794F9BF800308C
:105EF000391D3868FFF7D6FB0028EBD1CAF8388087
:105F0000721CCDF80090391D9BF800303868FFF7FF
:105F1000C9FB0028DED17E48CAF838800068FFF748
:105F2000FAFE20B13720A86140F2001045E60020BB
:105F300043E62DE9F0416B4D0124AC63FDF713FB03
:105F4000744E2702B84201D109200EE05F48AC63CD
:105F500081685F480068FFF7F8F96D490860401CE8
:105F600002D00020AC6399E42220B061384695E469
:105F70002DE9F34F674C81B0644D40F2001BA069DE
:105F8000012832D0524E2868DFF84C91311DDFF8DD
:105F90004481F26CCDF8008099F8003042433068BB
:105FA000521CFFF760FB0B2708B1A76142E049498B
:105FB0000298FFF74EF9F26C82462868311DCDF841
:105FC000008099F8003042433068921CFFF74BFB89
:105FD0000028EAD13F490198FFF77AF928B1BAF1D0
:105FE000000F02D00020BDE8FE8F0126A6610298B6
:105FF000FDF7BBFA411C1DD0DFF8E880B71EDFF8C3
:1060000010A170B1FDF779FA58454FF0090905D094
:10601000C8F838600298FFF7F1F820B1C4F818907A
:1060200008E0C8F83860CAF800702F60FFF781FFF9
:106030000028D8D05846D6E72DE9F041294D012453
:1060400035482702AC63D0F8AC12B1B1A0F580524C
:10605000A0F57763126D511AFF2208E0D0F8AC6208
:10606000F254D0F8AC62761CC0F8AC62491E00292C
:10607000F4D12A48FDF7DEF8E0B9AC63284C20786B
:10608000252817D2DFE800F0161616161818181370
:106090001813181818181813131818161616181895
:1060A0001816161818131818181818181800FCF7CE
:1060B0009BFF08B1384656E70020207053E743683D
:1060C0005B6B184743689B6C18470000E0D7724130
:1060D000200D7241E0A1724129EF7041AC9F56FE44
:1060E0007A127FCD00A00002AA73EE55DBBD5EE3FD
:1060F0009A1B7DAABC487D1FA1BE419DEAD2DEF15C
:1061000028EF704120ED714120FD71413CEF70415D
:1061100038EF704120337241E0C17241E0B1724109
:1061200070EF704102490968484307F001B9000067
:1061300004F0704130B5F34C85B0A06800281BD145
:106140000025039503A928460295FEF7F3FD0022DA
:106150006B46EDA103A8FEF7EFFD029808B1406879
:1061600020600022EBA16B4603A80295FEF7E4FD38
:10617000029860600120A06005B030BD30B1826936
:106180008A4203D900EB01101C3070470020704791
:1061900070B50B004FF0000120F001004FF0FF340C
:1061A0000ED06AB1002505261E6058B1DB4E01688D
:1061B000314046685E608669DE604069186104E0CF
:1061C000204670BD5C60DC601C6141F00500186019
:1061D00011015868C3E9055220F003002246C3E9C3
:1061E000010303F11C0006F08CFE002070BD30B5E9
:1061F000039C80B185698D420DD9C5686D1C0AD09C
:1062000000EB011105691544CD612031C0681044CF
:1062100019C1002030BD4FF0FF3030BD30B40C4606
:1062200011461A46BE4B984215D0002813D04B1C7D
:1062300011D03CB1BA4B103B98420CD1022030BC7B
:10624000FEF762BDC80602D18818C00601D003203F
:10625000F5E70120F3E730BC70472DE9FF4F884692
:10626000DFF8A0B20024154601F11C004FF0FF3CFE
:10627000D8F818E083B00BF10C0BA14626468246F5
:1062800021462BE003685A1C26D082681644B2428D
:1062900049D81CF1010207D1D8F810208C46521CB5
:1062A00001D1C8F810305C46B4B1964B02685B6807
:1062B000B3F1005F0CD99A4FDBF80C30BB4207D02A
:1062C000D30600D0002483681344DB0600D00024EA
:1062D00012EA090F00D00024491C103072468E4586
:1062E000D0D806B324B300202946FFF751FFD8F8D1
:1062F00004006860D8F810002168401A61680844FA
:10630000E860D8F810002861E06828604FF00009C4
:10631000686805F11C060699574620F00100CA4638
:106320000843686056E06FF0010007B0BDE8F08FE9
:1063300003984FF0000730F0010105D0C968B14261
:1063400010D2FEF72AFC039703A8CDE900073346D5
:106350004FF0FF36734831463246FEF786FC08B1EF
:106360003046E2E7D8F8182029460398FFF710FFD7
:10637000CCE73868411C0AD074B130603868DBF86B
:106380000020DBF80410801A084470600EE0B86842
:10639000B060F868F06019E0296901EB090030602D
:1063A000E96801EB09007060B9688944BB68B360B3
:1063B000F868F060069848B96868800706D45749BD
:1063C0002868326808400699FFF728FF1037103612
:1063D0000AF1010AD8F818105145CAD80398A4E761
:1063E0002DE9F0478146884614461D46FFF7A2FE78
:1063F00019F1010027D06068414620F0010040EA11
:1064000008006060E068401C20D02C602068C0F369
:106410000F10A0F50041C43915D06068800712D470
:106420003E4F002604F11C050AE02A68501C05D0E6
:1064300020684146AB683840FFF7F0FE761C103507
:10644000A069B042F1D84846BDE8F0872A680B46FB
:1064500021464846FFF701FF811CF5D12C60F2E789
:106460002DE9F05F07460E464FF00008FFF762FE89
:106470004FF0FF318FB186B17068BA69B36900F02F
:1064800001099A4209D33269521C06D03A69521C5A
:1064900003D0B9F1010F03D003E00846BDE8F09F37
:1064A000786806F11C04DFF874B007F11C0500F0F1
:1064B000020A1EE0BAF1000F10D1B9F1010F1DD090
:1064C00010480068A0F50051703907D1A368226810
:1064D0003068494600EA0B00FFF7A0FE21682868F3
:1064E000814202D0A268FEF789FA1034103508F113
:1064F0000108B1694145DDD80020CFE7AB682A68C3
:106500003868E6E7E8EF7041546172676574436686
:106510006700000044616C456E760000F0FF0F00DC
:10652000400C0800400C2800F8B5002406460D4633
:10653000274668460094FEF717FB009880B1416932
:106540000CE000EBC4029269B24206D1286000EB75
:10655000C400C06968600020F8BD641CA142F0D886
:106560002F604FF0FF306F60F8BD2DE9F047BC4D54
:1065700082468846EA688AB3BAF1000F50D0AC6808
:10658000002C4DD951B3504641F2055103E001EBC7
:106590004111401C19440378002BF8D1002004233A
:1065A00007E000EB400603EBC60696598E4202D088
:1065B000401C8442F5D8844232D000EB40001021C8
:1065C00001EBC001515831B11423894603EBC000DF
:1065D0000024165822E002EBC0012CE020E05046D7
:1065E00006F04AFB074656F82400E96800EB400035
:1065F00051F8300006F040FB87420ED1504606F0BD
:106600003BFB56F824100246E86801EB410150F8C4
:106610003110504606F04EEB30B1641C4C45DEDBC9
:106620004FF0FF30BDE8F08756F82400E96800EB32
:10663000400001EBC001C8F800100020F2E77CB573
:1066400000250C46694600950195FFF78EFF18B1AD
:106650002560681E65607CBD01A8FEF785FA01987B
:10666000206000988068606000207CBD2DE9F843C0
:106670000446006804251126C0F3150012271228CD
:106680005ED006DC022820D0082828D0112804D1AA
:1066900007E014283FD0182828D04FF0FF30BDE87D
:1066A000F8830D46104600210091042201466846F9
:1066B00006F080EB0099A86829440844A06006F021
:1066C000DBFA6060102020604DE004F10800114604
:1066D000042206F070EB0220C4E9000543E012F842
:1066E000010B2660401CC4E901023CE00D46104647
:1066F0000021009104220146684606F05CEBE86840
:1067000041190098401C0844A06010F8010C401C7E
:10671000C4E9006027E00D461046002100910422E4
:106720000146684606F046EB286941190098001DAD
:106730000844A06050F8040C401CC4E9007012E04A
:106740009046FEF715FA06004FF0000000900AD0C0
:1067500004224146684606F02EEB009856F82000C9
:106760002760C4E90150002099E72DE9FF4F83B06D
:1067700080464FF0000A994657464FF0FF3BCDF850
:1067800000A0D8E900603418002E5FD0002C5DD046
:10679000002001A9FFF7C8FE00B10127214604220D
:1067A000484606F008EBD9F80000241DB0F1FF2F91
:1067B00005D0810D0AD0800D0090002213E07FBB30
:1067C000D8F800000127F1694418E7E7207804228F
:1067D0008DF8000060788DF80100A0788DF8020037
:1067E000E0788DF803000025DDE9041300981444D7
:1067F0003AB151B172683044104406F0B2EB18B1AE
:1068000003E011B9984200D1012555B1012DC5D140
:10681000224631464846FFF729FF07B0BDE8F08F12
:1068200014E0D9F80000C0F31500122810D006DCDF
:1068300002280DD008280DD0112804D108E0142812
:1068400006D0182804D05846401CA7D15846E4E783
:10685000241D03E02078801CC0B204445046F3E7B6
:10686000ECD77241806800F05AB9F8B500250F46A0
:106870007C20164669460095FEF7E5F9040024D110
:1068800000987C220021FEF7BBF849493846009A5F
:1068900000F0FDF8040018D100984649C0E9051041
:1068A000454940F8101FFFF7DDFF4149009A0839BC
:1068B00002F110003060086810B90A6005E008466F
:1068C000816F0029FBD1826795672046F8BD70B5BE
:1068D0000446806800F031F9354A0546A068083A58
:1068E000116851B1884203D1886F106005E01146EC
:1068F0008A6F8242FBD1906F886715B9A068FEF756
:106900009BF9284670BD10B504468068C168486888
:106910001031FEF70FFAA068BDE8104000F044B94E
:10692000806800F073B9806800F085B9806800F075
:1069300084B9806800F088B9806800F077B94FF0BA
:10694000FF307047806800F084B9806800F086B935
:10695000806800F088B9806800F08AB9806800F02B
:106960008CB9806800F08EB9806800F090B98068BA
:1069700000F092B9806800F094B9806800F096B990
:10698000806800F09BB9806800F09DB9806800F0D5
:10699000A2B9806800F0A7B9806800F0A9B9806842
:1069A00000F0ABB9806800F0B0B9806800F0B5B90C
:1069B00020F0704104E670411FDA1FDA30B401693B
:1069C000002913D101220C46C0E9042100F118036B
:1069D00004E0C26802FB0132491C546082688A42AA
:1069E000F7D80168002901D030BC084730BC704797
:1069F0002DE9F74F0024D1F808800D46A346A146A3
:106A00000846FFF7DBFF05F1180A19E0E96801FB0A
:106A100004A6F06A90B1009806F02EF90746F06AD5
:106A200006F02AF987420AD1009806F025F9F16AA2
:106A30000246009806F03EE9C8B100E0A046641C9A
:106A4000A868A042E2D840450DD0EA680023294654
:106A500002FB08A04246814600F094F800994FF0EE
:106A6000010BC9F82C100298C06820B108E0A86892
:106A7000B1468046E7E702985A46494600F089F851
:106A80000020B9F1000F00D1401EBDE8FE8F2DE9B6
:106A9000F0470025814692460E462C464FF00208EC
:106AA0000846FFF78BFFB36806F11807581E0FE082
:106AB000F16801FB00714968494503D14FF00008B6
:106AC000054607E011B94FF001080546401E641C59
:106AD000A342EDD8B8F1000F06D0B8F1010F05D0F0
:106AE0004FF0FF30BDE8F087002208E0F0684B4629
:106AF0002A46314600FB057000F044F80122F06898
:106B000000FB0571504600F044F80020EAE70168F8
:106B1000491C0160C0684169491C41617047C168F6
:106B20000A68521C0A60C168C9684A69521C4A61F5
:106B30000168491C01600846704770B50446C0688A
:106B40002168C06831B141694FF00005491E4161BB
:106B500002D007E0002070BD016919B105614168EC
:106B600001B18847E0680168491E016004D1E0680E
:106B70004560C5608560C5622068401E2060EAD11E
:106B8000E56070BD10B50024C0E90221C0E90043F2
:106B900010BDC268002A02D102604260C160704725
:106BA00000207047002070472DE9F041C7684FF082
:106BB000FF36804635461020344607F1180207F1AB
:106BC0004001FEF72FF868B97868A0F100705038DE
:106BD00002D0EF2806D101E0062000E0072000F0F7
:106BE000A1F80446601C0CD0206828B909E0404692
:106BF0008847050008D0241D14B121680029F6D16A
:106C000015B13046BDE8F0810020FBE770B5C468DF
:106C10004FF0FF35D4F8C0108968884720B9206C40
:106C2000FDF7BBFF002800D0284670BDC368D3F82D
:106C3000C0301B68184700207047C168D1F8C010E9
:106C400049680847002070474FF4803048600020B2
:106C50007047C268D2F8C020D2681047C368D3F822
:106C6000C0301B691847C168D1F8C010496908478E
:106C7000C368D3F8C0309B691847C268D2F8C020F7
:106C8000D2691047C168D1F8C010096A0847C168C5
:106C9000D1F8C010496A0847C368D3F8C0309B6A6E
:106CA0001847C368D3F8C030DB6A184730B4C468EB
:106CB000D4F8C040246BA44630BC6047C368D3F806
:106CC000C0305B6B184730B4C468D4F8C040A46BC4
:106CD000A44630BC604730B4C468D4F8C040E46B0C
:106CE000A44630BC6047C368D3F8C0301B6C18475B
:106CF000C368D3F8C0305B6C184730B4C468D4F8AC
:106D0000C040A46CA44630BC604730B4C468D4F81A
:106D1000C040E46CA44630BC6047C268D2F8C020D2
:106D2000126D104706281BD006DC05280CD2DFE8C0
:106D300000F00E0E10131E00072813D00B280DD0E4
:106D40000E2804D0162810D04FF0FF3070470020D6
:106D5000704741F28000704701207047042070475F
:106D60000548704704480830704740207047024883
:106D7000001F704770470000ECF1704170B50025AE
:106D8000FF4C6E1E206818B1FDF707FF00B13546B5
:106D9000A06918B1FDF701FF00B13546F8490020A0
:106DA000A061103920604860284670BD2DE9FC5F65
:106DB000F34E824600258B46103E7068012802D1B2
:106DC000FFF7DCFF0546EE4C00F0F4FB30684FF4B3
:106DD0000017B046012800D1EA4F6DB94FF0000905
:106DE0004FF0FF365346314632463846CDE900492A
:106DF000FDF73BFF28B13546FFF7C0FF2846BDE849
:106E0000FC9F2068211DFDF76BFF60680A22FF21AF
:106E1000FDF7F6FD04F118015B46CDE90019314696
:106E200032463846FDF721FF0028E4D1A06904F17D
:106E30001C01FDF755FF201D0121C8F8041007C8EB
:106E400000F0BFFB1C3407CC00F0BBFBD6E770B5ED
:106E50000546CB4800241E4610380068012802D0A1
:106E60001160204670BD134628680A463146FFF778
:106E7000B7FA2860401CF4D1C41FF2E770B5D0E91E
:106E80001763056C00249B1BAB40A51F012A0DD086
:106E9000994208D28E189E4205D8806A431E0B4044
:106EA0009918814200D92C46204670BD9942FAD2E9
:106EB000FAE710B500242146FFF760F9204610BD1F
:106EC00000207047002070476FF0010070476FF09E
:106ED000010070476FF0010070476FF001007047CC
:106EE0006FF00100704770B50446406F00254068A0
:106EF00060B1E068006CFDF79DFE606F4168204660
:106F000088470546E068006CFDF795FE9E48856061
:106F1000284670BD70B50446406F002570B180688A
:106F200060B1E068006CFDF785FE606F8168204607
:106F300088470546E068006CFDF77DFE90481038F4
:106F40000168012902D1406C00B180478E488560FC
:106F5000284670BD70B50446C0680E46006CFDF74B
:106F600069FEE0683146D0F8C4006067204601F051
:106F70007DF9050005D1606F3146C2682046904713
:106F80000546E068006CFDF756FE7F4885602846A0
:106F900070BD2DE9F0410546006800260C461746F5
:106FA00018B144B1012C55D0761E77490020886075
:106FB0003046BDE8F081E86814462022416C04F1B7
:106FC000100000F02AFBE868806C2060E868C06C64
:106FD0006060E868006DA060E868C06EE063E86823
:106FE000406DE060E868006E2063E868406E6063B2
:106FF000E868806EA063A86C2064686A6064A86A10
:10700000A064E86AE064286B2065E86B6065E86D61
:10701000A065A86DE065E868D0F880002066E868A3
:10702000D0F884006066E86C58B1606C4008606419
:10703000E06C4000E064206D40002065606D400021
:107040006065E868D0F8CC00E066E868D0F8C80071
:10705000A066AAE7686F00690028A6D0E868006CFF
:10706000FDF7E8FD686F3A462146036928469847D0
:107070000646E868006CFDF7DEFD96E72DE9F0476F
:107080000546C0680027884691460C461646006CA7
:10709000FDF7D0FD0CE0D4E900010844D5E9172143
:1070A000401E891A884202D36FF005070BE00C34AA
:1070B000761EF0D23FB9686F836923B14A464146D4
:1070C00028469847074630488760E868006CFDF717
:1070D000B2FD3846BDE8F08730B5C0680B09090736
:1070E0000325C90E006F8D4050F82340AC43012AA0
:1070F00040F8234007D0022A05D0042A02D12C43AD
:1071000040F8234030BD8A401443F9E72DE9F041AF
:107110000446C06800250E461746006CFDF78AFD40
:10712000D4E91710401AB04201D8AD1F0EE0606FCD
:10713000836A5BB13A46314620469847050005D13F
:10714000E06D002281192046FFF7C6FF0E488560DA
:10715000E068006CFDF76FFD28462AE72DE9F04155
:107160000446C06800250F469046006CFDF762FD9E
:10717000D4E91701091AB94208D8AD1F24E000006C
:107180000CD87241400C28004CD87241616FCB6A18
:10719000D3B1C619E0683109006F50F821003107FA
:1071A000C90EC84000F0030001280BD0022809D006
:1071B000032806D0424639462046984705000BD0A2
:1071C00002E00420C8F80000EA488560E068006C2E
:1071D000FDF731FD2846ECE6D8F800203146204680
:1071E000FFF77AFFF0E72DE9F8430546C068002471
:1071F000894690461E46006CFDF71CFDD6E900123C
:107200002846FFF73BFEA71F00B13C467168404689
:10721000FFF74FFE08B13C461BE0D4B9686F006B26
:10722000B8B1286F01236A46011D00914146FFF75E
:107230000EFE04000DD10098414600F065F90400EF
:1072400007D1686F3346009A4946046B2846A04729
:107250000446C8488460E868006CFDF7ECFC2046F2
:10726000BDE8F8832DE9F8430546C0680024894647
:1072700090461E46006CFDF7DDFCA96A3269306855
:1072800001FB0201706882082846FFF7F7FDA71F7F
:1072900000B13C4671684046FFF70BFE08B13C4622
:1072A0001BE0D4B9686F806BB8B1286F01236A46C0
:1072B000011D00914146FFF7CAFD04000DD1009861
:1072C000414600F021F9040007D1686F3346009A67
:1072D0004946846B2846A0470446A6488460E8686F
:1072E000006CFDF7A8FC2046BAE72DE9F8430546F7
:1072F000C0680024894690461E46006CFDF79AFC43
:10730000D6E900122846FFF7B9FDA71F00B13C4699
:1073100071684046FFF7CDFD08B13C461CE0DCB982
:10732000686FC06BC0B1286F00236A46011D0091D1
:107330004146FFF78CFD04000ED1686F3346009A7A
:107340004946C46B2846A04700990446404600F0D1
:10735000DBF808B14FF0FF3486488460E868006CC1
:10736000FDF769FC20467BE72DE9F0410446406FBC
:107370000E46174698464FF0FF35806C78B1E068AE
:10738000006CFDF757FC606F43463A463146856C0A
:107390002046A8470546E068006CFDF74CFC2846EF
:1073A00007E66FF0010070472DE9F0470746C06817
:1073B000002590468A462E460C46006CFDF73AFCA6
:1073C0006FF0050910E0A26838462168FFF756FD06
:1073D00008B14E4613E0D4E901123846FFF74EFDDE
:1073E0000028F6D10C346D1C4545ECD33EB9786FBE
:1073F000436C23B1424651463846984706465D489D
:107400008660F868006CFDF716FC304662E62DE9F0
:10741000F0410446406F6FF001050E46174698464E
:10742000C06C78B1E068006CFDF704FC606F434607
:107430003A463146C56C2046A8470546E068006CD0
:10744000FDF7F9FB4B4885602846B2E570B5C66884
:107450006FF00104054600F01DF828B1012100205D
:1074600045A2FDF7EBFB11E0E868006CFDF7E2FBDD
:107470004D48C6F8C000284600F053FB0446E868B3
:10748000006CFDF7D8FB0CB1FFF778FC394884603D
:10749000204670BD70B500F045F8040030D1434D72
:1074A000661E6868012817D00120FFF73BFC0446E0
:1074B0000220FFF737FC01462046FFF777FC044621
:1074C0000E20FFF72FFC01284FF0000106D000200E
:1074D00000F050FF24B113E00024FBE70120F7E7A0
:1074E0000320FFF71FFC411C0CD0A8600B20FFF706
:1074F00019FC411C06D02E49E860042000F03AFF38
:10750000204670BD3446FBE70246284810B50024EB
:107510000068012804D11046FEF7A2FF00B1641EE6
:10752000204610BD70B506464FF0FF340020FFF72F
:10753000F9FB411C1BD01D4D012802D00020286002
:1075400011E00C20FFF7EEFB411C0DD0016859B192
:1075500050B1012129600168144840308847296CE6
:107560003046884700B90024286800F0F2FF204622
:1075700070BD00004CD87241466C6173683A204679
:1075800061696C656420746F20646F20696E697432
:1075900069616C697A6174696F6E20666F722070C0
:1075A000726F626521000000FCF17041FCD77241EE
:1075B0007377704170490020086070476E49086019
:1075C000704710B56C4C2368022B09D203EB4303C0
:1075D00004EB8303D960C3E901022068401C2060EA
:1075E00010BDF0B5644E00210C46356811E001EB8A
:1075F000410206EB820252F8043F5F1C08D083422E
:1076000006D857681F44874202D99268C31AD41813
:10761000491C8D42EBD82046F0BD70B50446154696
:10762000FDF7ECF90021601900F8011C70BD2DE98F
:10763000FF5F0D464FF0FF34A346DDE90E6802936D
:10764000D0E90B01009000208146019007E055F839
:1076500020305B1C02D04FF0000B05E0401CB0EB6B
:10766000910FF4D3002C7CD110680024B04202D2D8
:10767000C8F8000001E0C8F800600027D8F80060F2
:1076800000987100039105F0F4ED82461EE0039925
:10769000794321F0030000EB050E701820F0030081
:1076A0004219002008E052F820C05EF820306FEA4E
:1076B0000C0C634503D1401CB0EB960FF3D3B0EB39
:1076C000960F02D104B98946641C7F1CBA45DED8E6
:1076D0008CBB0120019000980027B100039105F0B8
:1076E000C8ED009024E00399C6F35D0C794321F0C6
:1076F000030000EB050A01EB460020F0030000EB5D
:10770000050E00200BE05AF8202042F0FF235EF81F
:10771000202002F0FF12D243934202D1401C844544
:10772000F1D8844502D104B98946641C00987F1CB5
:10773000B842D8D8B4B10198012802D00022002064
:1077400009E00122FBE700FA02F14B19029913F854
:1077500009300B54401CD8F800108142F3D8C8F807
:10776000000002E00021C8F8001004B05846BDE84F
:10777000F09FFDF7D4BA000060D8724101464FF087
:10778000FF3010B5CB68F949A1F11004DA6D6468D7
:10779000012C0FD1F6484C680460CC684460C8697D
:1077A0009060CC69DB6F2344D3604A6AFF21FDF708
:1077B00027F9002010BD0020704710B58EB0EB49AE
:1077C00002464FF0FF34002010390C900120009049
:1077D00001900CAB4869099088690A90C8696946AC
:1077E0000B90D0690DAA00F099FF0C9890B9E04B6E
:1077F0000D991868084418605A68521A0146C40660
:107800005A6002D0203121F01F01081A101A0024FA
:10781000C3E900100EB0204610BD70B50025044627
:10782000C06900F0FDFD681EE061206F20B1FDF72A
:1078300003FA054600202067284670BD7CB5044643
:10784000C06800263546426FC16DA262826FE26257
:10785000C26F2263C74AC0F8C4204E604A780978D4
:10786000E06900F048FE1620FFF75CFA0146C048C8
:107870008068026CE06900F048FEA06A012101E026
:107880004008491C21640228FAD1A06C01281ED0AE
:10789000022820D0032803D0E5630220A0641BE067
:1078A000E069032100F0C8FDE06901A900F054FE81
:1078B000019A00215068E56305E0E36B491CC56847
:1078C00010302B44E36313688B42F6D808E0E5637D
:1078D0000121E06902E0E5630221E06900F0ACFD0E
:1078E000206F80B940F6200569462846FDF7ABF9C0
:1078F00010B14FF0FF307CBD009800212A46FDF703
:107900007FF800982067E068D0F8C40060673046D0
:107910007CBD70B50026044600F0ACF9701EE06135
:10792000E0680025C06D18B1FDF786F9E068C5650F
:10793000E068006F18B1FDF77FF9E0680567E0685F
:10794000D0F8D00020B1FDF777F9E068C0F8D0504A
:10795000874CA06810B1FDF76FF9A560304670BD87
:107960006CE72DE9FF4104464FF0000C03EB830068
:107970004FF00108664602EB8005EB680093A868AB
:107980000DE093F828200F78BA4206D193F8292009
:107990004F78BA4201D100931AE0401E54330028B8
:1079A000EFD1BCF1000F13D120460A46694602F020
:1079B000F2FA50B101AA20466946019601F09FFFF4
:1079C00008B1019631E0019878B30098C0E90168E8
:1079D000009858B304220273016852025300082928
:1079E00002D0102909D021E0816B914201D10673A8
:1079F0000DE099421AD1022108E0816B914202D137
:107A000080F80C8003E0994210D103210173007BC0
:107A100003AA296951F8200002C8CDE90110E069E4
:107A200001A900F0A2FF039800B10096009804B0ED
:107A3000BDE8F0812DE9F0478CB005460720894666
:107A400000240890661EE868C76D0AA8079602F031
:107A5000BDFA0A9B002002E0022A17D0401C00EB6E
:107A6000800153F82120002AF6D130466FF0010A38
:107A70008046401C06D008AA07A904A800F0B4FC60
:107A8000089890B150460CB0BDE8F08702220492ED
:107A900000EB800203EB82025268069201220592FB
:107AA00053F821100029E0D0E0E7069840F60001E5
:107AB00028620798E86100F0FAFC2846FFF77DFE8F
:107AC00008B1344622E0B968C9F80010B8680090DF
:107AD000FFF787FD01900420029000200390694683
:107AE000079801F021FA0028EBD109A802F06EFAFC
:107AF000D9F800104346099A2846FFF732FF1C497F
:107B000000288860DDD00698286244B10798411C9F
:107B100005D000F085FC2846EE6100F0ABF8204669
:107B2000B1E72DE9F04F85B00446012111484FF02F
:107B3000000A114ACDF810A0CDE900A1E168CDF806
:107B40000CA002600D4A42600D4A82600D4AC2607C
:107B5000C1F8C400242003A9FDF775F84FF0FF36E3
:107B600090B1304605B0BDE8F08F00000CD87241EE
:107B700050F2704170F27041B77770411B787041DC
:107B80001379704161797041E1680398C8652046B6
:107B9000FFF7F4FD6FF0060B20B1E0695D4600F0E1
:107BA0003FFC61E004A92046FFF744FF08B13546D9
:107BB00051E0E06901A900F064FCE069002100F0F7
:107BC00047FC0198012803D9E069012100F040FC3D
:107BD000B44FDFF8D492386801281CD1D9F80800D6
:107BE00002AAD0E90E51CDF808A0E0698846B9682C
:107BF00000F088FD0120FFF795F8029908440290F3
:107C000005EB08014031FFF7D1F810B92046FFF726
:107C1000B5FD05001CD1D9F808102046DDE9003279
:107C200000F035F8050013D1FF682046FFF706FE87
:107C300005462046FFF7C1FD08B15D460BE03DB9A2
:107C4000072F13D0082F11D0204600F065FA054603
:107C50009648C46045B1E069411C05D000F0E0FBE6
:107C60002046E66100F006F828467BE7204600F053
:107C700050FAECE710B50446C068C06DFCF7DCFFB5
:107C8000E1680020C86588490860486010BD2DE99A
:107C9000F041884687490446854800251E461A4615
:107CA000086085484860854888608548C8604146C6
:107CB000204600F05CF86F1E50B93246414620461F
:107CC00000F0B2F820B9E169404600F007F808B1C9
:107CD0003846ADE60220A0642846A9E670B50E46F7
:107CE000816B0025044688B0304600F0E0FBE16B74
:107CF000304600F0E8FB2168304600F0F0FBE06C15
:107D0000C0F38051C0F3C0521140C0F30060014085
:107D1000304600F039FC0221304600F08DFB694608
:107D2000304600F025FC94F84C00C1061CD0C0F38E
:107D300004010798814217D9002468460CE000EB43
:107D400084029268914206D800EB84008168304634
:107D500000F0A1FB03E0641C019AA242EFD8019855
:107D6000A04201D16FF0010508B0284670BD2DE991
:107D7000F041C46800277E1E0D46E06D28B924201E
:107D800004F15C01FCF75FFFE8BB4A48C4F8C4009B
:107D900005F1140060640220A06495F84E0010F014
:107DA0000C0000D00120E06405F10C0555F80C0C26
:107DB00020654FF001006065286CC0F38051C0F36E
:107DC000C05201EA0201C0F3006001EA0001A165AE
:107DD000287F2066687F6066A87FA066686AE06684
:107DE000A96A6167E96AA167D5E90B121144E167E5
:107DF000296CC4F88010696CC4F88410216F89B9AB
:107E00000009800000E004E004F17001FCF71BFFB2
:107E100008B130460CE6E06E002100098200206FB8
:107E2000FCF7EEFD384603E670B5C4680025E26D48
:107E3000A36FD1614E6C16618E6C5661194E10366F
:107E40001662C068C06D006AC6699660C069E46F5A
:107E50002044D060D1E90D40096B60430324800ABF
:107E60004143880A0221B3F5007F11D0B3F5006FBA
:107E700007D0B3F5805F04D0B3F5005F01D0C81E12
:107E800070BDFF2801D9147000E01170517006E038
:107E9000402801D3147000E0117001205070284672
:107EA00070BD0000FCD7724150F270414CD8724155
:107EB000B777704170F270411B787041137970414F
:107EC000617970412DE9F0470127054688469146C2
:107ED0001E46FF4CC06802222146C06D006A8069C0
:107EE000FEF756F900212046FEF748F904460660E1
:107EF0003046FFF776FB60600023E868012209F056
:107F0000FF01806FC4E9020704F11000C0E90237E5
:107F1000E868846FEE483C30C0F80080C3600346D8
:107F2000C0E901242846EA4ABDE8F047FEF7D3BE7F
:107F30002DE9F84F0446C068002789463E46D4E93B
:107F400017B2D0F8D0800092D8F80CA00BE0C6EBA6
:107F5000C601102208EB810549461035284604F079
:107F6000AAEE18B1761C5645F1DB00254FF0FF3123
:107F7000C5B32869E0656869421C0BD02A691044C2
:107F80002066E268D26E904200D90F46686960624E
:107F900047B131E0E068C16E2166C06E2969401AC0
:107FA0006861F3E7697E287E40EA0120A97E40EA05
:107FB000014000F47F01A165297EFF2902D1697E7D
:107FC000FF2916D0E168896D11B1C1B203290AD029
:107FD0000021E164C0F30721012906D010F47F4F8E
:107FE00005D006E007E00121F3E7032100E00221CC
:107FF000A164A06500E00F46781C03D1C4F85CB012
:10800000009820663846BDE8F88F2DE9F84F0646FF
:10801000C068924688464FF000096A46C06D846881
:108020003046FEF73EFE00286DD1009802286AD047
:10803000F06800222346456F816F304605FB08F546
:10804000CF002946FFF73EFF00285CD1A1492068F8
:10805000884258D1A0496068884254D1A068042859
:1080600051D1B9B2D4F80C804A460F462046F8F7F1
:108070004FF96D1C81460022234629463046FFF702
:1080800021FFF0BB9549206888423CD19449606843
:10809000884238D1A068032835D14A46394620465F
:1080A000F8F736F96D1C81460022234629463046F2
:1080B000FFF708FF28BB8B492068884223D18A48F4
:1080C000616881421FD1A06803281CD14A46394605
:1080D0002046F8F71DF9691C074600222346304662
:1080E000FFF7F0FE68B98149206888420BD18049CA
:1080F0006068884207D1A068012804D1E068B842CE
:1081000000E000E001D000207DE70120CAF80080F7
:1081100079E74FF0FF3070472DE9FE4F0026044607
:10812000B04635460096374601964FF0FF3BC16892
:10813000C86D80680290D1F8D00030B9D03140F2DB
:108140000040FCF780FD00287DD14020C4E9175095
:10815000002560626A4629462046FFF756FF01283F
:1081600009D06D1C402DF5DDE168C1F8CCB0E168A7
:10817000C1F8C8B075E0402D4FF0010AA946F3DC04
:1081800009F1010507E001AA29462046FFF73DFF56
:1081900001280AD06D1C402DF5DD5AEA070007D0F2
:1081A000BAF1000F12D057B118E001272E46F4E7BC
:1081B000E168C1F8CCB0E168C1F8C8B022E0E1687C
:1081C000C1F8C890E168C1F8CCB01BE037B1E068F5
:1081D000C0F8CC60E168C1F8C8B013E0DDE9000187
:1081E000884241D007D9E2688046C2F8C890E16869
:1081F000C1F8CC6006E0E0688846C0F8C860E26874
:10820000C2F8CC90E068D0F8C8104A1C29D018F108
:10821000010229D0406F0022029B41432046491CA5
:10822000FFF750FEE8B902982C4A0168914218D134
:108230002B4A4168914214D18068032811D1E0682B
:10824000D0F8D00000E00FE0029940F20042FCF7C5
:10825000D5FB284840F278210160E168D1F8D010C0
:1082600041600020BDE8FE8F5846FBE72DE9F04154
:1082700004460F46022000250922A0641EA13846AC
:1082800004F018ED002670B1062238461DA104F056
:1082900012ED60B139462046FFF74AFE00B16D1E6F
:1082A0002846BDE8F081E0680321A16404E0114A9A
:1082B0000121E068121F1170C16E006F09098A0068
:1082C0000021FCF79DFBE665E068C06E20661DE0BE
:1082D0007CD87241AC9F56FE7A127FCDAA73EE55C0
:1082E000DBBD5EE39A1B7DAABC487D1FA1BE419DFC
:1082F000EAD2DEF160F27041303A414C4C5F4553B6
:1083000000000000303A414C4C0000006062C7E7BA
:1083100010B540EA01040346A40710D02AB90EE0C4
:1083200011F8014B521E03F8014B43EA0104A40764
:1083300005D0002AF4D102E010C9121F10C3042A8C
:10834000FAD222B910BD11F8014B03F8014B521EAD
:10835000F9D210BD10B5044604F0C0EF204610BDA0
:1083600010B500230446C9B201E0E1545B1C9342FE
:10837000FBD310BD164A10B5AFF21B03052808D277
:10838000DFE800F003080B101500124810601248D7
:10839000506010BDAFF2870001E0AFF24700C2E9C4
:1083A000000310BD086890604868D06010BD11617E
:1083B00010BD074B1B681847054B5B6818470449FD
:1083C0008A680260C96841607047014909690847C5
:1083D000C8D87241A4CD7041EDCE7041FCA10160BE
:1083E0007047704770477047F8B505460E46012044
:1083F0001060801E14460860684601F0EDFD009B89
:10840000581C0CD0C3EB0310F64900EB831033600B
:10841000224601EB800128460B6002F05AF8F8BDB5
:10842000002810B507D101F0EFFDEE48D0F8D010CC
:10843000BDE81040084710BDC0EB001202EB8012EF
:10844000E84800EB82008163012180F8C01070478A
:10845000C0EB001202EB8012E24800EB82000165E3
:10846000D0F8F420002A01D0084610477047C0EB2E
:10847000001202EB8010DB4A02EB8000006D086006
:108480007047C0EB001202EB8010D64A02EB80006E
:10849000806D08607047C0EB001202EB8012D1487B
:1084A00000EB8200C163012180F8C0107047C0EB6F
:1084B000001202EB8012CB4800EB820041640121E4
:1084C00080F8C0107047C0EB001202EB8012C54864
:1084D00000EB82008164012180F8C0107047C0EB7E
:1084E000001202EB8012BF4800EB820041630121C1
:1084F00080F8C0107047C0EB001303EB8013B9483D
:1085000000EB8300C0E91B12704710B5044601FB65
:1085100002F004F0E6FFB44AB44B04F0F5FFB44AAD
:10852000B44B04F009FF04F0AFFFC4EB041101EBFE
:108530008412AC49401C01EB820100F0FE00801E59
:10854000D1F8DC104008002902D0BDE810400847EF
:1085500010BDA94908707047C0EB001202EB8012F1
:10856000A04800EB820202F12800D2F8E820104770
:10857000C0EB001202EB80129A4800EB820202F17B
:108580002800D2F8D8201047C0EB001202EB80126E
:10859000944800EB82004165012180F8C0107047CB
:1085A000C0EB001101EB80108E4901EB8000406DA3
:1085B000704770B50D469149044616460020086084
:1085C0001146284601F025FDC4EB0410324600EBAD
:1085D0008411844800EB8100294600F12803D0F87B
:1085E000E0401846A446BDE870406047C0EB00116B
:1085F00001EB80117B4800EB810101F12800D1F8EB
:10860000E41008472DE9F0410F467B4914460978EC
:10861000012903D001201060BDE8F081C0EB0011FA
:1086200001EB80126F4901EB82057449096801B1C1
:1086300001212160C0EB001395F8C02003EB8010EE
:10864000684B03EB80062836012A05D121B9D5F8FD
:10865000D420214630469047D5F89C0040B1206890
:108660000028D9D1D5F8CC30224665493046984704
:1086700020680028D0D1634963484A6802600A68CC
:108680004260CA6982608969C1603860C4E7C0EB32
:10869000001303EB8010534B03EB8000D0F8F03055
:1086A0002830184770B50D46C0EB001101EB801261
:1086B0004C4901EB82045149096801B1012129604B
:1086C000C0EB001394F8C02003EB8010454B03EB84
:1086D00080062836012A05D121B9D4F8D4202946AC
:1086E00030469047D4F89C0000280AD0286800281B
:1086F00007D1D4F8CC302A4630464149BDE8704015
:10870000184770BDC0EB001303EB8013354800EB36
:10871000830303F12800D3F8EC30184730B4C0EBE2
:10872000001404EB80102F4C04EB8000D0F8F840CC
:10873000A44630BC6047C0EB001303EB801329480C
:1087400000EB830303F12800D3F83431184730B429
:108750002A4D00242C60C0EB001404EB8010214C47
:1087600004EB8000D0F80041A44630BC604730B430
:10877000224D00242C60C0EB001404EB8010194C37
:1087800004EB8000D0F80441A44630BC604730B40C
:108790001A4D00242C60C0EB001404EB8010114C27
:1087A00004EB8000D0F80841A44630BC604730B4E8
:1087B000124D00242C60C0EB001404EB8010094C17
:1087C00004EB8000D0F80C41A44630BC60470000A8
:1087D000464C4153482048414C2076312E302E30B3
:1087E00000000000DCD87241FCA9F1D24D62503F7C
:1087F000CDCCCCCCCCCCEC3FF0F67041F4F6704153
:1088000068F2704128DA724118DA724130B4604C73
:1088100000252560C0EB001404EB80105D4C04EBD8
:108820008000D0F8104114B1A44630BC60471560F8
:108830000320186030BC704730B4554C00252560CB
:10884000C0EB001404EB8010524C04EB8000D0F815
:10885000144114B1A44630BC604715600320186071
:10886000E8E730B44A4D00242C60C0EB001404EB60
:108870008010484C04EB8000D0F81841A44630BC6E
:10888000604730B4424D00242C60C0EB001404EB70
:108890008010404C04EB8000D0F81C41A44630BC52
:1088A000604730B43A4C00252560C0EB001404EB5F
:1088B0008010384C04EB8000D0F8204114B1A4465D
:1088C00030BC6047156003201860B3E730B4304C0B
:1088D00000252560C0EB001404EB80102D4C04EB48
:1088E0008000D0F8244114B1A44630BC6047156024
:1088F000032018609EE730B4254C00252560C0EBAE
:10890000001404EB8010234C04EB8000D0F82841C5
:1089100014B1A44630BC604715600320186089E795
:1089200030B41B4D00242C60C0EB001404EB80100D
:10893000184C04EB8000D0F82C41A44630BC6047B2
:1089400030B4134C00252560C0EB001404EB8010FC
:10895000104C04EB8000D0F8304114B1A44630BC78
:10896000604715600320186064E730B4084C0023AA
:108970002360C0EB001303EB8010064B03EB800079
:10898000D0F838310BB130BC18470320106051E7E4
:10899000F4F67041DCD8724170B50446FF480D46CC
:1089A000016841B1826C294620469047FC482968FD
:1089B000C0E9004170BD29462046FFF773FEF5E788
:1089C0002DE9F0410546F5480F461646C16C38467C
:1089D0008847040004D1324639462846FFF7ABFEEB
:1089E000EF483168C0E900512046BDE8F0812DE92B
:1089F000F04706460F4615469846089C4FF000097A
:108A0000ECB9306A002806D010680222314600F026
:108A1000DEFEC6F82090BDE8F087241A306A30B137
:108A200002223146184600F0D2FEC6F8209028688F
:108A300020302860D8F80000801EC8F800002B689D
:108A4000D868A042E9D9002CE5D0306A30B90222BA
:108A50001946304600F0BBFE012030622868BA6833
:108A6000016802FB041101602868BA68416802FBD2
:108A7000041141602868BA68816802FB14118160A2
:108A80002868C168091BC1602868FA68016902FB8F
:108A9000041101612868FA68416902FB041141610F
:108AA0002868FA68816902FB141181612868C1692C
:108AB000091BC161AFE77CB501226B46002400921F
:108AC00001AAC569C06C0028284606D0FFF79EFEA3
:108AD000B2480068012803D00AE0FFF768FEF7E714
:108AE000009840B901996A462846FFF769FF044695
:108AF000009820B11CB9082803D04FF0FF3420465D
:108B00007CBD6FF00404FAE72DE9F04F8FB04FF011
:108B1000010980460E460027CDF82890BB46C06963
:108B20000B9048690D904C6808699C492546099747
:108B30000C908868A04200D80546756004B15FB10A
:108B40000CAB31460DAACDF800B001A8FFF74FFFDE
:108B500038460FB0BDE8F08F8A46B9F1000F04D156
:108B6000D8F80C00006CFCF765F8D8F84C000AAB9C
:108B70000EAA314600280B9806D0FFF747FEDAF818
:108B80000000012803D00AE0FFF711FEF7E70A987A
:108B900038B90E990AAA0B98FFF712FF07460A98F0
:108BA00018B108281ED04FF0FF37641BC8D0002F23
:108BB000C6D1D8F80C00006CFCF73DF80CABB946F8
:108BC0000DAA314601A80095FFF711FF3068AC42AD
:108BD0002844306000D2254675600C9830610D98AD
:108BE0007061BAE76FF00407DFE77CB501226B46DE
:108BF0000024009201AAC569C06C0028284606D04E
:108C0000FFF764FE65480068012803D00AE0FFF71B
:108C100038FEF7E7009838B901996A462846FFF709
:108C2000CFFE0446009808B14FF0FF3420467CBDCB
:108C30002DE9F04F8FB04FF0010907460E464FF077
:108C40000008CDF82890C346C0690B9048690D9084
:108C50004C68086951492546CDF824800C908868F5
:108C6000A04200D80546756014B1B8F1000F09D0D4
:108C70000CAB31460DAACDF800B001A8FFF7B7FE46
:108C8000404666E78A46B9F1000F03D1F868006CE8
:108C9000FBF7D0FFF86C0AAB0EAA314600280B9800
:108CA00006D0FFF713FEDAF80000012803D00AE02F
:108CB000FFF7E7FDF7E70A9838B90E990AAA0B986B
:108CC000FFF77EFE80460A9808B14FF0FF38641B1C
:108CD000CED0B8F1000FCBD1F868006CFBF7ABFF3A
:108CE0000CAB4FF000090DAA314601A80095FFF723
:108CF0007EFE3068AC422844306000D22546756064
:108D00000C9830610D987061BDE72DE9F04F8BB084
:108D10004FF0010900258246A8464846CDF8249028
:108D2000CA68CAB1DAF81C2008924C691B4A103490
:108D30000023D1E90076D2F808B0CDE90073CB6802
:108D400002936368049323680393C968CDE905100F
:108D500016B1B8F1000F02D040460BB0FAE6B9F1F7
:108D6000000F06D1DAF80C00006CFBF763FF4FF040
:108D70000109089809AB694607AAFFF75DFD074896
:108D80000068012807D1099838B9DDE9071009AA58
:108D9000FFF716FE8046099830B103E0FCD7724118
:108DA0004CD872414FF0FF38761E07F10107D3D03F
:108DB000B8F1000FD0D1BBF1010F06D1DAF80C00E9
:108DC000006CFBF738FF4FF00009E0686D1CA8420B
:108DD00001D82034002502990097606805FB010046
:108DE0000490206805FB01000390B8E72DE9F04FDF
:108DF0008BB04FF0010900258246A8464846CDF8C1
:108E00002490CA68CAB1DAF81C2008924C69F94A61
:108E100010340023D1E90076D2F808B0CDE9007310
:108E2000CB6802936368049323680393C968CDE910
:108E3000051016B1B8F1000F01D040468DE7B9F129
:108E4000000F06D1DAF80C00006CFBF7F3FE4FF0D0
:108E50000109089809AB694607AAFFF74CFDE548E8
:108E60000068012807D1099838B9DDE9071009AA77
:108E7000FFF7A6FD8046099808B14FF0FF38761E2F
:108E800007F10107D9D0B8F1000FD6D1BBF1010F1E
:108E900006D1DAF80C00006CFBF7CDFE4FF00009AC
:108EA000E0686D1CA84201D8203400250299009783
:108EB000606805FB01000490206805FB0100039039
:108EC000BDE730B585B0012300240393C368C569AD
:108ED000DB6D5B68002BC36D1944036C00D05B1C19
:108EE0009940836A8DE80E00C06C03AB04AA694602
:108EF0000028284606D0FFF723FDBE480068012859
:108F000003D00AE0FFF70CFDF7E7039838B904999E
:108F100003AA2846FFF754FD0446039808B14FF012
:108F2000FF3405B0204630BD7CB505466B460120B8
:108F30000024009001AA2846FFF709FCAD4800680C
:108F4000012807D1009838B901996A462846FFF7E9
:108F500037FD0446009818B1022801D04FF0FF34C5
:108F600020467CBD2DE9F047012780460D469246FC
:108F70004FF0000930E02E68002429E02FB9D8F81E
:108F80000C00006CFBF756FE0127D8F84C00A8B186
:108F9000710001224046FFF794FFA96841F82400C0
:108FA000A86850F8240008B14FF0FF396868641CC5
:108FB000A0420CD9B9F1000F03D008E001223146DC
:108FC000E8E7D8F80C00006CFBF735FE0027761CAC
:108FD0006868A042D2D80C35BAF1010ACBD2484613
:108FE00019E52DE9F0470446C0680026012A3546F8
:108FF0008EB0D0F85C9004D0022A4FF0FF3A79D1BD
:1090000008E0E06C00B1490020460122FFF759FF5B
:10901000064679E0206CE26C8140002AE268D26D5D
:1090200048D0D2F804C0A26ABCF1000FA2F101023C
:1090300002EA010321EA02014CD003EB4101E36D96
:1090400021FA00F7401C3B44834011401CF801000A
:109050001844226B8046D9F81C0000210769D9F812
:109060000800FBF7CDFCE0690121FFF7E5F9D9F82D
:1090700008008146FEF7B5FA0121CDE90090206B8A
:10908000CDE9020100200490CDE906010590099187
:10909000216BCDE90A1002200C905648CDF834D04F
:1090A0005549406A884228D0226B02204946FBF786
:1090B0002BFE22E0526852B1E76D21FA00F3401C0A
:1090C0003B448340A06A401E0840105CC0E7E26D4C
:1090D000824003E003EB4102E16D81405018B8E7A4
:1090E00008E0396801EB0800089008A92046FFF75E
:1090F0007CFD08B1564607E00C3728466D1C022857
:1091000002D2B8680028ECD10EB0304683E42DE9D5
:10911000F74F8AB00B460121002708913D46C168F0
:10912000C269D1F85C80D8F81C100C690792FF2244
:109130000968D8F80860082901D04FF6FF72616805
:10914000934601D04FEA5101C06D8946012100EBE1
:10915000030A0798FFF770F90C9901200860CDF811
:109160000490A06802903046FEF73BFACDE9036018
:10917000A068DFF88090059032E0002030601E4942
:10918000D9F82400884204D0A26801203146FBF7B8
:10919000BBFDD8F81C0008AB2168426B0AFB02102B
:1091A000009009AA07986946FFF75BFBD9F8000011
:1091B000012807D1089838B9099908AA0798FFF734
:1091C000FFFB0746089808B14FF0FF3731682BEADC
:1091D0000100384303D00C980221016007E00C34F1
:1091E00028466D1C022802D2A0680028C5D10DB007
:1091F0003846AFE4FCD77241400C080070B5054614
:10920000C06C0C46164660B161002846FFF77FFF30
:1092100000280AD13168012907D10120324600EB2C
:1092200044012846BDE8704071E770BD2DE9F04764
:10923000002604460329924686B01D4688463746D6
:1092400002D0A16CE06901E0E0690121FFF7F4F8C8
:1092500000215046FCF792FF86465FEA080006D0E0
:10926000012809D0022804D0B8F1030F05D1AE6857
:1092700003E0D5E9026700E0EF68E06C0028E068F1
:10928000C06D2ED02968D0F80490A06AB9F1000F03
:10929000A0F1010001EA000221EA00013AD002EB4C
:1092A000410C216CE36D2CFA01F20CEA000C491C14
:1092B000134419F80C008B401844009001A9686809
:1092C000B8F1010FC1C1DAF81800CDE9040E28D0B9
:1092D000019869460128204628D0FFF7A9FC06B06E
:1092E0007EE6D0F804C0BCF1000F0DD02868236CD6
:1092F000E26D20FA03F15B1C1144A26A9940521EF0
:1093000010401CF800000AE0216CE06D88402968DC
:109310000844D2E7E06D02EB4101226C9040084422
:10932000CBE769462046FFF761FDD8E7FFF75DFC14
:10933000D5E72DE9F047002604460329924686B07A
:109340001D468846374602D0A16CE06901E0E0691D
:109350000121FFF771F800215046FCF70FFF864608
:109360005FEA080006D0012809D0022804D0B8F12D
:10937000030F05D1AE6803E0D5E9026700E0EF68AE
:10938000E06C0028E068C06D2DD02968D0F804900A
:10939000A06AB9F1000FA0F1010001EA000221EA80
:1093A000000139D002EB410C216CE36D2CFA01F283
:1093B0000CEA000C491C134419F80C008B401844AB
:1093C000009001A96868B8F1010FC1C1DAF818006E
:1093D000CDE9040E27D0019869460128204627D000
:1093E000FFF792FB7BE7D0F804C0BCF1000F0DD073
:1093F0002868236CE26D20FA03F15B1C1144A26A19
:109400009940521E10401CF800000AE0216CE06DEB
:10941000884029680844D3E7E06D02EB4101226CE3
:1094200090400844CCE769462046FFF76EFC56E7BB
:10943000FFF741FB53E72DE9F74F92B04FF0010AD8
:1094400004464FF000090D46CB46CDF800A051462A
:10945000C068C66DE069FEF7EFFFB6683046FEF7FC
:10946000C0F80121CDE90960206BCDE90B01002096
:109470000E900D90CDE90F010491216BCDE90510FF
:109480000220079009A80890B4E0E06C0028E0688A
:10949000C06D2AD0416800295AD0A06A2A68A0F17C
:1094A0000100E76D02EA000322EA000203EB420238
:1094B000236C22FA03F602EA00023E4403F10103A0
:1094C000885C06FA03F6064453D1A16A6868A1F1E4
:1094D000010100EA010220EA010002EB4001226CD6
:1094E000E06D00FA02F0084457E04068002819D007
:1094F0002968226CE66D21FA02F3334402F101027D
:1095000003FA02F3A26AA2F1010201EA0201415C3C
:1095100003EB01060ED1216CE06D00FA01F06968E1
:1095200008443AE0226CE16D01FA02F12A6801EB8D
:109530000206EFE76968226CE76D21FA02F3521C1C
:109540003B449340A26A521E1140405C184424E000
:10955000A26A2868A2F1010200EA020320EA0200DE
:1095600003EB4002236CE06D00FA03F002EB00060F
:10957000AAE7A06A6A68401EE76D02EA0003824318
:1095800003EB420C226C2CFA02F30CEA000C521C86
:109590001F4411F80C0097403844AF68804622E021
:1095A000BAF1000F05D1E068006CFBF743FB4FF008
:1095B000010A204603A90396761CFFF77CFA10B136
:1095C0006FF002000AE003A92046CDF80C8008F1F4
:1095D0000108FFF70AFB10B16FF0030081467F1E00
:1095E000B9F1000F12D017B1B9F1000FD8D00C3576
:1095F0000BF1010B14998B45FFF447AFA16CE069A7
:10960000FEF71AFF15B04846BDE8F08F002FEED0E8
:1096100000980128C4D1E068006CFBF70CFB4FF008
:10962000000ABDE72DE9F04F8BB088464FF00009E6
:109630000121CB46CDF80490CDF808900891C1687F
:10964000D8F80C40CD6DE9680791D8F8041009B935
:109650004FF0FF3919F101016FD0C1690091FF216D
:10966000D0F830A0A8685246FBF7CAF9009801214B
:10967000FEF7E2FE009809A9FEF76EFF5B4F02209D
:109680005B4E3A683168FBF73FFB3A6831680098F7
:10969000FEF78FFF00263DE0207838B1032805D281
:1096A000217C032902D2617C032903D34FF0FF30D0
:1096B0000BB0A9E76178012800980CD001F032F8CE
:1096C0006068E0B10622002101A8FBF799F9207A31
:1096D000012803D00EE001F004F8F1E7E168002072
:1096E00001AA04E06B781718D955090A401C2B7899
:1096F0008342F7D8616801AA009801F03AF8207C0B
:1097000002281CD0617C41F28832009801F052F8A6
:10971000761C1434D8F80800B042BDD80098FEF783
:1097200065FF009808A9FFF737F9079808990068BE
:1097300051EAC07001D04FF0FF394846B8E7A86839
:109740000390CDE905ABA968C8F8041003A90098F7
:1097500001F07FF841F28837617C00983A4601F0C9
:1097600029F80098702100F0BCFF009801213A46CA
:1097700001F020F8079A0121009801F034F8C7E7BA
:10978000F0B50446C06887B00F4615461E46C06D4A
:10979000C168039106A9C069407B00F0FFFE0698EE
:1097A00090B10168049102A9406805902046FFF736
:1097B00039FFCDE9005606983B460399826820465A
:1097C000FDF735FF07B0F0BD4FF0FF30FAE709E0D5
:1097D0000B6803604B6843608B688360CB68C36031
:1097E00010301031521EF3D27047000054F2704115
:1097F00050F27041F0B5054644F64E7048F2050C43
:109800004FF6FF7E48F2000410E015F8016B80224D
:1098100000EA04034004000C164200D063400BB180
:1098200080EA0C005208F3D100EA0E000A00A1F110
:10983000010189B2E9D1F0BD2DE9FF4F8BB0894616
:1098400000241746082526460994A246C168C06927
:10985000D1F85C8001210890FEF7EEFDD8F80800F1
:109860000390FDF7BEFE049018980197CDE9050A14
:10987000059A01200399FBF747FADFF870B24FF021
:10988000FF3A9B4FB9F1900F009409AB07AA6946C4
:10989000B8680290089806D0FEF779FFDBF8000060
:1098A000012803D00AE0FEF762FFF7E7099828B91C
:1098B000DDE9071009AAFFF783F80646AEB9099853
:1098C00098B102280FD10520B86065B1042D07D0EA
:1098D000082D02D064006D1ED4E741F20004FAE7BF
:1098E0004FF48034F7E7564605E0D8F80810189A88
:1098F0000E98FBF783F80FB03046BDE8F08F2DE9E6
:10990000F74F82B04FF0000AC2F800A00420902167
:10991000154600902022029801ABD146FFF78CFF3C
:1099200006007ED1734801998142FAD103995420EF
:10993000FBF789F90600F4D16D4940F20020FBF7EE
:1099400082F9060003986DD14FF0020B04680120E4
:10995000286040F20020664DEC21009052460298AB
:109960002B68FFF769FF060008D12F68461ED8460E
:1099700060483968814202D04FF00109A1E05C4D96
:10998000FE2138466F60FFF735FF6D6895F8FF10D0
:1099900095F8FE2042EA0121814278D10020291861
:1099A0002218401C91F82C101428117500D2F6DBF7
:1099B00004F12404002605F16000E67003F020FBAA
:1099C00095F864104843E06095F840002071FF204E
:1099D00066710126C4E90806A979A4F124044FF0B0
:1099E0000800C90700D010202060074605F150008C
:1099F000804603F005FBB0F5007F49D0297A304658
:109A0000C90603D5A979C90600D5022004F134049A
:109A1000617E60F307116176287AC0F34002207EF0
:109A200001E060E05CE062F3471020762A7AC2F33E
:109A3000000262F30301617695F8701061F304008F
:109A4000207605F15C0003F0DBFA2060404603F06D
:109A5000D7FA6060014695F85500B1F5006F95F8AA
:109A6000542042EA0020A0602148A4F1340400F10F
:109A70000C0000D02C302061082F00D00226866018
:109A800020694661287A800604D5042007E00DE0AD
:109A90000020BBE795F840002C2805D00620607315
:109AA00064202064002667E70220F8E7B9F1000F80
:109AB000A8F1010807F5807703D1B8F1000F7FF412
:109AC00057AFDA44BAF1200F03D2B9F1000F3FF4D7
:109AD00040AF701C03D103980068FBF7ADF8044851
:109AE0000068FBF7A9F805B0304606E7FCD77241DD
:109AF000C4F270414F4E46492DE9F05F0026894679
:109B0000542090463746FBF79EF8050072D198F82E
:109B1000010040F2004A40F6000BAA2863D028DC7E
:109B2000742840F2001556D012DC552848D008DCC5
:109B3000352847D036284AD0452841D046287ED1FE
:109B400043E0562841D071284BD07228F7D142E02B
:109B5000792842D006DC752834D0762837D078288A
:109B6000EDD13AE0A1283AD0A32844D0A528E6D1E7
:109B700044E0C52842D012DCBA2834D008DCAC2836
:109B800035D0B1282BD0B32835D0B52857D135E002
:109B9000BC282CD0C12822D0C32850D12BE0D528F6
:109BA0002CD006DCCA281ED0CC2820D0D32846D101
:109BB00021E0DA2817D0DC2817D0F1283FD10EE0B9
:109BC000102700E0082701261AE0102700E00827E8
:109BD0000126750214E0102700E0082701265546EB
:109BE0000EE0082701265D460AE00827012641F21B
:109BF000000505E0A9E042F2000501E044F200059D
:109C0000D9F80040082004E0221818F8001082F863
:109C10002810401EF8D20822E7A104F11400FAF738
:109C2000EDFE0020207796202064FF206064012054
:109C3000A064012E45D098F80310082000E07EE0D3
:109C4000490600D51020206094F84C0020F01F0039
:109C5000001D84F84C0098F80300C0F301000AFAD4
:109C600000F6A66398F80300B10AC0F30112402081
:109C7000904003F0FEEA6063700A98F80310C1F3A5
:109C800080018840C000E06300205E4503D0B6F547
:109C9000805F00D006206073A16B606B0E4641436D
:109CA000E808000503F0E4EA20630025C4485E45A7
:109CB0001BD194F84C20D20641D01021C0F804B03A
:109CC0001DE040F20020A06394F84C0020F01F003B
:109CD000801C84F84C00202060631020E063052085
:109CE00060732760D8E7022110E041F200018E4244
:109CF0000ED194F84C20D20621D041602021816100
:109D00000162012120612268082AECD181601CE0F7
:109D1000B6F5007F13D194F84C00C0060FD0206830
:109D2000082805D0102806D000202061451E0CE030
:109D3000A348583001E0A2482C30206105E0D9F852
:109D400000004FF0FF35FAF777FF2846BDE8F09F97
:109D50002DE9F05F00258B4654201646A846A946FB
:109D6000FAF771FF07007ED1707840F2004740F2A9
:109D7000002ABA284ED01CDCA52854D00EDCA0281E
:109D800040D006DC362835D0462837D079286BD12C
:109D90003AE0A1283CD0A328F9D141E0AA380C2808
:109DA00044D2DFE800F037433A4343432F35433D85
:109DB0004340CC2831D00EDCC32831D006DCBC288F
:109DC0002BD0C0281ED0C128E1D121E0C5282AD03F
:109DD000CA28DCD11EE0D52825D006DCD02811D039
:109DE000D12815D0D3283FD11AE0DA2812D0DC28A8
:109DF0003AD112E008204FF0010802E010204FF0A5
:109E000001088146554613E04FF001084FF008095C
:109E10003D460DE040F600050AE041F2000507E08E
:109E200042F2000504E044F2000501E0002D1BD0E1
:109E3000DBF80040042003E02218315C82F828108F
:109E4000401EF9D208225FA104F11400FAF7D6FDF2
:109E500000202077C8202064FF2060640120A064D7
:109E6000B8F1010F01E094E08DE012D0F178082004
:109E7000490600D510202060F078C0F38100E0B1E1
:109E800001281AD0022894F84C0020F01F001BD1A2
:109E900019E0C4F838A04FF0100894F84C0020F0F6
:109EA0001F00801C84F84C00C4F83C8020206063B4
:109EB00005206073C4F8009027E094F84C0020F06F
:109EC0001F00401C00E0083084F84C00F078C0F31C
:109ED00001008740A763F078B90AC0F3011240205F
:109EE0009040804603F0C4E96063780AF178C1F3DA
:109EF00081018840C000E0630120B7F5006F03D006
:109F0000B7F5805F00D006206073E801414603F09A
:109F1000B0E920630027A06B40F600022849904278
:109F200008D194F84C00C0062DD010204A600BE0F8
:109F3000022010E041F2000290420ED194F84C0051
:109F4000C00620D020204A6088610862012021617B
:109F50002268082AECD188601BE0504513D194F8A0
:109F60004C00C0060FD02068082805D0102806D065
:109F700000202061471E0CE01148583001E01048D5
:109F80002C30206105E0DBF800004FF0FF37FAF7D6
:109F900053FE3846DAE630B4137804464FF0FF300B
:109FA000982B04D0EC2B05D1204630BCA4E52046EC
:109FB00030BCCDE630BC704753414D53554E470041
:109FC00028F37041544F5348494241000149016010
:109FD00070470000B4F6704100214A1E0260454AF5
:109FE00052F821305BB1491CFAD00068401C05D101
:109FF0004048001F016841F04001016070470123A3
:10A0000042F821300160F0E7002801D139490860A9
:10A0100070472DE9F041002905463AD0A1F50577B2
:10A020006421C7EB0710800003F022E9064607EB26
:10A0300047006421C0EB471003F01AE900F50474EF
:10A0400007EB87006421400003F012E906F00301EA
:10A0500004F00302C1F10401C2F1040231442244BC
:10A06000254C00F003030E09C3F1040303442560EB
:10A070000020C4E901066E18C4E903609608666111
:10A080002A441144C4E906101421184603F0F0E8EC
:10A090002062BDE8F081184B002230B502601A69D9
:10A0A0005D695418AC4207D2DC6804EB820202609E
:10A0B00018690844186130BD0E48001F016841F05E
:10A0C0000201016030BD0C4AD2E90713994209D25E
:10A0D000936901EB810103EB81010160D069401CB0
:10A0E000D06170470348001F016841F0040101601E
:10A0F00070470000F8F6704128DA7241012809D053
:10A10000022809D003280AD04FF0FF30002900D0E0
:10A11000C0437047FF20F9E74FF6FF70F6E76FF096
:10A120007F40F3E700231360C069B0F5007F11D0D2
:10A1300040F60003984217D0B0F5805F09D101299D
:10A1400040F6E83004D040F26450484300F63850FE
:10A1500010607047012940F20050F9D0C1EB411066
:10A16000C00000F25C50F3E7012904D040F2D42093
:10A17000414301F6DC031360704700220A60026964
:10A18000002A46D0C369B3F5006F0DD0B3F5805FE8
:10A1900021D0B3F5007F3CD1012A35D0022A31D03D
:10A1A000032A36D1022030E04069082805D0022A6F
:10A1B0000FD0032A0BD0032027E0022A05D0032A60
:10A1C00001D0062021E008201FE007201DE0052027
:10A1D0001BE0042019E04069082805D0022A0FD0AE
:10A1E000032A0BD0092010E0022A05D0032A01D04F
:10A1F0000C200AE00E2008E00D2006E00B2004E011
:10A200000A2002E0012000E00020DC4A02EBC0004E
:10A210000860704701200870042248700220CA615B
:10A22000C1E901020820C8607047D44A103A516859
:10A2300021F4FC0141EA404050607047F0B5002233
:10A240000A60D0E907241119C0F88410416D21F08B
:10A250000065456540F210218166C768082F00D06F
:10A26000491040F20026B2424FF6C073016703D195
:10A2700045F48031416501E0082F04D005690421CF
:10A28000032D10D003E0016903290CD00521056DD1
:10A2900025F0F06545EAC1511025C56601650569DF
:10A2A000012D24D00EE040F203210166B44D016D72
:10A2B000294021F0F06141F4812141F40001016560
:10A2C0000A21C166416DB24221F0010141651BD0F6
:10A2D000C4F50472402303EB821211434165026905
:10A2E000032A10D121F4FC0141F4802113E0426DD6
:10A2F00021F0F06141F0407142F001129A4342F4C2
:10A300008862C0E91412F0BD026921EA0301032A40
:10A3100003D041F4C0714165F0BD41F08001FAE71E
:10A32000F0B540F214228266C168082900D05210AC
:10A330000267C46C1029C56904EB840205EB820234
:10A34000C0F88420426D42F00062426505D1836D01
:10A3500023F4F85343F460638365076906234FF6DB
:10A36000C076032F04D0022F38D0012F46D024E02E
:10A37000082901D04FF00403016D03F2FF170766AF
:10A380007F4F21F0F06101EA07014FF4802707EBCE
:10A39000432741EA070101657A4F816D01EA070110
:10A3A0004FF0007707EB034341EA030181654FF06B
:10A3B0000D0101D04FF00E01C1666FF0840148F22B
:10A3C0004053B2434C4305EB840103EB811111432D
:10A3D0004165816D21F001018165F0BD082901D041
:10A3E0004FF00403016D21F0F06141EAC3510165B2
:10A3F0004FF01301E0D04FF01401DDE7836D42F41C
:10A400008032B24343F0010342F4A8620829C0E954
:10A410001523016D21F0F06103D041F04071016519
:10A42000F0BD41F06071FAE7544A70B500250D6047
:10A43000103A0446C563056410682065506860657D
:10A440009368A365D268C4F8902040F2FF12226698
:10A45000E269520AE2641D22E265E268102A02D132
:10A4600040F0020060656069082820460DD0FFF7C3
:10A47000E5FED4E91112206D114420F0605040EA4D
:10A48000C160206584F8985070BDFFF749FFF0E780
:10A49000D0F8FC10002900D0084770470120106058
:10A4A000002915D00868072812D1496836480B687A
:10A4B00003604B6843608B688360CB68C3600B6943
:10A4C00003614B694361896981614FF0000010604D
:10A4D000704770B51546044601222A6000680228BC
:10A4E0004BD101F1280301F1CC0028490E6826F078
:10A4F0000306761C0E600E6826F00C060E602168BE
:10A500001960A16899600821D96061680024DC6342
:10A510001C641A635960194910390E681E65496830
:10A52000596540F2FF1119661D21D965911EC3E9D5
:10A530001D41DC67D102D96140F210211C67996688
:10A5400002211961402183F89820C3E9274110496D
:10A550008160AFF2C30141600E49C160AFF2E531E5
:10A56000C161AFF23F4101620B4984620161AFF208
:10A57000D301C16601F067F92C6070BD0CF7704122
:10A58000FF01F8FFFFFF00FC7000401B0000301BC4
:10A5900029A4704115A270412BA27041062805D252
:10A5A000044A00EB400002EB800000E0002008605D
:10A5B0007047000004F9704170B500250446681E1C
:10A5C00041F6D0322946C4E91D50CF48FDF7F4FECC
:10A5D000CE49CF4ECC4848603560A06E81083046E9
:10A5E000FFF759FD306818B1A26EFF21FDF7E4FEB8
:10A5F000C848007801280AD1206B012807D9D4E97E
:10A600000D01BDE870400423002201F095B970BD32
:10A61000BE495923826F5A43496851F8223043F4A6
:10A62000805341F82230816F491C416770472DE902
:10A63000F04F8A46814600245868D2E9008CD2E95E
:10A6400002129B4625460AF11003A6463DE0C3F8D8
:10A650000480D9F86860076806FB14761E600F4610
:10A6600046688E42B04400D837469F604668DE6038
:10A670001033C3F804C0D9F86860876806FB147605
:10A680001E601646C768974200D83E469E60C66860
:10A69000BCF1000FDE6001D0C668B44447681033D7
:10A6A0008F4200D9DAB1D9F86860354476468F42D6
:10A6B00000D8CE1BC76831467646974200D8D61BD5
:10A6C00032460E4305D01030641CDBF80060A64211
:10A6D000BDD86000801CCAE90250BDE8F08F0D446F
:10A6E000E4E7C0EB001202EB80108B4A10B502EBDE
:10A6F00080028648592452F8A03F40685B1C1360D2
:10A700000122634340F8232000EB830080F86111AD
:10A7100000214160C16080F85011C0F85411C0F8A8
:10A72000581110BDC0EB001202EB80107A4A30B510
:10A7300002EB8000754A50F8A03F52685B1C036032
:10A740005920434302EB8300A0F5B274256825F03D
:10A7500001052560012442F8234080F861110021A1
:10A760004160C16080F85011C0F85411C0F8581110
:10A7700030BDF0B5C0EB001404EB8010664C002334
:10A7800004EB8000614C64680AE0D0F8A0505927BF
:10A79000D65C7D4304EB85051D445B1C85F85C613C
:10A7A0008B42F2D3D0F8A0005922504304EB800032
:10A7B0004160F0BDC0EB001303EB8010564B30B589
:10A7C00003EB8000514B592550F8A04F5B686C4358
:10A7D00003EB8404C4F854110068684303EB800061
:10A7E000C0F8582130BDC0EB001303EB80104A4B7A
:10A7F00030B503EB8000454B59250224D0F8A0006A
:10A800005B68684303EB8000012380F85041C0E996
:10A810000213C0E905210021016130BDC0EB001326
:10A8200003EB80103C4B30B503EB8000374B5925D0
:10A830000124D0F8A0005B68684303EB800080F837
:10A840005041C0E902148161C1610021C0E90412D4
:10A8500030BDF8B50E46C0EB001101EB80122E4959
:10A86000592501EB8204294902234A68D4F8A01033
:10A87000694302EB8105694685F85031FDF76CFEAE
:10A88000009B04F1280032462946FFF7D0FEF8BDB0
:10A89000F8B50E46C0EB001101EB80121E49592598
:10A8A00001EB8204194901234A68D4F8A0106943D6
:10A8B00002EB8105694685F85031FDF74DFE009B9E
:10A8C00004F1280032462946FFF7B1FEF8BD70B505
:10A8D000C0EB001404EB80100F4C592604EB8000F1
:10A8E0000A4C0225D0F8A0006468704304EB800095
:10A8F000012480F85051C46040F2102482618460C9
:10A90000C261C0E9041370BD4CDA724168F2704153
:10A9100040F97041F0F67041DCD872412DE9F04108
:10A9200000240E464FF0DA5743F2B0657869306084
:10A93000000705D00120FDF748FD641CAC42F5D3AB
:10A94000AC4204D1FF48016841F008010160BDE854
:10A95000F081F8B50E4600214FF0DA540091A0B115
:10A96000F948C4F8A8000B2020600125256169463C
:10A970002846FFF7D3FF009810F4887F00D0356099
:10A98000F1484030C4F8A800F8BDEF485038E8E777
:10A9900070B501241460D0F89430DB0617D5082375
:10A9A0001360CB684968042B00D01944E74B194465
:10A9B0000B1DD1E9006535406D1C07D14569082D97
:10A9C00006D05B68DB431B041B0C12D0146070BD07
:10A9D00053F8045F6D1C00D01460C5685B68102DCF
:10A9E0006FEA030320D0DBB2002BEFD11368012BF9
:10A9F000EDD00369022BEAD144690923082C15D054
:10AA00000A3131F8025B0C882C40A4F57F45FF3DEC
:10AA100000D01360C0680828D9D18878C04310F0EE
:10AA2000FF0FD4D0136070BD9BB2DDE7C468082C63
:10AA300001D00E31E5E711F80D4FE44314F0FF0F9C
:10AA400000D01360491CDCE72DE9FF4F00271C46AE
:10AA500081B01F6090F8C01000F12805012904D1D1
:10AA6000D0F8D420194628469047286D4FF0DA5682
:10AA7000B74920F4E070084020F0605040F00060DA
:10AA80002865A96806EB01110862A968686D06EBE4
:10AA900001114862A968A86D06EB81018862002255
:10AAA0001146284600F012FFE86DC6F8AC00286E8B
:10AAB000C6F8F000C6F8E0700D2030600225DFF81F
:10AAC000848201274FF00F0A40F23F1B4FF00B0921
:10AAD000C6F814A0376101206946FFF71FFF0098F0
:10AAE00010F4887F15D000EA0B00B0F5807F05D008
:10AAF0002760D8F8001041F4805108E02068012850
:10AB000001D002202060D8F8001041F48041C8F83C
:10AB10000010C6F800906D1EDAD1316C0298006802
:10AB2000016005B0BDE8F08FF8B50E461D46002166
:10AB3000196090F8C01000F12804012904D1D0F860
:10AB4000D420194620469047206D4FF0DA578049AF
:10AB500020F4E070084020F060502065B16840EAC1
:10AB6000C1602065A16807EB01110862A168606DF2
:10AB700007EB01114862A168A06D07EB81018862B3
:10AB80002046D6E9001200F0A1FE0B2038600F200D
:10AB9000786101243C6169462046FFF7BFFE0098BA
:10ABA00010F4887F14D040F23F1108406549B0F599
:10ABB000807F04D02C60086840F4805007E028684B
:10ABC000012801D002202860086840F48040086015
:10ABD000386CF1680860F8BD2DE9F8430F461D4652
:10ABE0000021009100F12804196090F8C01001299B
:10ABF00004D1D0F8D420194620469047206D4FF05C
:10AC0000DA5620F4E07020F060502065B96840EA20
:10AC1000C1602065A16806EB01110862A168606D42
:10AC200006EB01114862A168A06D06EB8101886204
:10AC3000206EC6F8F0004748C6F8A4001C20C6F8ED
:10AC4000AC0007F10C08D7E90012204600F03EFEE8
:10AC5000342030600F2070614FF00109C6F8109069
:10AC600069464846FFF75AFE0098364F10F4887F31
:10AC700015D040F23F110840B0F5807F05D0C5F8EF
:10AC80000090386840F4805007E02868012801D01F
:10AC900002202860386840F48040386006E02B4984
:10ACA000D8F80820D8F80000FDF783FB2A4846F8BA
:10ACB000A40FE06DB0603868000701D5042028605B
:10ACC000BDE8F8832DE9FF4F87B0894605461F4848
:10ACD0004FF0000B0A9905F1280403905F46D8460F
:10ACE000C1F800B095F8C000012804D1D5F8D420EF
:10ACF00020460A999047D5F8E82006A920469047B3
:10AD0000E1694FF0FF304FF0DA5A00EB5121206D2E
:10AD100020F4E07040EA811020F060502065D4E912
:10AD20001112114440EAC1602065A2680AEB0212C8
:10AD30001062A268606D0AEB02125062A2680AEB10
:10AD400082020BE0F4F670415070FFF00001401BEE
:10AD5000FF01F8FFEC000FF000300FF0A06D9062E3
:10AD6000206ECAF8F000E069B0F5007F04D1E06D14
:10AD700020F00101CAF8AC1021693320032900D06A
:10AD800034200590D9F81400D9F80C60D9F80010D7
:10AD900002680192002200690290204600F096FDB0
:10ADA000069854F81C1F45684FF0FF3000EB5129FE
:10ADB000606F0AF1E8010860606F20F001006067D1
:10ADC000A4F11C0408604FF0DA5A0598CAF8000094
:10ADD000DAF81400FF4940F00F000860CAF81400C8
:10ADE0000120CAF8100004A9FFF798FDDAF8EC007A
:10ADF0002946C4F894002046049B6A464FF0000A96
:10AE0000CDF800A013F4887F03D1C3F3033ECE45F1
:10AE10000FD040F23F1C03EA0C03B3F5807F1AD039
:10AE2000FFF7B6FD0098082818D010B101460A981F
:10AE30000160A16E28686A6801FB1700039901444C
:10AE40000198FDF7B6FAA16EA86801FB1700216909
:10AE5000022906D00EE002200090E7E70BF1010B7B
:10AE6000E7E762695146082A03D1E268082A00D15F
:10AE70000121401A6EB1EA683146B24200D2114651
:10AE800088460399424601440298FDF792FAA6EBE0
:10AE9000080669680198B9F1010905F1100508442F
:10AEA0000190029807F10107404402908BD5E26CB3
:10AEB000C9485A4506D10A9908220A60016841F436
:10AEC000006101600068000702D50A980421016052
:10AED000E069B0F5007F02D1C048E16D01600BB0C0
:10AEE00020E62DE9F04F0026DFF8F0A28BB01E60BF
:10AEF00000F12804054690F8C0000AF1540A0F46F4
:10AF00009B46012804D1D5F8D420594620469047C5
:10AF1000D5F8E82009A920469047E1694FF0FF38AD
:10AF2000206D08EB512120F4E07040EA811020F000
:10AF300060502065D4E91112114440EAC1602065D7
:10AF40004FF0DA50216EC0F8F010A268216D00EBCE
:10AF500002121162A268616D00EB02125162A268D6
:10AF6000A16D00EB8200816236202169032900D0A7
:10AF7000392007907D6900223968204600F0A6FC40
:10AF8000D5F8009028690590F86806900998E1695D
:10AF9000456808EB51276069E846082830D0102240
:10AFA0004046FF21FDF708FADDE905124046FDF7AE
:10AFB00000FAA16E28686A6801FB160049465044F1
:10AFC000FDF7F7F9EA683AB1696801EB0A00414612
:10AFD000FDF7EFF9E968884407984FF0DA51086007
:10AFE00048697C4A40F00F00106048610120086108
:10AFF00008A9FFF793FC089810F4887F06D101E0B8
:10B000001422CDE7C0F30330B84207D00120CBF8BB
:10B0100000007148016841F40041016069687F1EC9
:10B0200005F11005894406F10106C2D56A48006899
:10B03000000702D50421CBF800104FF0DA50C021F0
:10B040004164202141614AE72DE9F84300261E6052
:10B05000884690F8C01000F128041D46012904D14B
:10B06000D0F8D420194620469047206D4FF0DA578B
:10B070005B4920F4E0700840616C20F0605040EAC9
:10B08000C1602065A16807EB01110862A168606DCD
:10B0900007EB01114862A168A06D07EB810188628E
:10B0A0002024D8F800007860BE603A2038607869C3
:10B0B000484940F00F000860786101263E6169460A
:10B0C0003046FFF72BFC009810F4887F424804D0EC
:10B0D0002E60016841F4803101600068000701D5ED
:10B0E00004202860C02078647C61E9E52DE9FE4FEA
:10B0F0004FF0000A054600F128048946CDF800A06B
:10B100009B46C3F800A0574690F8C0005646194623
:10B11000012803D1D5F8D42020469047D5F8E8205F
:10B1200002A9204690474FF0DA51206EC1F8F00096
:10B13000A06D40F00100A065206D20F4E07020F0CB
:10B1400060502065D4E911231A4440EAC2602065AA
:10B15000A26801EB02121062A268606D01EB02129C
:10B160005062A268A06D01EB82018862D9F80C00E0
:10B1700001900298D9F8088021C80CE0E96831B143
:10B180007042A96800EB401001EB001A05E0761C44
:10B19000103507F50477B042F0D8E068102800D1E8
:10B1A0007F08D9F800103A46204600F08FFB4FF098
:10B1B000DA56332030607069064940F00F000860AD
:10B1C00070610127376169463846FFF7A7FB40F2F7
:10B1D000002907E044F97041F4F67041AC00401BCF
:10B1E000FF01F8FFE069484504D1E06D20F001005F
:10B1F000C6F8AC00009810F4887F02D0CBF800703D
:10B200000AE0E8684246904200D2024622B1FF4975
:10B2100001985144FDF7CDF8E069484502D1E06D51
:10B22000C6F8AC00BDE8FE8F2DE9FC5F05460F4671
:10B2300000209B460090D5F88810A1F58073FF3B55
:10B2400006D05B4639462846FFF750FFBDE8FC9F15
:10B25000CBF8000005F1280495F8C00059460128F4
:10B2600003D1D5F8D42020469047D5F8E82001A98D
:10B27000204690474FF0DA51206EC1F8F0004FF6AB
:10B28000C072606908287DD0206D20F4F000206530
:10B29000606D40F00100904340F488606065206D6F
:10B2A000DB4A20F4E070104020F0F06040F40060D1
:10B2B0002065606D40F480306065206D20F0605046
:10B2C0002065D4E911231A4440EAC2602065A268CF
:10B2D00001EB02121062A268606D01EB0212506273
:10B2E000A268A06D01EB820290624FF0FF320198DC
:10B2F000D7E902694568E06902EB502A60690828CD
:10B30000E0687AD010287FD0AA68521CE069B0F5B6
:10B31000007F7DD03968204600F0D8FA4FF0DA512E
:10B32000342008604869BB4A40F00F001060486153
:10B330004FF00108C1F8108069464046FFF7EEFA69
:10B34000009810F4887F01D0CBF800803046E9687F
:10B35000B14200D208465FEA000804D0AB49024679
:10B360004846FDF726F8E968B6EB080689441ED082
:10B37000E069B0F5007F15D001984068A84211D16E
:10B38000A54800E025E04FF0DA51C1F8A400206D97
:10B39000A36C20F0605242EAC362A26801EB021182
:10B3A00008622065BAF1010A05F11005A6D54FF033
:10B3B000DA509A49C0F8A410E169B1F5007F7FF432
:10B3C00045AFE16DC0F8AC1000205946FFF7C1FA57
:10B3D0003CE7934BA06D184020F4F85020F001009A
:10B3E00040F4802040F00100A065606D904340F47F
:10B3F000A86053E701E007E00AE0102801D0AA683E
:10B4000084E7A868401C01E0A868801C42087DE72A
:10B41000E068396810280CD0A2F50072204600F0D0
:10B4200055FAE06D20F001017E4881607E4901609F
:10B4300074E7A2F58072F1E72DE9FC4706460D4658
:10B440000020186006F128041F4656F8D42F19462C
:10B4500020469047726901A92046904760694FF6DF
:10B46000C071082852D0206D20F4F0002065606D76
:10B4700040F00100884340F488606065206D4FF023
:10B48000DA56634920F4E07008402065A96840EA74
:10B49000412020F0F0602065606D40F480306065F0
:10B4A000206D20F060502065D4E91112114440EA6B
:10B4B000C1602065A16806EB01110862A168606D9A
:10B4C00006EB01114862A168A06D06EB810188625C
:10B4D000D4F89000C6F8E80040F20029E069D5E908
:10B4E000028A484526D1E0686A6810281FD0A2F574
:10B4F00000722968204600F0E9F9E06D20F00100B3
:10B50000C6F8AC004848C6F8A40018E0444AA06D4C
:10B510001040A065AA6840EA024020F4F85040F0CC
:10B520000100A065606D884340F4A860A5E7A2F51E
:10B530008072DEE7D5E90012204600F0C7F932201C
:10B5400030607069334940F00F0008607061012578
:10B55000356169462846FFF7E1F9009810F4887FC5
:10B5600001D03D6007E05FEA080004D027490246A9
:10B570005046FCF71EFFE06948450AD106F1A406D3
:10B58000E06DB0602548306039464FF00000FFF7AD
:10B59000E0F9BDE8FC872DE9FE4F0F460546002186
:10B5A000196000F1280490F8C0009B46012804D1DE
:10B5B000D5F8D420594620469047D5F8E82002A96E
:10B5C000204690474FF0DA51206EC1F8F0006069D4
:10B5D00008287ED0206D20F4F0002065606D40F0DA
:10B5E00001006065206D0A4A20F4E07010404FF6BB
:10B5F000C07220F0F06040F400602065606D904300
:10B6000040F480306065206D10E000000001401BB8
:10B61000FF01F8FF44F9704105E00FF000300FF032
:10B62000FFFF00FCA400401B50300FF020F06050E2
:10B630002065D4E9112389461A4440EAC260206596
:10B64000A26801EB02121062A268606D01EB0212A7
:10B650005062A268A06D01EB820188624FF0FF3159
:10B660000298D7E9026A4568E06901EB5028B0F515
:10B67000007105D0E868B04202D29B4AC9F8A02008
:10B6800060690828E0687ED010287DD0AA68521C26
:10B69000E069B0F5007F78D03968204600F016F9EF
:10B6A000E8683246B04200D202465AB14FF0FF304D
:10B6B0005146019001A8FCF77CFE8C4801A9EA687C
:10B6C000FCF777FE4FF0DA51362008604869884A67
:10B6D00000E072E040F00F00106048614FF0010997
:10B6E000C1F8109069464846FFF718F9009810F421
:10B6F000887F01D0CBF80090E069B0F5007F52D090
:10B70000E868B0424FD27C487A49016060690828F5
:10B71000E0687BD010287AD0AA68521C396820468D
:10B7200000F0D4F8E9683046B14200D208465FEA3A
:10B7300000090CD04FF0FF304A465146019001A855
:10B74000FCF737FE694801A9EA68FCF732FE4FF0C2
:10B75000DA51362008604869654A40F00F001060F1
:10B760004861012008616946FFF7D8F8009810F495
:10B77000887F02D00120CBF80000E968B6EB09060B
:10B780008A4410D002E025E02BE02EE01035B8F11D
:10B79000010F02D0E868B04202D357485749016010
:10B7A000B8F10108B2D54FF0DA555548C5F8A000F8
:10B7B000E069B0F5007F39D03CE0524AA06D1040FE
:10B7C00020F4F85020F0010040F4802040F0010007
:10B7D000A06507E7102801D0AA6859E7A868401CAF
:10B7E00001E0A868801C420852E7E0683968102828
:10B7F0000ED0A2F50072204600F068F801205946EC
:10B80000FFF7A7F83E48C9F8A00049E703E009E0C0
:10B81000A2F58072EFE7102801D0AA687EE7A86839
:10B82000401C01E0A868801C420877E700205946C8
:10B83000FFF78FF8C020686420206861F2E4704749
:10B84000002018607047AFF20701C162AFF211012A
:10B8500001632D4941632D4981632D49C1632D4900
:10B8600001642D4981642D49C1642D4901652D492B
:10B87000C1652D4901662D4901602D4941612D4960
:10B880008161002141628166416441658165416653
:10B8900070470021AFF25902C0E90B121A4A426305
:10B8A0001A4A82631A4AC2631A4A02641B4AC0E9EE
:10B8B00012120165C16501660160416181618166A5
:10B8C000416241644165816541667047806CC30097
:10B8D000C0F1040001FA03F3C0001343C1404FF06C
:10B8E000DA5043608160704760D080850001401B62
:10B8F00044F9704160D08570A000401B60D0851075
:10B9000060D08010FFFF00FC49AA704129AB704154
:10B91000D9AB7041C5AC704129B2704139B47041A6
:10B92000E3AE704197B5704149B070413BCA704178
:10B93000B9A5704111A670412DE9F8431E4D064688
:10B9400000200F46009090469946D5E9001001EB83
:10B950000014A968884212D201216846FEF79BFBB9
:10B960000098002809D0076048F0080001C400983A
:10B97000A4E841026868401C6860BDE8F8830F488D
:10B98000016841F001010160F7E7F0B50A4DD5E922
:10B990000046AF68BE4204EB061407D2E3602260A3
:10B9A000C4E901106868401C6860F0BD0348016884
:10B9B00041F001010160F0BD28DA7241F4F67041F6
:10B9C0002DE9FE4F05460E460120904600901024BA
:10B9D00001900020D5E9229A02902869032800D11D
:10B9E0000A24A6F1100702A8FEF76DFB02984FF497
:10B9F000403BC0F800B07A6802EB090141600421C5
:10BA00004FF0FF390830A0E8020603E00121684644
:10BA1000FEF741FB0098C006F8D1032101A8FEF70C
:10BA20003AFBF8683168884201D1F1680844F84966
:10BA30000978002908EB000118D00098102223464D
:10BA4000FFF7A3FF0020029002A8FEF73CFB02983C
:10BA5000C0F800B0009941602969032900D0A41EF4
:10BA6000C0E90249C0F81090BDE8FE8F0098224658
:10BA7000FCF79FFCE6E72DE9F8430027814601200B
:10BA800088460097164617603D46CC6826E0216838
:10BA9000CB031DD589031BD461680B68E16819408D
:10BAA0002369994214D0C80502D5022030601CE0F9
:10BAB000511B6A4604F1140001F04BF80099082963
:10BAC00002D0012902D003E07F1C01E00121316096
:10BAD000054400EB800004EB80040120D8F8082026
:10BAE000AA4202D931680129D1D1D9F84C00C949FB
:10BAF000B84202D1082030600AE03068082807D038
:10BB0000022809D001280BD1086840F4007006E033
:10BB1000086840F4006002E0086840F48040086073
:10BB2000BDE8F8832DE9F0470024064605290D46B7
:10BB3000904627460ED9B748016841F480610160FC
:10BB4000BDE8F08718F80400E10088400743641C52
:10BB5000042C01D2AC42F5D301212846FEF7CEFADF
:10BB6000F16B4FF0DA5ADFF8A89201403943F163E4
:10BB700099F8000050B1042300220AF10400FFF7F5
:10BB8000DBFE0027042D38460AD80FE0CAF804105F
:10BB9000F7E718F80400E100203988400743641CE7
:10BBA000AC42F6D30121281FFEF7A8FA316C014000
:10BBB0003943316499F8000058B1974804230022B2
:10BBC000FFF7BAFE306D20F0605040EAC560306586
:10BBD000B6E7CAF80810F5E72DE9FC478C4E044695
:10BBE000DFF8348200204FF0DA57914608F10C0854
:10BBF0001D463178012902D00024009037E0012150
:10BC0000CDE9001003E001216846FEF744FA0098F0
:10BC1000C006F8D13078B8B1804A04230098414674
:10BC2000FFF7B3FE01A8FEF74EFA01984FF48031FA
:10BC30000160009941600421C0E90219202141EA14
:10BC400004310161BDE8FC87786900990860E9E783
:10BC50003078B0B10423414600226846FFF795FED4
:10BC60000098000705D00120FCF7AFFB641CAC4234
:10BC7000EED3AC42E6D16748016841F008010160AB
:10BC8000E0E778690090ECE72DE9F04F87B04FF0DE
:10BC90000008614F04469B464546CDF80080F837C2
:10BCA000CDF81080CDF81480C3F8008049B191F828
:10BCB000500102280AD0EAB192F8500102280FD0B0
:10BCC00012E00120186007B0BDE8F08FD1F80880BD
:10BCD00001F11005D1F854010090D1F8580108E0A5
:10BCE000D2F8088002F11005D2F854010090D2F881
:10BCF0005801049091F861112AB192F8610141EA6A
:10BD00000021E06D02E0E06D20F00100404EB1F551
:10BD1000405F02904FF0DA5A0AD04148327841EA47
:10BD200000015AB13C48042300229C30FFF704FE76
:10BD30005FEA0801A8F1010004D102E0CAF8A410EA
:10BD4000F6E7084640F2102101F066E90190206D07
:10BD5000019920F4E07040EA8111216560690828AA
:10BD6000606D20F0006001D140F0006060652269E4
:10BD70003320032A00D0342003903078A268B8B171
:10BD800025480423183000EB02100022FFF7D4FDF1
:10BD90003078A268616D78B11F4804231C3000EB35
:10BDA00002100022FFF7C8FD6069082808D013E0E0
:10BDB0000AEB02100162EBE70AEB02104162F3E7C3
:10BDC0003078A268A16D68B313480423203000EBDB
:10BDD00082000022FFF7B0FD3078B146216E30B30B
:10BDE0000D4804230022E830FFF7A6FD99F8000073
:10BDF000F8B10948042302990022A430FFF79CFD02
:10BE00004646B6F5047F6ADA2069012815D066E057
:10BE1000F0F67041F4F670410800401B120001007A
:10BE200000000FF0FFE70AEB82008162D4E7CAF856
:10BE3000F0100298CAF8AC00E2E7FF4926F00106CC
:10BE4000206DB61C084040EA462020F0F0602065D6
:10BE50006169082925D020F4F000206599F80000D8
:10BE6000A268216D30B3F548042300EB02100022D4
:10BE7000FFF762FD606D40F480314FF6C070814382
:10BE8000616599F80000A268C0B1EC480423001D68
:10BE900000EB02100022FFF74FFD6069082811D067
:10BEA0001DE0E749A06D084040EA064020F4F85044
:10BEB000A065D3E70AEB02100162DBE70AEB021090
:10BEC0004162EAE799F80000A268A16DF0B3DB488F
:10BED0000423083000EB82000022FFF72DFD99F8C3
:10BEE0000000A0B3042303991A465046FFF724FD2F
:10BEF00099F8000060B3D1480423002201211038D2
:10BF0000FFF71AFD049B4FF23F12DDE90010FFF727
:10BF100063FE6DB1AA685AB199F80000002828683C
:10BF200000EB070168683BD013461022FFF72DFD98
:10BF3000103511D0AA687AB199F800000028286855
:10BF400000EB070168682ED0134602E01AE01DE0FE
:10BF50001FE01022FFF719FDD4F8841041450CD1E1
:10BF60002069012809D099F8002005AB2046294610
:10BF7000012A3A461AD000F09DFD05981035012897
:10BF800017D019E00AEB82008162A8E70398CAF88B
:10BF900000000F21CAF814100121CAF81010B1E7EF
:10BFA000FCF707FAC4E7FCF704FAD5E7FFF708FD4A
:10BFB000E3E70120CBF800000198A6F50476401EC7
:10BFC00001907FF51EAF0398B0F5405F09D099F856
:10BFD00000009C49D8B19948042300228430FFF71F
:10BFE000ABFCE16D0298814208D099F8000088B15D
:10BFF0009248042300228C30FFF79EFCDBF80000FF
:10C0000001283FF460AE0599CBF800105BE6CAF852
:10C01000A410E6E7CAF8AC10F0E72DE9FF4F04469C
:10C02000894885B0006850B3844F91F85001E037DB
:10C0300078B38D6801F11006D1F854010490D1F85D
:10C0400058014FF0DA5A039091F8610192F86111AA
:10C05000DFF8F88140EA0120B0F5845F0CD04DF2A2
:10C06000600101EB004198F80000E0B1734804233F
:10C0700000228030FFF760FC681EC5B916E0089901
:10C08000012008607248016841F40051016009B064
:10C090001AE6FFE7956802F11006D2F85401049001
:10C0A000D2F85801CDE7CAF8A010E5E7284640F2DB
:10C0B000102100F0B2EF8346206D20F4E07040EADA
:10C0C0008B11216560690828606D20F0006001D146
:10C0D00040F00060606522693620032A00D03920D4
:10C0E000019098F800004546A268B0B15348042377
:10C0F00000EB02100022FFF71FFC2878A268616D98
:10C1000078B14E480423001D00EB02100022FFF717
:10C1100013FC6069082808D014E00AEB02100162E1
:10C12000EBE70AEB02104162F3E72878A268A16D01
:10C1300000287ED041480423083000EB8200002212
:10C14000FFF7FAFB2878216E002874D03B480423BF
:10C150000022D030FFF7F0FBA94600250095B0681B
:10C1600068B330F003080BD099F800000028D6E936
:10C17000000138446FD008224346FFF706FC4546CD
:10C18000B16841451BD901216846FDF784FF00983D
:10C190004FF0FF310160B2687368A2EB080203EB55
:10C1A0000801FCF706F999F80000002807EB0500E4
:10C1B00076D0009904230822FFF7E7FB2D1DF068D5
:10C1C000A8420AD999F80010A1B31F49431B781956
:10C1D00008220968FFF7D9FBF5681036B068C8B3C4
:10C1E00030F003080BD099F800007168002807EBC5
:10C1F000050061D008224346FFF7C7FB4544B168FC
:10C2000041452FD901216846FDF745FF00984FF0C1
:10C21000FF310160B2687368A2EB080203EB08010A
:10C22000FCF7C7F899F80000002807EB050047D095
:10C2300012E029E039E02BE0FF01F8FF2000401B6D
:10C24000FFFF00FC00300FF040F97041F0F6704144
:10C25000F4F6704106E01FE0009904230822FFF77E
:10C2600094FB2D1DB5F5047F0DD299F8000060B345
:10C27000FE4978190822C5F504730968FFF785FBA4
:10C280002069012829D078E00AEB8200816259E711
:10C29000CAF8F01060E703E04246FCF78AF86EE760
:10C2A00000990422FCF785F888E7F049421B7819C9
:10C2B0000968FCF77EF88FE74246FCF77AF89DE7BD
:10C2C00000990422FCF775F8CBE7E8497819C5F521
:10C2D00004720968FCF76DF8D2E7E549206D084063
:10C2E00040EA452020F0F06020656169082925D0EA
:10C2F00020F4F000206599F800004D46A268216DF9
:10C3000028B3DC48042300EB02100022FFF714FBE3
:10C31000606D40F480314FF6C070814361652878CC
:10C32000A268C0B1D3480423001D00EB0210002214
:10C33000FFF702FB6069082811D01CE0CE49A06D10
:10C34000084040EA054020F4F850A065D3E70AEB26
:10C3500002100162DCE70AEB02104162EAE728788A
:10C36000A268A16DE8B3C3480423083000EB820043
:10C370000022FFF7E1FA3620019099F8000010360C
:10C380004D4678B3042301991A465046FFF7D4FA74
:10C39000287840B3B7480423002201211038FFF762
:10C3A000CBFADDE903314FF23F125846FFF714FC98
:10C3B0002069012814D02878012811D0002002908B
:10C3C0002878A8B3AB49042300220C3902A8FFF750
:10C3D000DCFA029810F4887F02D0089901200860E6
:10C3E00002E017E01AE01FE0BBF1010B7FF5B5AEEC
:10C3F0000198B0F5845F09D099F800009F49E0B139
:10C400009C48042300228030FFF796FA0899002008
:10C4100008603CE60AEB82008162ACE70F21CAF8B3
:10C4200014100199CAF800100120CAF81000B8E7EA
:10C43000FFE7DAF814000290CCE7CAF8A010E5E7AD
:10C440002DE9F04F85B004464FF23F100E46DFF85D
:10C4500030824FF0DA550190934691F850014FF039
:10C46000010A89694FF000090491022896F8617168
:10C47000D6F854110291D6F85811009106F5AE7114
:10C4800003911CD001287ED0FF2F0CD07D4840EABC
:10C49000074198F80000002876D07648042300224F
:10C4A0008830FFF749FA206D20F4E070206598F895
:10C4B0000000A168012801F0010166D0FDE071686B
:10C4C0002046039AFFF72EFB049804287ED8902F6D
:10C4D00010D0702F02D14FF23F0001906A4847EA16
:10C4E000000198F8000080B16248042300228830DF
:10C4F000FFF722FA206D20F4E071216560690828B9
:10C50000606D20F0006003D004E0C5F8A810F1E7EA
:10C5100040F00060606598F80000C0B1A268042394
:10C52000544800EB02100022FFF706FA98F80000CA
:10C5300090B150480423A268001D616D00EB021009
:10C540000022FFF7F9F9606908280BD017E0A0680E
:10C5500005EB00100162E9E7A168606D05EB0111D0
:10C560004862F0E798F8000088B342480423A268C4
:10C570000830A16D00EB82000022FFF7DDF998F88A
:10C580000000F0B302E08CE093E095E0394804232A
:10C59000E16D00228C30FFF7CFF998F8000088B3E6
:10C5A00034480423216E0022D030FFF7C5F998F8F3
:10C5B0000000444638B32F48002204231146C030FF
:10C5C000FFF7BAF92078C0B3042301E062E036E057
:10C5D0000B211A462846FFF7AFF9207870B325489B
:10C5E0000423002201211038FFF7A6F9009B002048
:10C5F000DDE90121FFF7F0FA98F80000444698B30E
:10C6000002E022E024E026E01A49042370691022A7
:10C610002031FFF7BAF9902F0AD02078002879D07E
:10C62000194904231348002290318830FFF784F918
:10C63000CBF8009005B0BDE8F08F0EE011E0A168E6
:10C64000A06D05EB8101886299E7E06DC5F8AC004B
:10C65000206EC5F8F000C5F8E0900F2068610B204F
:10C660002860C5F810A0C1E710E0000040F9704153
:10C67000FF01F8FF2000401BFFFF00FC60D080108E
:10C68000F0F67041907000F00070FFF0286C716956
:10C690000860C0E700225B4631462046FFF7F4FA07
:10C6A000C6E7FD48C2F800A0016841F080010160C2
:10C6B000C0E7C5F8A810F6E6091D6369082B636D8D
:10C6C00023F0006301D143F00063636518B3F348BE
:10C6D00004230022FFF730F998F80000E0B1EF489A
:10C6E0000423A2681430216D00EB02100022FFF732
:10C6F00023F998F80000A8B1E8480423A26818308C
:10C70000616D00EB02100022FFF716F9606908283E
:10C710000ED01AE075E0E960A168206D05EB01110B
:10C720000862E6E7A168606D05EB01114862EDE77C
:10C7300098F80000F0B3D9480423A2681C30A16D1A
:10C7400000EB82000022FFF7F7F898F8000090B3A2
:10C75000D2480423E16D0022A030FFF7EDF898F8ED
:10C76000000048B3CD480423216E0022E430FFF7D7
:10C77000E3F898F8000098B3C84800220423114653
:10C78000D430FFF7D9F8716819B1039A2046FFF742
:10C79000C9F998F80000444660B3042328460D21E7
:10C7A0001A46FFF7C9F8207840B30423BB4800229B
:10C7B000012102E00EE014E016E0001DFFF7BCF8D6
:10C7C000009B0020DDE90121FFF706FAFF2F7FF42F
:10C7D00024AF2DE7A168A06D05EB81018862B4E765
:10C7E00005E0E06DC5F8AC00206EC5F8F000C5F8B6
:10C7F000E090C8E70F2068610D202860C5F810A000
:10C80000DEE7A748C5F8A80012E72DE9FC5F04465B
:10C8100091F8610190468A4601F5B2750A4691F891
:10C82000C512AB464FF0010940EA012692F85011BB
:10C83000994839B1C8F80090016841F08001016061
:10C84000BDE8FC9F95F85071696831B1016841F00D
:10C8500080010160C8F80090F2E7516802F5AE72FD
:10C860002046FFF75FF9022F29D0012F30D0002F8B
:10C87000E6D1DFF830A24DF2600B5E454FF0DA579B
:10C880000AD09AF8000046F0845150B3834804233C
:10C8900000229430FFF750F8D5F854010190D5F8F4
:10C8A000580100908049206D084020F4E071216516
:10C8B00060690828606D20F0006015D016E002B0B5
:10C8C00043465A4651462046BDE8F05FFFF7DCB9C3
:10C8D00002B043465A4651462046BDE8F05FFFF796
:10C8E0009CBBC7F8A010D7E740F0006060659AF8DD
:10C8F000000055460028A06817D0684A0423143267
:10C9000002EB00100022FFF717F8287888B1634A7D
:10C910000423A0681832616D02EB00100022FFF7BB
:10C920000BF8606908280AD019E007EB00100162D3
:10C93000EBE7A168606D07EB01114862F1E75B4826
:10C94000A16D0140A16528780028A06837D0534A1E
:10C9500004231C3202EB80000022FEF7EDFF287852
:10C9600088B34E480423216E0022E430FEF7E4FF32
:10C97000287848B3042338463A211A46FEF7DCFFEC
:10C98000287848B34548042300220121001DFEF702
:10C99000D3FF00204FF23F12DDE90031FFF71CF911
:10C9A0005E4508D028784249C8B13C48042300229B
:10C9B0009430FEF7C1FF0021C8F8001040E707EBF4
:10C9C00080008162CBE700E002E0206EC7F8F00053
:10C9D0000F2078613A203860C7F81090D9E7C7F87F
:10C9E000A010E8E72DE9F84380460C4600201646E3
:10C9F0000090012710602068D4F8541100F0010560
:10CA00003846294300D000206A4600282146404687
:10CA100008D0FFF7FAFED4F8640104F5327400F090
:10CA2000010503E0FFF70CFD04F5B274009800B1B6
:10CA30003060002DDFD0BDE8F883F8B54C680746BC
:10CA4000154E0020009015461060BCB16A46214684
:10CA50003846FFF7C7FF01E004F5B2742068C0074D
:10CA6000FAD02068C0F30031009800B12860002996
:10CA700004F5B274EAD02868012805D0306800288F
:10CA800008D0B0F5006F05D0306840F480503060B9
:10CA900001202860F8BD0000F4F670410C00401B36
:10CAA0009070FFF0F0F67041FF01F8FFFFFF00FC0F
:10CAB00060D080102DE9F84F00F110000E460021E3
:10CAC000924600910F25D0E91E890068A6F1100753
:10CAD0001C46032800D10A254B480078A0B14B49D9
:10CAE000042300226846FEF750FF00984FF0010231
:10CAF00010F4887F0DD02260796851F808104945FC
:10CB000025D10820206007E04FF0DA5040690090FE
:10CB1000ECE7206808281AD1F968002033689942A8
:10CB200001D1F36819440AEB810105E00B685B1C35
:10CB300000D02260091D401CB0EB950FF6D3206891
:10CB4000082804D13248016841F400610160BDE861
:10CB5000F88F2DE9F05F4FF0010AC2F800A090466F
:10CB600002688B460021920345D50823C8F800309F
:10CB700041E0426803691268934202D0C8F800A0FD
:10CB80003EE086690A2500F1140401F101092846F6
:10CB90000021FDF7B3FAE1682269084031680240DC
:10CBA0000140914202D0C8F800A003E0361D2D1FBD
:10CBB000002DECDCA5680A2D19D96768E6680837EE
:10CBC000083D12E0042D04DA00212846FDF796FA0C
:10CBD00006403868216930403140884203D009213D
:10CBE000C8F8001003E03F1D2D1F002DEADC04F102
:10CBF000140009F10101594502D202689203B8D428
:10CC00000846BDE8F09F0000F0F670411400401B9C
:10CC1000F4F67041002000F0C3FAAFF30080012069
:10CC200000F0B8FA40EA010310B59B070DD1042AC1
:10CC30000BD310C808C9121F9C42F8D021BA1ABAE7
:10CC40000120914200D8801E10BD1AB1D30703D035
:10CC5000521C07E0002010BD10F8013B11F8014BF9
:10CC60001B1B07D110F8013B11F8014B1B1B01D115
:10CC7000921EF1D1184610BD421C02E010F8011BB3
:10CC800069B18107FAD14FF0013302C8C3FA51F1FB
:10CC90000029FAD0801A0A0603D0C01E7047801AF5
:10CCA00070470A0401D0801E70470902FCD0401E64
:10CCB00070470000013080E170402DE9030013E36C
:10CCC000D8609F052000001A040052E31E00003ABD
:10CCD000043090E4044091E4042042E2F35F66E60D
:10CCE000000055E31000000AFF0003E2FF1004E219
:10CCF000010040E0051C90E17080BD187300FFE664
:10CD00007410FFE6010040E0051890E17080BD1846
:10CD1000FF04C3E3FF14C4E3010040E0051490E105
:10CD2000230CA001240C40007080BDE8040053E1F6
:10CD3000E4FFFF0A330FBFE6341FBFE6010050E1F6
:10CD40000000E0930100A0837080BDE8000052E382
:10CD50000000A0037080BD080130D0E40140D1E4A0
:10CD6000000053E30B00000A040053E10900001A1D
:10CD7000012052E20700000A0130D0E40140D1E472
:10CD8000000053E30300000A040053E10100001A0D
:10CD9000012052E2EFFFFF1A040043E07080BDE87B
:10CDA0000101010101402DE9010000EB0180BDE816
:10CDB0007847C046030052E32A00009A03C010E2FD
:10CDC0000800000A0130D1E402005CE30C2082E09C
:10CDD00001C0D1940130C0E40130D13401C0C0940D
:10CDE000042042E20130C034033011E22500000A81
:10CDF000042052E21B00003A03C031E7020053E373
:10CE00000800000A0F00008A2C34A0E104C0B1E53C
:10CE1000042052E20C3C83E1043080E4F9FFFF2A55
:10CE2000011081E20F0000EA2C38A0E104C0B1E556
:10CE3000042052E20C3883E1043080E4F9FFFF2A39
:10CE4000021081E2070000EA2C3CA0E104C0B1E539
:10CE5000042052E20C3483E1043080E4F9FFFF2A1D
:10CE6000031081E20000A0E1822FB0E10130D12463
:10CE700001C0D1240120D1440130C02401C0C0240C
:10CE80000120C0441EFF2FE110402DE9202052E276
:10CE90000500003A1850B1E8202052E21850A0E8EE
:10CEA0001850B1E81850A0E8F9FFFF2A02CEB0E10F
:10CEB0001850B1281850A0281800B1481800A048F0
:10CEC0001040BDE802CFB0E104309124043080244A
:10CED0001EFF2F01822FB0E1B230D1200120D144BA
:10CEE000B230C0200120C0441EFF2FE101F0FF033B
:10CEF000114601B543EA032242EA024200F059F921
:10CF000001BD02F0FF0343EA032242EA024200F0BD
:10CF100050B94FF0000200B51346944696462039AA
:10CF200022BFA0E80C50A0E80C50B1F12001BFF4E2
:10CF3000F7AF090728BFA0E80C5048BF0CC05DF848
:10CF400004EB890028BF40F8042B08BF704748BF96
:10CF500020F8022B11F0804F18BF00F8012B70470A
:10CF6000030010E3030011031700001A00402DE92D
:10CF700084E09FE5042090E4043091E40EC042E098
:10CF800002C0CCE18EC31CE003005201F8FFFF0A8F
:10CF90000040BDE8030CA0E1020C50E0FF0E1C03B2
:10CFA0000700001A0308A0E1020850E0FF0C1C0370
:10CFB0000300001A0304A0E1020450E0FF081C0370
:10CFC000020053006000A0111EFF2FE10120D0E4F9
:10CFD0000130D1E4010052E3030052210400001AA1
:10CFE0000120D0E40130D1E4010052E303005221DA
:10CFF000F5FFFF0A030042E01EFF2FE101010101DE
:10D00000427801788378C07841EA022141EA0341FD
:10D0100041EA006070470000013090E12100004AC1
:10D020000020B0E3A03071E01A00003A203271E035
:10D030000F00003A203471E00100003A00C0A0E384
:10D04000200000EAA03371E0810340200220B2E01A
:10D05000203371E0010340200220B2E0A03271E0F1
:10D06000810240200220B2E0203271E00102402023
:10D070000220B2E0A03171E0810140200220B2E044
:10D08000203171E0010140200220B2E0A03071E0C7
:10D09000810040200220B2E0011050E00010A031D9
:10D0A0000200A2E01EFF2FE1022111E20010614206
:10D0B00040C032E000006022203271E01D00003AE2
:10D0C000203471E00F00003A0113A0E1203471E038
:10D0D0003F2382E30B00003A0113A0E1203471E00A
:10D0E0003F2682E30700003A0113A0E1203471E0FB
:10D0F0003F2982E30113A0213F2C8223003071E2FB
:10D100001D00002A2113A021A03371E081034020DB
:10D110000220B2E0203371E0010340200220B2E09F
:10D12000A03271E0810240200220B2E0203271E0A2
:10D13000010240200220B2E0A03171E081014020D4
:10D140000220B2E0203171E0010140200220B2E073
:10D15000EBFFFF2AA03071E0810040200220B2E006
:10D16000011050E00010A0310200A2E0CCCFB0E1ED
:10D1700000006042001061221EFF2FE1CCCFB0E121
:10D180000000604201402DE90000B0E30000A0E192
:10D190000280BDE801491820ABDFFEE7260002004F
:10D1A00010B500F02DF8BDE8104000F023B84FF0A6
:10D1B00000020429C0F0128010F0030C3FF4ABAE63
:10D1C000CCF1040CBCF1020F18BF00F8012BA8BF72
:10D1D00020F8022BA1EB0C01FFF79DBE5FEAC17C9A
:10D1E00024BF00F8012B00F8012B48BF00F8012BE9
:10D1F00070477047002801D0FFF7CCBF7047000090
:10D2000010B5002102A000F013F8012010BD0000AD
:10D21000534947414252543A2041626E6F726D61E8
:10D220006C207465726D696E6174696F6E000000C8
:10D2300070B505460C460A2000E06D1C00F011F8A0
:10D2400035B128780028F8D102E0641C00F009F814
:10D2500014B120780028F8D1BDE870400A20AFF35F
:10D26000008008B569468DF800000320ABDF08BDDB
:10D270000020B0E3203171E083FFFF3AA03271E07B
:10D2800078FFFF3A203471E06DFFFF3A00C0A0E361
:10D290008CFFFFEA0000000000000000000000001A
:10D2A0000B10A0E3910000E0A002A0E1010050E219
:10D2B000FDFFFFCA1EFF2FE1912000E10200A0E167
:10D2C0001EFF2FE19F1F90E10100A0E11EFF2FE153
:10D2D000912F80E10200A0E11EFF2FE1FF472DE921
:10D2E0000080A0E10190A0E102A0A0E120005AE3AB
:10D2F000020000AA00005AE3060000CAFF87BDE84A
:10D30000FF00B9E8FF00A8E820A04AE220005AE3A5
:10D31000FAFFFFAAF6FFFFBA0100B9E80100A8E88A
:10D3200004A04AE200005AE3FAFFFFCAF2FFFFDA64
:10D330007847C046D9FFFFEA10B591EA030F48BF0E
:10D3400083F0004300F1E681841A71EB030C05D2EF
:10D35000121943EB0C03001B61EB0C01DFF824E115
:10D360004FEA1154A4EB135C1EEA430F18BF9EEA68
:10D37000445F73D023EA0E03DCF1200E21EA04514E
:10D3800043F4801332D322FA0CFE10EB0E0023FA82
:10D390000CFE41EB0E01CCF1200E03FA0EFE10EB59
:10D3A0000E0051F10001B1F5801FCCF1200E32D2F8
:10D3B00001EB045112FA0EF2BDE8104058BF70475D
:10D3C000401C38BF5FEA420218BF7047002814BFF4
:10D3D00020F0010041F100014FEA410313F5001F65
:10D3E00038BF7047A1F1C04100F086B9012A43EB74
:10D3F0000302ACF1200CDCF11F0E32BF4FF0000E27
:10D4000023FA0CF310EB030041EB0451B4EB115F72
:10D41000D0D0A1EB045101F5801149085FEA30003A
:10D4200001EB04510ED350F1000038BF12FA0EFE8A
:10D4300008D1BDE81040C9E7401C38BF5FEA42028E
:10D44000CAD1C3E7BDE810404FEA410313F5001FFE
:10D4500038BF7047A1F1C04100F04EB99EEA445F69
:10D4600008D011EA5E0FBDE8104004BF01F0004192
:10D4700000207047BDE8104070B500F0EFF800BF25
:10D4800064FBBE3E0000E0FF4FEA1153A3F580634A
:10D49000D3F11E03A8BFD3F1200C08DB4FF00042EC
:10D4A00042EAC12252EA505232FA03F0704709426E
:10D4B0000BD4102BC4BF0020704703F5787CBCF15F
:10D4C000FF3F05D04FF0FF3070474FF0000070472E
:10D4D00070B500F0C3F800BF499224800020704767
:10D4E000F0E7B0FA80F310FA03F10AD0C3F11D039C
:10D4F00003F580634FEA41504FEA035202EBD1211A
:10D5000070474FF000007047DFF848C170B51CEA63
:10D51000111E1EBF1CEA13159EEA0C0F95EA0C0F94
:10D5200000F06F8081EA030423EA4C134EEAD47EB4
:10D5300021EA4C1141F4801143F48013AE44A1FB65
:10D54000024CA0FB0365AEF17F7E361955EB0C054E
:10D55000A1FB034C4CF10003A0FB021C16EB0C06D4
:10D56000654153F10003094218BF46F0010613F468
:10D57000007F0BD14FEA03314FEA0530340341EA13
:10D58000155140EA16506FF003020AE04FEAC3213A
:10D590004FEAC520F40241EA555140EA56506FF077
:10D5A000020202EB2E4201EB025585EACE710AD04F
:10D5B0005FEA440C18BF24F0004450F1000041F130
:10D5C000000120EAD47040F2FE7C624500D270BDBA
:10D5D000A84214BF4FF080444FF04044002E08BFD3
:10D5E0000024BEF1806FA8BFA1F1C041BDE870402A
:10D5F00080F282804FF0000001F1C04101F0004153
:10D6000070479EEA0C0F0CEA131518BF95EA0C0F31
:10D6100006D04FF0000081EA030E0EF0004170BD0D
:10D6200000F01CF88900013E00F007B800F009B8CE
:10D630004FEA430C5FEA5C5C08D081EA030100F02A
:10D640005BB84FEA410C5FEA5C5CF6D14FF000003A
:10D65000014970470000FF070000F87F0EF1020E3D
:10D660002EF0030E5EF8046B364205D4012A43EB1C
:10D67000030515F5001F12D8012841EB010C1CF51C
:10D68000001F0CD80ED14FEAD17C15F5001F0CEB12
:10D690004C0C0CF1020C08BF4CEBD37C04E04FF0B7
:10D6A000080C01E04FEAD37C0CEB4C0526FA05F69A
:10D6B00006F00706B6F1040C06D20EEB860CBDE8A8
:10D6C00070404CF0010C6047DFE80CF0090B0202DF
:10D6D0004FF000414FF00000A1F5002170BD194648
:10D6E0001046012851EB010418BFD4F5001484BF83
:10D6F000002001F0004170BD0808A0F500114FEABC
:10D700003101704710B591EA030F48BF83F0004321
:10D710003FF51AAE841A71EB030C07D212198CF084
:10D72000004C43EB0C03001B61EB0C01DFF8A4E1A0
:10D730004FEA1154A4EB135C1EEA430F18BF9EEA94
:10D74000445F00F0B08023EA6E03524221EA0451A4
:10D75000C3EB6E0338BF5B1EDCF1200E25D322FA2B
:10D760000CFE10EB0E0043FA0CFE41EB0E01CCF167
:10D77000200E03FA0EFE10EB0E0051F10001CCF169
:10D78000200E29D412FA0EF201EB0451BDE810402C
:10D7900058BF7047401C1CBFB2F1004F70470028B3
:10D7A0000CBF491C20F00100704712EB020E43EB46
:10D7B000030218BF4FF0010E4EEA4202ACF1200CFA
:10D7C000DCF11E0E54D943FA0CFE10EB0E0051F1A1
:10D7D000FF31CCF11E0ED5D50EF1010E12FA0EFE60
:10D7E000404141EB010101EB445C5FEA5C5C10D914
:10D7F00010EBDE7001EB045138BFBEF1004FBDE805
:10D80000104018BF704700280CBF491C20F00100D1
:10D81000704730D24FEAD42C11F5001124F4006483
:10D820001BD0B1FA81F20B3AA41AA41ED2F1200344
:10D83000914030FA03F31943904001EBCC71002C76
:10D8400001EB0451BDE81040A8BF704701F1C04191
:10D850004FF0000001F000417047B0FA80F310FA79
:10D8600003F100D110BDE41A173C4805C90AE4E7EA
:10D8700001EB045110BD491001EB0451BDE810400B
:10D880004FEA300002E04FF0000170474A0008BF45
:10D890000042F8D0B2F5001F28BF704701F00041E8
:10D8A0004FF0000070479EEA445F07D011EA5E0F18
:10D8B000BDE8104004BF002100207047BDE81040C3
:10D8C00070B5FFF7CBFE00BF40DFF63E83F00041AE
:10D8D000104670470000E0FF41524D505247207300
:10D8E000697A65206D7367206F76657272756E0058
:10D8F000546F74616C20627974657320726563641F
:10D900002062792041524D5052472030780000006B
:10D9100000000000C7B9302049CA51208E73610051
:10D92000552D93209294A3001CE7C200DB5EF220E9
:10D930006DE31621AA5A260124294701E390772195
:10D9400038CE8501FF77B5217104D421B6BDE4013D
:10D950001D7F1D22DAC62D0254B54C02930C7C2289
:10D9600048528E028FEBBE220198DF22C621EF02C1
:10D97000709C0B03B7253B2339565A23FEEF6A03ED
:10D9800025B19823E208A8036C7BC903ABC2F92335
:10D99000FD470A243AFE3A04B48D5B0473346B24C9
:10D9A000A86A99046FD3A924E1A0C8242619F80411
:10D9B00090A41C05571D2C25D96E4D251ED77D051D
:10D9C000C5898F250230BF058C43DE054BFAEE2555
:10D9D000E038170627812726A9F246266E4B7606E1
:10D9E000B515842672ACB406FCDFD5063B66E52689
:10D9F0008DDB01274A623107C411500703A8602755
:10DA0000D8F692071F4FA227913CC3275685F307EC
:10DA10003D362428FA8F140874FC7508B345452850
:10DA2000681BB708AFA2872821D1E628E668D60888
:10DA300050D53209976C0229191F6329DEA65309B4
:10DA400005F8A129C24191094C32F0098B8BC029FC
:10DA50002049390AE7F0092A6983682AAE3A580A48
:10DA60007564AA2AB2DD9A0A3CAEFB0AFB17CB2AE0
:10DA70004DAA2F2B8A131F0B04607E0BC3D94E2B8C
:10DA80001887BC0BDF3E8C2B514DED2B96F4DD0B34
:10DA9000C0712E0C07C81E2C89BB7F2C4E024F0C68
:10DAA000955CBD2C52E58D0CDC96EC0C1B2FDC2C10
:10DAB000AD92382D6A2B080DE458690D23E1592DDC
:10DAC000F8BFAB0D3F069B2DB175FA2D76CCCA0D74
:10DAD000DD0E332E1AB7030E94C4620E537D522E00
:10DAE0008823A00E4F9A902EC1E9F12E0650C10E48
:10DAF000B0ED250F7754152FF927742F3E9E440F54
:10DB0000E5C0B62F2279860FAC0AE70F6BB3D72F8B
:10DB1000BDD578307A6C4810F41F291033A619301F
:10DB2000E8F8EB102F41DB30A132BA30668B8A1057
:10DB3000D0366E11178F5E3199FC3F315E450F1163
:10DB4000851BFD3142A2CD11CCD1AC110B689C31AB
:10DB5000A0AA651267135532E96034322ED9041237
:10DB6000F587F632323EC612BC4DA7127BF49732CF
:10DB7000CD4973330AF0431384832213433A12339B
:10DB80009864E0135FDDD033D1AEB1331617811343
:10DB900040927214872B423409582334CEE1131477
:10DBA00015BFE134D206D1145C75B0149BCC80341F
:10DBB0002D716435EAC8541564BB3515A3020535CB
:10DBC000785CF715BFE5C7353196A635F62F961563
:10DBD0005DED6F369A545F1614273E16D39E0E36AF
:10DBE00008C0FC16CF79CC36410AAD3686B39D16F7
:10DBF000300E7917F7B7493779C42837BE7D181723
:10DC00006523EA37A29ADA172CE9BB17EB508B375A
:10DC100080E35C18475A6C38C9290D380E903D18BE
:10DC2000D5CECF381277FF189C049E185BBDAE3856
:10DC3000ED004A392AB97A19A4CA1B1963732B3922
:10DC4000B82DD9197F94E939F1E78839365EB819CA
:10DC50009D9C413A5A25711AD456101A13EF203A56
:10DC6000C8B1D21A0F08E23A817B833A46C2B31A8E
:10DC7000F07F571B37C6673BB9B5063B7E0C361B9A
:10DC8000A552C43B62EBF41BEC98951B2B21A53BE2
:10DC90007DA4563CBA1D661C346E071CF3D7373C76
:10DCA0002889C51CEF30F53C6143943CA6FAA41CBE
:10DCB0001047401DD7FE703D598D113D9E34211DEA
:10DCC000456AD33D82D3E31D0CA0821DCB19B23D22
:10DCD00060DB4B1EA7627B3E29111A3EEEA82A1E6E
:10DCE00035F6D83EF24FE81E7C3C891EBB85B93E16
:10DCF0000D385D3FCA816D1F44F20C1F834B3C3FC2
:10DD00005815CE1F9FACFE3F11DF9F3FD666AF1F59
:10DD100000002110422063308440A550C660E770A7
:10DD2000088129914AA16BB18CC1ADD1CEE1EFF14F
:10DD30003112100273325222B5529442F772D662F7
:10DD4000399318837BB35AA3BDD39CC3FFF3DEE39F
:10DD50006224433420040114E664C774A444855447
:10DD60006AA54BB528850995EEE5CFF5ACC58DD5EF
:10DD70005336722611163006D776F6669556B44697
:10DD80005BB77AA719973887DFF7FEE79DD7BCC73F
:10DD9000C448E5588668A7784008611802282338E7
:10DDA000CCC9EDD98EE9AFF9488969990AA92BB98F
:10DDB000F55AD44AB77A966A711A500A333A122A37
:10DDC000FDDBDCCBBFFB9EEB799B588B3BBB1AABDF
:10DDD000A66C877CE44CC55C222C033C600C411C87
:10DDE000AEED8FFDECCDCDDD2AAD0BBD688D499D2F
:10DDF000977EB66ED55EF44E133E322E511E700ED7
:10DE00009FFFBEEFDDDFFCCF1BBF3AAF599F788F7E
:10DE10008891A981CAB1EBA10CD12DC14EF16FE15E
:10DE20008010A100C230E320045025404670676096
:10DE3000B9839893FBA3DAB33DC31CD37FE35EF3AE
:10DE4000B1029012F322D2323542145277625672E6
:10DE5000EAB5CBA5A89589856EF54FE52CD50DC5FE
:10DE6000E234C324A0148104667447642454054436
:10DE7000DBA7FAB79987B8975FE77EF71DC73CD74E
:10DE8000D326F2369106B016576676761546345686
:10DE90004CD96DC90EF92FE9C899E9898AB9ABA99E
:10DEA0004458654806782768C018E1088238A328D6
:10DEB0007DCB5CDB3FEB1EFBF98BD89BBBAB9ABBEE
:10DEC000754A545A376A167AF10AD01AB32A923A26
:10DED0002EFD0FED6CDD4DCDAABD8BADE89DC98D3E
:10DEE000267C076C645C454CA23C832CE01CC10C76
:10DEF0001FEF3EFF5DCF7CDF9BAFBABFD98FF89F8E
:10DF0000176E367E554E745E932EB23ED10EF01EC5
:10DF10000000891112239B322446AD573665BF7429
:10DF2000488CC19D5AAFD3BE6CCAE5DB7EE9F7F8D9
:10DF30008110080193331A22A5562C47B7753E6409
:10DF4000C99C408DDBBF52AEEDDA64CBFFF976E8B9
:10DF500002218B30100299132667AF763444BD55E9
:10DF60004AADC3BC588ED19F6EEBE7FA7CC8F5D999
:10DF700083310A2091121803A7772E66B5543C45C9
:10DF8000CBBD42ACD99E508FEFFB66EAFDD874C979
:10DF900004428D5316619F702004A9153227BB36A9
:10DFA0004CCEC5DF5EEDD7FC6888E1997AABF3BA59
:10DFB00085520C4397711E60A1142805B3373A2689
:10DFC000CDDE44CFDFFD56ECE9986089FBBB72AA39
:10DFD00006638F7214409D512225AB343006B91769
:10DFE0004EEFC7FE5CCCD5DD6AA9E3B8788AF19B19
:10DFF00087730E6295501C41A3352A24B116380749
:10E00000CFFF46EEDDDC54CDEBB962A8F99A708BF8
:10E01000088481951AA793B62CC2A5D33EE1B7F028
:10E020004008C919522BDB3A644EED5F766DFF7CD8
:10E03000899400859BB712A6ADD224C3BFF136E008
:10E04000C1184809D33B5A2AE55E6C4FF77D7E6CB8
:10E050000AA583B4188691972EE3A7F23CC0B5D1E8
:10E060004229CB38500AD91B666FEF7E744CFD5D98
:10E070008BB502A499961087AFF326E2BDD034C1C8
:10E08000C3394A28D11A580BE77F6E6EF55C7C4D78
:10E090000CC685D71EE597F42880A1913AA3B3B2A8
:10E0A000444ACD5B5669DF78600CE91D722FFB3E58
:10E0B0008DD604C79FF516E4A9902081BBB332A288
:10E0C000C55A4C4BD7795E68E11C680DF33F7A2E38
:10E0D0000EE787F61CC495D52AA1A3B03882B19368
:10E0E000466BCF7A5448DD59622DEB3C700EF91F18
:10E0F0008FF706E69DD414C5ABB122A0B992308348
:10E10000C77B4E6AD5585C49E33D6A2CF11E780FF7
:10E1100000000000B71DC1046E3B8209D926430DE3
:10E12000DC7604136B6BC517B24D861A0550471E7B
:10E13000B8ED08260FF0C922D6D68A2F61CB4B2B1B
:10E14000649B0C35D386CD310AA08E3CBDBD4F38C3
:10E1500070DB114CC7C6D0481EE09345A9FD524163
:10E16000ACAD155F1BB0D45BC2969756758B5652FB
:10E17000C836196A7F2BD86EA60D9B6311105A679B
:10E1800014401D79A35DDC7D7A7B9F70CD665E7443
:10E19000E0B6239857ABE29C8E8DA19139906095A3
:10E1A0003CC0278B8BDDE68F52FBA582E5E66486BB
:10E1B000585B2BBEEF46EABA3660A9B7817D68B3DB
:10E1C000842D2FAD3330EEA9EA16ADA45D0B6CA003
:10E1D000906D32D42770F3D0FE56B0DD494B71D923
:10E1E0004C1B36C7FB06F7C32220B4CE953D75CA3B
:10E1F00028803AF29F9DFBF646BBB8FBF1A679FF5B
:10E20000F4F63EE143EBFFE59ACDBCE82DD07DEC82
:10E2100077708634C06D4730194B043DAE56C53912
:10E22000AB0682271C1B4323C53D002E7220C12A4A
:10E23000CF9D8E1278804F16A1A60C1B16BBCD1F4A
:10E2400013EB8A01A4F64B057DD00808CACDC90C92
:10E2500007AB9778B0B6567C69901571DE8DD47592
:10E26000DBDD936B6CC0526FB5E6116202FBD066CA
:10E27000BF469F5E085B5E5AD17D1D576660DC53CA
:10E2800063309B4DD42D5A490D0B1944BA16D84012
:10E2900097C6A5AC20DB64A8F9FD27A54EE0E6A152
:10E2A0004BB0A1BFFCAD60BB258B23B69296E2B20A
:10E2B0002F2BAD8A98366C8E41102F83F60DEE878A
:10E2C000F35DA9994440689D9D662B902A7BEA9452
:10E2D000E71DB4E0500075E4892636E93E3BF7EDD2
:10E2E0003B6BB0F38C7671F7555032FAE24DF3FE8A
:10E2F0005FF0BCC6E8ED7DC231CB3ECF86D6FFCB0A
:10E300008386B8D5349B79D1EDBD3ADC5AA0FBD8D1
:10E31000EEE00C6959FDCD6D80DB8E6037C64F6431
:10E320003296087A858BC97E5CAD8A73EBB04B77E9
:10E33000560D044FE110C54B383686468F2B4742A9
:10E340008A7B005C3D66C158E4408255535D435171
:10E350009E3B1D252926DC21F0009F2C471D5E28B1
:10E36000424D1936F550D8322C769B3F9B6B5A3B69
:10E3700026D6150391CBD40748ED970AFFF0560E29
:10E38000FAA011104DBDD014949B93192386521DF1
:10E390000E562FF1B94BEEF5606DADF8D7706CFCF1
:10E3A000D2202BE2653DEAE6BC1BA9EB0B0668EF29
:10E3B000B6BB27D701A6E6D3D880A5DE6F9D64DA69
:10E3C0006ACD23C4DDD0E2C004F6A1CDB3EB60C9B1
:10E3D0007E8D3EBDC990FFB910B6BCB4A7AB7DB071
:10E3E000A2FB3AAE15E6FBAACCC0B8A77BDD79A3A9
:10E3F000C660369B717DF79FA85BB4921F467596E9
:10E400001A163288AD0BF38C742DB081C330718530
:10E4100099908A5D2E8D4B59F7AB085440B6C95080
:10E4200045E68E4EF2FB4F4A2BDD0C479CC0CD4398
:10E43000217D827B9660437F4F460072F85BC176F8
:10E44000FD0B86684A16476C93300461242DC56520
:10E45000E94B9B115E565A1587701918306DD81C00
:10E46000353D9F0282205E065B061D0BEC1BDC0F18
:10E4700051A69337E6BB52333F9D113E8880D03A78
:10E480008DD097243ACD5620E3EB152D54F6D429A0
:10E490007926A9C5CE3B68C1171D2BCCA000EAC8C0
:10E4A000A550ADD6124D6CD2CB6B2FDF7C76EEDB58
:10E4B000C1CBA1E376D660E7AFF023EA18EDE2EE38
:10E4C0001DBDA5F0AAA064F4738627F9C49BE6FDE0
:10E4D00009FDB889BEE0798D67C63A80D0DBFB8440
:10E4E000D58BBC9A62967D9EBBB03E930CADFF97D8
:10E4F000B110B0AF060D71ABDF2B32A66836F3A2B8
:10E500006D66B4BCDA7B75B8035D36B5B440F7B15F
:10E510003031323334353637383941424344454659
:10E520000051434F4D206661737420646F776E6CA9
:10E530006F61642070726F746F636F6C20686F73AB
:10E54000740051434F4D206661737420646F776E81
:10E550006C6F61642070726F746F636F6C20746194
:10E56000726700040309043E035100750061006CEA
:10E570000063006F006D006D002000430044004DFB
:10E58000004100200054006500630068006E006FC9
:10E59000006C006F00670069006500730020004D8B
:10E5A0000053004D002403500072006F006400759A
:10E5B000006300740020006E0061006D00650020A3
:10E5C00000680065007200650022033100320033EC
:10E5D0000034003500360037003800390030004183
:10E5E0000042004300440045004600005D4B70417E
:10E5F0000000000054EF70416B68704102000000A1
:10E600000CF070416B687041CF68704107697041D0
:10E6100021697041276970412D69704133697041EA
:10E62000396970413F697041656870414569704161
:10E630004B69704151697041576970415D69704122
:10E6400063697041696970416F69704175697041B2
:10E650007B69704181697041876970418D69704142
:10E6600093697041996970419F697041A5697041D2
:10E67000AB697041070000008004E0049A41F0415A
:10E680008081E08100C000D000C000C000C000C098
:10E6900000C000C0070000008004E0049949F04574
:10E6A0008081E08100C000CC00C000C000C000C07C
:10E6B00000C000C0070000008004E0049A41F0415F
:10E6C0008081E08100C400C400C000C000C000C060
:10E6D00000C000C0000000000000000000000000BA
:10E6E000000000000000000000000000000000002A
:10E6F00000000000000000001002000010020000F6
:10E700000000000000000000000200000A020000FB
:10E7100004000000000000000002000000020000F1
:10E7200004000000000000000402000010020000CD
:10E73000000000001002000004020000200400009D
:10E740000000000020040000040200003006000069
:10E750000000000030060000F40100002408000062
:10E760001000000000000000000200000A0200008B
:10E770000400000010020000000200001A04000063
:10E780000400000020040000000200002A0600002F
:10E790000400000030060000000200003A080000FB
:10E7A0000400000000000000100200001002000041
:10E7B0000000000010020000100200002004000011
:10E7C00000000000200400001002000030060000DD
:10E7D00000000000300600001002000040080000A9
:10E7E000000000000000000004020000140200000D
:10E7F00000000000140200000402000028040000D1
:10E800000000000028040000040200003C06000094
:10E81000000000003C060000F40100003008000089
:10E820001000000000000000000200000E020000C6
:10E830000400000014020000000200002204000096
:10E84000040000002804000000020000360600005A
:10E85000040000003C060000000200004A0800001E
:10E860000400000000000000140200001402000078
:10E870000000000014020000140200002804000040
:10E880000000000028040000140200003C06000004
:10E89000000000003C0600001402000050080000C8
:10E8A0000000000000000000040200001002000050
:10E8B000000000001002000004020000200400001C
:10E8C00000000000200400000402000030060000E8
:10E8D00000000000300600000402000040080000B4
:10E8E000000000004008000004020000500A000080
:10E8F00000000000500A000004020000600C00004C
:10E9000000000000600C000004020000700E000017
:10E9100000000000700E0000E40100005410000030
:10E920002000000000000000000200000A020000B9
:10E930000400000010020000000200001A040000A1
:10E940000400000020040000000200002A0600006D
:10E950000400000030060000000200003A08000039
:10E960000400000040080000000200004A0A000005
:10E9700004000000500A0000000200005A0C0000D1
:10E9800004000000600C0000000200006A0E00009D
:10E9900004000000700E0000000200007A10000069
:10E9A000040000000000000010020000100200003F
:10E9B000000000001002000010020000200400000F
:10E9C00000000000200400001002000030060000DB
:10E9D00000000000300600001002000040080000A7
:10E9E000000000004008000010020000500A000073
:10E9F00000000000500A000010020000600C00003F
:10EA000000000000600C000010020000700E00000A
:10EA100000000000700E00001002000080100000D6
:10EA200000000000000000000402000014020000CA
:10EA3000000000001402000004020000280400008E
:10EA40000000000028040000040200003C06000052
:10EA5000000000003C060000040200005008000016
:10EA6000000000005008000004020000640A0000DA
:10EA700000000000640A000004020000780C00009E
:10EA800000000000780C0000040200008C0E000062
:10EA9000000000008C0E0000E40100007010000077
:10EAA0002000000000000000000200000E02000034
:10EAB0000400000014020000000200002204000014
:10EAC00004000000280400000002000036060000D8
:10EAD000040000003C060000000200004A0800009C
:10EAE0000400000050080000000200005E0A000060
:10EAF00004000000640A000000020000720C000024
:10EB000004000000780C000000020000860E0000E7
:10EB1000040000008C0E0000000200009A100000AB
:10EB200004000000000000001402000014020000B5
:10EB3000000000001402000014020000280400007D
:10EB40000000000028040000140200003C06000041
:10EB5000000000003C060000140200005008000005
:10EB6000000000005008000014020000640A0000C9
:10EB700000000000640A000014020000780C00008D
:10EB800000000000780C0000140200008C0E000051
:10EB9000000000008C0E000014020000A010000015
:10EBA0000000000000000000000100000000000064
:10EBB0000000000000000000000000000000000055
:10EBC000F0D87041D8D8704100000000000000006B
:10EBD0000000000000000000000000000000000035
:10EBE0000000000000000000000000000000000025
:10EBF000303A445350310000D7087041C908704181
:10EC0000F1097041C9087041450B7041C908704154
:10EC1000530B7041C9087041F10B7041C908704134
:10EC2000030B7041C9087041C9087041C90870419F
:10EC3000C9087041C9087041290C7041C908704168
:10EC4000790C7041C908704111107041C9087041B8
:10EC500065107041C908704191107041C908704138
:10EC600081117041C9087041430C7041C90870415D
:10EC7000C9087041C9087041C9087041C90870418C
:10EC8000C9087041C9087041C9087041C90870417C
:10EC9000C9087041B7127041C9087041C908704174
:10ECA000C9087041C9087041C9087041C90870415C
:10ECB000C908704127127041C90870410200000064
:10ECC00000000000000000001C0351004800530039
:10ECD0005500530042005F00410052004D005000BB
:10ECE00052004700F11A70418F1A7041791A704131
:10ECF0006D1A7041751A7041000000006B1C704164
:10ED0000551C7041611B7041971B70410B1C704179
:10ED1000291C7041931C70413F1C70410000000091
:10ED200000000000000000000000000012010002CE
:10ED300000000040C6050890000001020001090221
:10ED4000200001010080010904000002FFFFFF0014
:10ED50000705810240000007050102400000820310
:10ED600000000000000000000000000000000000A3
:10ED70000000000000000000000000000000000093
:10ED80000000000000000000000000000000000083
:10ED90000000000000000000000000000000000073
:10EDA0000000000000000000000000000000000063
:10EDB0000000000000000000000000000000000053
:10EDC0000000000000000000000000000000000043
:10EDD0000000000000000000000000000000000033
:10EDE000F4ED70410000000008EE704100000000EA
:10EDF00000000000000000000000000008EE70416C
:10EE00000000000000000000000000000000000002
:10EE100020EE7041E0ED70410000000000000000B5
:10EE2000000000000000000030EE70410000000013
:10EE30000000000020EE7041CCEE704100000000A8
:10EE4000F71C7041000000000000000000000000FE
:10EE500000000000000000000000000000000000B2
:10EE600000000000000000000000000000000000A2
:10EE70000000000000000000000000000000000092
:10EE80000000000000000000000000000000000082
:10EE90000000000000000000000000000000000072
:10EEA0000000000000000000000000000000000062
:10EEB0000000000000000000000000000000000052
:10EEC000000000000000000000000000D8EE7041CB
:10EED00063E5704100000000E4EE704167E57041B9
:10EEE00009040100F0EE7041A5E57041090402003B
:10EEF00000000000C9E5704109040300F4010000AE
:10EF0000B5227041D9227041FD21704100000000FE
:10EF100000000000000000000000000000000000F1
:10EF200000000000000000000000000000000000E1
:10EF3000FFFFFFFF00000000FFFFFFFFFFFFFFFFDD
:10EF4000000000000000000000000000000050125F
:10EF50000000541203000002000000000000000046
:10EF600000000000FFFFFFFF0000000000000000A5
:10EF70000000000000000000500000003000000011
:10EF800038000000380000003800000003000000D6
:10EF9000000000003800000050000002480000009F
:10EFA0003F0100024C00000044616C456E76000099
:10EFB00002000000000000000102000000FF00FF4E
:10EFC00000FF00FF00FF00FF78EF704174EF704119
:10EFD0000000000000000000ECE57041F8E5704121
:10EFE00002000000D8EF70410000000000000000A7
:10EFF000000000000000000000000000FFFFFFFF15
:10F00000400C0800140000000A000000500000023C
:10F010003F010002000000000000000000000000AE
:10F02000A16B7041A56B704102000000D800000088
:10F0300000000000000000000000000000000000D0
:10F0400000000000000000000000000000000000C0
:10F0500000000000000000000000000000000000B0
:10F0600000000000000000000000000000000000A0
:10F070000000000000000000000000000000000090
:10F080000000000000000000000000000000000080
:10F090000000000000000000000000000000000070
:10F0A0000000000000000000000000000000000060
:10F0B0000000000000000000000000000000000050
:10F0C0000000000000000000000000000000000040
:10F0D0000000000000000000000000000000000030
:10F0E0000000000000000000000000000000000020
:10F0F0000000000000000000000000000000000010
:10F1000000000000000000000000000000000000FF
:10F1100000000000000000000000000000000000EF
:10F1200000000000000000000000000000000000DF
:10F1300000000000000000000000000000000000CF
:10F1400000000000000000000000000000000000BF
:10F1500000000000000000000000000000000000AF
:10F16000000000000000000000000000000000009F
:10F17000000000000000000000000000000000008F
:10F18000000000000000000000000000000000007F
:10F19000000000000000000000000000000000006F
:10F1A000000000000000000000000000000000005F
:10F1B000000000000000000000000000000000004F
:10F1C000000000000000000000000000000000003F
:10F1D000000000000000000000000000000000002F
:10F1E0000000000000000000756D70414D7470411A
:10F1F000000000000000000000000000C16E70412F
:10F20000E76E7041156F7041556F7041936F70419B
:10F21000C56E70417D707041C96E7041CF6E704196
:10F22000D56E70410D7170415D717041E771704133
:10F23000E16E704165727041EB727041DB6E70413E
:10F24000A9737041697370410F747041A373704169
:10F2500000000000000000000000000000000000AE
:10F26000000000000000000000000000000000009E
:10F27000000000000000000000000000000000008E
:10F280000000000000000000658F704100000000D9
:10F290000000000000000000E38F7041FD9170410C
:10F2A0002D92704100000000000000003393704177
:10F2B0000000000037947041819770410000000009
:10F2C000000000000000000000000000010000003D
:10F2D0000000000000080000020000000100000023
:10F2E0000008000002000000100000000000000004
:10F2F00010000000000000000000000000000000FE
:10F3000000100000010000000100000000100000DB
:10F3100001000000200000000000000020000000AC
:10F3200000000000000000000000000000080000D5
:10F3300002000000010000000008000002000000C0
:10F34000100000000000000010000000000000009D
:10F3500000000000000000000002000002000000A9
:10F360000100000000020000020000000400000094
:10F370000000000004000000000000000000000089
:10F380000000000005020000010000000100000074
:10F390000502000001000000040000000000000061
:10F3A00004000000000000000000000074E670414E
:10F3B00094E67041B4E67041D4E67041000000006C
:10F3C000000800000100000001000000000800002B
:10F3D000010000001000000000000000100000000C
:10F3E0000000000000000000000000000008000015
:10F3F0000200000001000000000800000200000000
:10F4000010000000000000001000000000000000DC
:10F4100000000000080000000000000001000000E3
:10F4200000060000BCF3704148394441324747317F
:10F43000474A414D4352000000000000ADAA0000C1
:10F44000000000000008000040000000000800006C
:10F450004000000064000000FF0000000100000008
:10F46000010000000000000010000000000000008B
:10F470000100000001020000E8F370414D543239F0
:10F48000463447313641424300000000000000008E
:10F490002CBC000000000000001000004000000034
:10F4A000000800004000000064000000FF000000B1
:10F4B000010000000100C001000000000800000081
:10F4C000000000000100000000020000BCF37041D9
:10F4D0004D54323946344730384142430000000031
:10F4E000000000002CAC0000000000000010000034
:10F4F0004000000000080000400000006400000020
:10F50000FF000000010000000100000000000000FA
:10F5100010000000000000000100000001020000D7
:10F52000E8F370414D543239463247313641424456
:10F5300000000000000000002CBA000000000000E5
:10F54000000800004000000000080000400000002B
:10F5500064000000FF000000010000000100000046
:10F560000000000008000000000000000100000092
:10F5700000020000BCF370414D543239463247302E
:10F580003841424400000000000000002CAA0000A6
:10F59000000000000008000040000000000800001B
:10F5A0004000000064000000FF00000001000000B7
:10F5B0000100000000000000080000000000000042
:10F5C0000100000000060000BCF37041464D3641CA
:10F5D00044324731474100000000000000000000B5
:10F5E000C8AA000000000000000800004000000061
:10F5F000000800004000000064000000FF00000060
:10F6000001000000040000000000000008000000ED
:10F61000000000000100000000060000BCF3704183
:10F620004A5346424178324E373241427800000018
:10F630000000000001AA0000000000000008000017
:10F6400040000000000800004000000064000000CE
:10F65000FF000000010000000100000000000000A9
:10F66000080000000000000001000000000600008B
:10F67000BCF370414D44354E30324730314753442E
:10F68000314100000000000098AA000000000000C6
:10F69000000800004000000000080000800000009A
:10F6A00064000000FF0000000100000008000000EE
:10F6B0000000000002000000000000000800000040
:10F6C00014F47041ACF3704102000000010000002E
:10F6D0000800000014F47041ACF370410000000019
:10F6E000000000000000000000000000000000001A
:10F6F0000000000000000000000000000000548036
:10F700001C000400100D0042030000000100000076
:10F71000F4E670410100000004E7704101000000C0
:10F7200014E7704104000000A4E7704104000000E9
:10F7300064E770410400000024E770410400000009
:10F7400064E870410400000024E8704104000000F7
:10F75000E4E7704108000000A4E9704108000000DF
:10F7600024E9704108000000A4E87041080000008E
:10F7700024EB704108000000A4EA7041080000007A
:10F7800024EA704101FF00000100000000000000B9
:10F790000000000000010000013000000000000037
:10F7A00000000000000000000000000001650000F3
:10F7B0000000000000000000000000000000000049
:10F7C0000100000005000000010000000000000032
:10F7D00000000000023000000000000000000000F7
:10F7E000000000000201000001FF00000100000015
:10F7F00000000000000000000001000001FF000008
:10F8000001000000000000000000000000010000F6
:10F81000015A00000000000000000000000000008D
:10F820000000000001B50000000000000000000022
:10F8300000000000000000000100000005000000C2
:10F840000100000000000000000000000230000085
:10F8500000000000000000000000000002010000A5
:10F8600001FF000001000000000000000000000097
:10F870000001000001FF0000010000000000000086
:10F88000000000000001000001AF000005000000C2
:10F890000100000000000000000000000230000035
:10F8A0000000000000000000000000000201000055
:10F8B00001FF000001000000000000000000000047
:10F8C0000001000001000000050000000100000030
:10F8D0003C0000000000000001ED000001000000FD
:10F8E0000200000000000000020000001000000004
:10F8F0000200000055AA00001000000000000000F7
:10F90000FF0000000600000084F77041ECF8704131
:10F9100006000000FCF77041ECF8704104000000A4
:10F9200074F87041F8F8704101000000C4F87041AB
:10F93000ECF8704101000000D8F87041F8F870410F
:08F940000000000000000000BF
:040000054170000046
:00000001FF
